:100000000C948D090C94B5090C94B5090C94B509A0
:100010000C94B5090C94B5090C94B5090C94B50968
:100020000C94B5090C94B5090C94B5090C94B50958
:100030000C94B5090C943C500C94B5090C94B5097A
:100040000C94B5090C9436610C947D290C94B50977
:100050000C94312B0C94B5090C94B5090C94B5098A
:100060000C94B5090C94B5090C94B5090C94B50918
:10007000084AD73B3BCE016E84BCBFFDC12F3D6C0F
:1000800074319ABD56833DDA3D00C77F11BED9E475
:10009000BB4C3E916BAAAABE000000803F05A84C55
:1000A000CDB2D44EB93836A9020C50B99186880821
:1000B0003CA6AAAA2ABE000000803F6563686F3A8A
:1000C00000656E717565696E672022002200737489
:1000D00061727400506F77657255700020457874B6
:1000E00065726E616C205265736574002042726F98
:1000F000776E206F757420526573657400205761A8
:10010000746368646F672052657365740020536F71
:10011000667477617265205265736574004D617213
:100120006C696E2000312E302E3000204C617374CB
:1001300020557064617465643A2000323031322D8C
:1001400030352D303200207C20417574686F723A52
:1001500020006572696B002046726565204D656DF3
:100160006F72793A20002020506C616E6E65724289
:10017000756666657242797465733A20006F6B002C
:10018000446F6E6520736176696E672066696C6581
:100190002E004572726F723A004C696E65204E7582
:1001A0006D626572206973206E6F74204C61737488
:1001B000204C696E65204E756D6265722B312C2066
:1001C0004C617374204C696E653A00636865636BBB
:1001D00073756D206D69736D617463682C204C615B
:1001E0007374204C696E653A004E6F2043686563F6
:1001F0006B73756D2077697468206C696E65206E0D
:10020000756D6265722C204C617374204C696E654B
:100210003A004E6F204C696E65204E756D626572B6
:10022000207769746820636865636B73756D2C2033
:100230004C617374204C696E653A006F6B005072AC
:10024000696E7465722073746F7070656420647574
:100250006520746F206572726F72732E2046697804
:1002600020746865206572726F7220616E642075FB
:100270007365204D39393920746F2072657374614C
:100280007274212E202854656D70657261747572C8
:10029000652069732072657365742E205365742020
:1002A0006974206265666F7265207265737461722D
:1002B00074696E672900446F6E65207072696E7490
:1002C000696E672066696C6500426567696E2066C5
:1002D000696C65206C69737400456E642066696C96
:1002E00065206C697374006F6B20543A00202F00F6
:1002F00020423A00202F0020403A002042403A009D
:10030000543A0020453A0020573A00543A0020451C
:100310003A0020423A004649524D574152455F4EFD
:10032000414D453A4D61726C696E2056313B205308
:100330007072696E7465722F6772626C206D617382
:1003400068757020666F722067656E362046495268
:100350004D574152455F55524C3A687474703A2F6C
:100360002F7777772E6D656E64656C2D7061727472
:10037000732E636F6D2050524F544F434F4C5F5656
:10038000455253494F4E3A312E30204D4143484952
:100390004E455F545950453A4D656E64656C204535
:1003A000585452554445525F434F554E543A310AC2
:1003B00000583A00593A005A3A00453A0020436F33
:1003C000756E7420583A00593A005A3A00785F6DB9
:1003D000696E3A2000795F6D696E3A20007A5F6D30
:1003E000696E3A2000556E6B6E6F776E20636F6D8D
:1003F0006D616E643A2200220000000000000000DF
:1004000000000000000000000000000000000000EC
:100410000000004D4300004D430000F042FFFFFF8D
:100420000000A0400000A0400000803F00004D43BD
:1004300000004D430000F0425374657073207065F6
:100440007220756E69743A0020204D3932205800B0
:10045000205900205A002045004D6178696D756D66
:100460002066656564726174657320286D6D2F73F5
:10047000293A0020204D32303320580020590020E6
:100480005A002045004D6178696D756D20416363A8
:10049000656C65726174696F6E20286D6D2F7332A3
:1004A000293A0020204D32303120580020590020B8
:1004B0005A00204500416363656C65726174696F21
:1004C0006E3A20533D616363656C65726174696F58
:1004D0006E2C20543D726574726163742061636395
:1004E000656C65726174696F6E0020204D32303426
:1004F000205300205400416476616E636564207669
:1005000061726961626C65733A20533D4D696E207A
:10051000666565647261746520286D6D2F73292C82
:1005200020543D4D696E2074726176656C2066655D
:1005300065647261746520286D6D2F73292C2042CB
:100540003D6D696E696D756D207365676D656E745F
:100550002074696D6520286D73292C20583D6D61CC
:1005600078696D756D207859206A65726B20286DE9
:100570006D2F73292C20205A3D6D6178696D756D42
:10058000205A206A65726B20286D6D2F7329002018
:10059000204D323035205300205400204200205896
:1005A00000205A00204500486F6D65206F66667315
:1005B000657420286D6D293A0020204D3230362098
:1005C0005800205900205A00504944207365747423
:1005D000696E67733A002020204D3330312050007F
:1005E000204900204400526573656E643A006F6BC9
:1005F000005072696E7465722068616C7465642E57
:10060000206B696C6C28292063616C6C6564202107
:1006100021005072696E7465722073746F7070651A
:10062000642064756520746F206572726F72732E1A
:100630002046697820746865206572726F72206147
:100640006E6420757365204D39393920746F2072BE
:10065000657374617274212E202854656D70657203
:1006600061747572652069732072657365742E20DC
:10067000536574206974206265666F7265207265C7
:100680007374617274696E6729007C3C3E5E2B3D19
:100690003F2F5B5D3B2C2A225C006563686F3A004C
:1006A00020636F6C6420657874727573696F6E2057
:1006B00070726576656E7465640020746F6F206C6F
:1006C0006F6E6720657874727573696F6E207072D3
:1006D0006576656E746564006563686F3A00656E83
:1006E0006473746F7073206869743A200020583AFC
:1006F0000020593A00205A3A0024F427D3FD204D17
:100700000FB0119A05160CE9022D09C801650733CF
:10071000013206DE005405A700AD0483002A0469F7
:1007200000C10356006B03480023033D00E6023579
:1007300000B1022D00840228005C0223003902204F
:100740000019021C00FD011900E4011700CD01157C
:1007500000B8011300A50111009401100084010FDD
:100760000075010E0067010D005A010C004E010BCF
:100770000043010A0039010A002F0109002601097E
:10078000001D010800150107000E01080006010701
:1007900000FF000600F9000600F3000600ED000669
:1007A00000E7000500E2000500DD000500D80005B7
:1007B00000D3000400CF000500CA000400C60004F6
:1007C00000C2000400BE000300BB000400B7000329
:1007D00000B4000300B1000400AD000300AA000350
:1007E00000A7000200A5000300A20003009F000272
:1007F000009D0003009A000200980003009500028B
:100800000093000200910002008F0002008D0002A0
:10081000008B0002008900020087000200850002B0
:10082000008300020081000100800002007E0002BF
:10083000007C0001007B00020079000100780002CA
:1008400000760001007500010074000200720001D2
:100850000071000100700002006E0001006D0001D7
:10086000006C0001006B00020069000100680001DB
:1008700000670001006600010065000100640001DE
:1008800000630001006200010061000100600001DE
:10089000005F0001005E0001005D0001005C0001DE
:1008A000005B0000005B0001005A000100590001DC
:1008B00000580001005700000057000100560001D9
:1008C00000550001005400000054000100530001D5
:1008D00000520001005100000051000100500001D1
:1008E000004F0000004F0001004E0000004E0001CC
:1008F000004D0001004C0000004C0001004B0000C6
:10090000004B0001004A00010049000000490001BD
:1009100000480000004800010047000000470001B7
:1009200000460000004600010045000000450001AF
:1009300000440000004400010043000000430001A7
:1009400000420000004200010041000000410000A0
:10095000004100010040000000400001003F000095
:10096000003F0001003E0000003E0000003E00018C
:10097000003D0000003D0001003C0000003C000084
:10098000003C0001003B0000003B0000003B000178
:10099000003A0000003A0000003A0001003900006F
:1009A0000039000000390001003800000038000064
:1009B0000038000100370000003700000037000158
:1009C000003600000036000000360001003500004F
:1009D0000035000000350000003500010034000043
:1009E0000034000000340001003300000033000038
:1009F000003300000033000100320000003200002C
:100A0000003200000032000100310000003100001F
:100A10000031000000310001003000000030000013
:100A20000030000000300001002F0000002F000007
:100A3000002F0000002F0001002E0000002E0000FB
:100A4000002E0000002E0000002E0001002D0000EE
:100A5000002D0000002D0000002D0001002C0000E2
:100A6000002C0000002C0000002C0000002C0001D5
:100A7000002B0000002B0000002B0000002B0000CA
:100A8000002B0001002A0000002A0000002A0000BC
:100A9000002A0000002A0000002A000100290000AE
:100AA00000290000002900000029000000290000A2
:100AB0000029000100280000002800000028000094
:100AC0000028000000280001002700000027000087
:100AD000002700000027000000270000002700007A
:100AE000002700010026000000260000002600006C
:100AF00000260000002600000024F4B12873CB116A
:100B00001D62AECC159698F410A287900D127A193A
:100B10000BF96E4009B965D307E65DB5063157D0CC
:100B200005615116054B4C7D04CE47FD03D1439220
:100B3000033F403603093DE902203AA4027C376AAC
:100B40000212353602DC320802D430E101F32EBD48
:100B500001362D9E01982B8101172A6701B028507C
:100B60000160273B0125262801FD241601E7230704
:100B700001E022F800E821EB00FD20DE001F20D379
:100B8000004C1FC800841EBF00C51DB500101DAD60
:100B900000631CA500BE1B9E00201B9700891A91B4
:100BA00000F8198A006E198500E9187F006A187B21
:100BB00000EF1776007917710008176D009B166A11
:100BC0000031166500CC1562006A155F000B155BDD
:100BD00000B01458005814560002145200B01350BC
:100BE0000060134E0012134B00C71249007E1246DC
:100BF0000038124500F3114300B011400070113F5E
:100C00000031113D00F4103C00B8103A007E10385D
:100C100000461037000F103500DA0F3400A60F33EE
:100C200000730F3100420F3000120F3000E20E2D22
:100C300000B50E2D00880E2C005C0E2B00310E2A04
:100C400000070E2800DF0D2800B70D2700900D26A5
:100C5000006A0D2600440D2400200D2400FC0C2306
:100C600000D90C2200B70C2200950C2100740C2036
:100C700000540C1F00350C1F00160C1F00F70B1E34
:100C800000D90B1D00BC0B1C00A00B1C00840B1C0E
:100C900000680B1B004D0B1B00320B1A00180B19C0
:100CA00000FF0A1900E60A1900CD0A1800B50A1853
:100CB000009D0A1800850A17006E0A1600580A16C9
:100CC00000420A16002C0A1600160A1500010A1521
:100CD00000EC091400D8091400C4091400B0091468
:100CE000009C091300890913007609130063091297
:100CF00000510912003F0912002D0911001C0912B0
:100D0000000A091100F9081000E9081100D80810BC
:100D100000C8081000B8081000A808100098080FB4
:100D20000089080F007A080F006B080F005C080F9D
:100D3000004D080E003F080E0031080E0023080E7B
:100D40000015080E0007080D00FA070D00ED070D4D
:100D500000E0070D00D3070D00C6070D00B9070C12
:100D600000AD070C00A1070D0094070B0089070CCC
:100D7000007D070C0071070C0065070B005A070B7C
:100D8000004F070B0044070B0039070B002E070B21
:100D90000023070B0018070A000E070B0003070AC1
:100DA00000F9060A00EF060A00E5060A00DB060A5B
:100DB00000D1060900C8060A00BE060900B5060AE9
:100DC00000AB060900A20609009906090090060971
:100DD00000870609007E060900750609006C0608F2
:100DE00000640609005B060800530609004A06086D
:100DF00000420608003A060800320608002A0608E3
:100E000000220608001A060800120607000B060852
:100E10000003060800FB050700F4050800EC0507C1
:100E200000E5050700DE050700D7050700D0050728
:100E300000C9050700C2050700BB050700B4050788
:100E400000AD050700A6050600A0050700990507E7
:100E500000920506008C050600860507007F050642
:100E60000079050600730507006C05060066050697
:100E700000600506005A050600540506004E0506EA
:100E80000048050600420505003D05060037050639
:100E900000310505002C0506002605050021050684
:100EA000001B05050016050600100505000B0505CD
:100EB000000605060000050500FB040500F6040514
:100EC00000F1040500EC040500E7040500E2040558
:100ED00000DD040500D8040500D3040500CE040598
:100EE00000C9040500C4040500BF040400BB0405D8
:100EF00000B6040500B104050020626961733A2060
:100F00000020643A2000206D696E3A2000206D6157
:100F1000783A2000204B753A20002054753A200082
:100F200020436C61736963205049442000204B705A
:100F30003A2000204B693A2000204B643A200050B0
:100F40004944204175746F74756E65206661696CE3
:100F50006564212054656D706572617475726520D9
:100F6000746F2068696768006F6B20423A006F6B8E
:100F700020543A0020403A00504944204175746F93
:100F800074756E65206661696C6564212074696D95
:100F9000656F757400504944204175746F74756EA7
:100FA000652066696E6973686564202120506C61F4
:100FB000636520746865204B702C204B6920616E3E
:100FC00064204B6420636F6E7374616E7473206968
:100FD0006E2074686520636F6E66696775726174F0
:100FE000696F6E2E68004572726F723A00202D2074
:100FF000496E76616C696420657874727564657297
:10100000206E756D62657221001000C90210012CFE
:10101000014001220170011801B0010E01F001042C
:10102000015002FA00B002F0003003E600D003DC09
:10103000009004D2007005C800A006BE000008B4ED
:1010400000B009AA00D00BA000600E960060118CC1
:10105000000015820020197800C01D6E00A02264D7
:1010600000B0275A00902C500000314600E0343C7C
:101070000010383200903A2800603C1E00A03D1459
:1010800000803E0A00203F0000202D20496E76613E
:101090006C6964206578747275646572206E756D14
:1010A0006265722021003A20457874727564657219
:1010B000207377697463686564206F66662E204DBF
:1010C000415854454D502074726967676572656474
:1010D0002021003A20457874727564657220737718
:1010E000697463686564206F66662E204D494E54AE
:1010F000454D5020747269676765726564202100F0
:1011000054656D706572617475726520686561748F
:101110006564206265642073776974636865642020
:101120006F66662E204D415854454D5020747269AB
:10113000676765726564202121006563686F3A0006
:10114000534420696E6974206661696C004572724F
:101150006F723A00766F6C756D652E696E697420DA
:101160006661696C6564006F70656E526F6F7420A4
:101170006661696C65640053442063617264206F2A
:101180006B006F70656E206661696C65642C20462B
:10119000696C653A20002E0046696C65206F7065A9
:1011A0006E65643A002053697A653A0046696C6559
:1011B0002073656C6563746564006F70656E20668E
:1011C00061696C65642C2046696C653A20002E00CC
:1011D0006F70656E206661696C65642C2046696C71
:1011E000653A20002E0057726974696E6720746F2B
:1011F0002066696C653A20006F70656E20666169D3
:101200006C65642C2046696C653A20002E004669A6
:101210006C652064656C657465643A0044656C6552
:1012200074696F6E206661696C65642C2046696C18
:10123000653A20002E005344207072696E74696E06
:1012400067206279746520002F004E6F742053442C
:10125000207072696E74696E67006572726F7220B9
:1012600077726974696E6720746F2066696C6500B7
:101270000000000102000000000000000403070657
:10128000000000000000000000000000000000005E
:101290000102040810204080010204081020408050
:1012A0000102040810204080804020100804020140
:1012B00002020202020202020404040404040404FE
:1012C00003030303030303030101010101010101FE
:1012D000002225282B002124272A494E46494E4921
:1012E00054594E414E000020410000C84200401CAD
:1012F0004620BCBE4CCA1B0E5AAEC59D74CDCCCC8C
:101300003D0AD7233C17B7D13877CC2B329595E6D9
:10131000241FB14F0A007529792911241FBECFEF70
:10132000D0E1DEBFCDBF13E0A0E0B1E0EEEEF0EF24
:1013300002C005900D92AA32B107D9F71EE0AAE2C9
:10134000B3E001C01D92A33BB107E1F713E1C8E18F
:10135000D3E104C02297FE010E949972C631D107E1
:10136000C9F70E9446290C946A780C940000FC018D
:101370004591559165917491E52F362F272F642F54
:101380007E2F832F922F0895CF92DF92EF92FF92BC
:101390000F931F93CF93DF93EC01CC0FDD1FCC0F86
:1013A000DD1FCE0187509C4F0E94B709FE01E75C0C
:1013B000FC4FC080D180E280F3808E010B5B1C4F1C
:1013C000A70196010E948E6DF8016083718382836C
:1013D0009383CE018B5F9B4F0E94B7098E01035D03
:1013E0001C4FA70196010E948E6DF80160837183E6
:1013F00082839383CE018F5E9B4F0E94B709CA5FA1
:10140000DE4FA70196010E948E6D688379838A83DF
:101410009B83DF91CF911F910F91FF90EF90DF9011
:10142000CF9008952F923F924F925F926F927F924A
:101430008F929F92AF92BF92CF92DF92EF92FF92E4
:101440000F931F93CF93DF9300D000D000D0CDB780
:10145000DEB79C838B835C01AA0CBB1CAA0CBB1C53
:1014600025E4222E23E0322E2A0C3B1CD1011D92B2
:101470001D921D921C92139721E533E04DE453E039
:1014800069E473E085E493E00E94E44EC501845D65
:101490009B4F0E94B709EB81FC81E35EFB4F749088
:1014A000F501E650FA4FFA83E98320E030E040ECA2
:1014B0005FE30E943C716B017C01672D772767FD1C
:1014C0007095872F972F0E94096F2B013C019B017C
:1014D000AC01C701B6010E943C71A981BA816D932C
:1014E0007D938D939C931397F501EA5EFE4FFE83E7
:1014F000ED83608171818281938160932601709375
:101500002701809328019093290120E030E040E7F3
:1015100052E40E946E6E3CE2C32E33E0D32E7B0178
:101520008C0126E036E042E056E06EEF75E08AEF8F
:1015300095E00E947B440E948056D1011D921D922D
:101540001D921C92139721E533E04DE453E069E4CA
:1015500073E085E493E00E94E44EC501805E9B4FFA
:101560000E94B7094B015C019058A30192010E94AF
:101570003C71E981FA81608371838283938320E0E7
:1015800030E040E752E4609126017091270180919C
:101590002801909129010E946E6E7B018C0126E04A
:1015A00036E042E056E06EEF75E08AEF95E00E948B
:1015B0007B440E948056A5019401C501B4010E949C
:1015C0008E6DA30192010E943C71A981BA816D9335
:1015D0007D938D939C93139720E030E040E05FE390
:1015E000ED81FE8160817181828193810E943C71D5
:1015F000FB01462F5F2F682F792F409326015093D0
:101600002701609328017093290120E030E040E732
:1016100052E4BF010E946E6E7B018C0126E036E031
:1016200042E056E06EEF75E08AEF95E00E947B4461
:101630000E9480568B819C810E94C409F1018081A7
:101640009181A281B381E981FA8180839183A28310
:10165000B383109226011092270110922801109254
:10166000290126960FB6F894DEBF0FBECDBFDF91DD
:10167000CF911F910F91FF90EF90DF90CF90BF908F
:10168000AF909F908F907F906F905F904F903F9022
:101690002F900C942C50AF92BF92CF92DF92EF928A
:1016A000FF920F931F93CF93DF93CDB7DEB7E097F1
:1016B0000FB6F894DEBF0FBECDBF80E1E5E5F1E0E7
:1016C000DE01919601900D928A95E1F780E1E5E6C1
:1016D000F1E0DE01519601900D928A95E1F780E1EB
:1016E000E5E7F1E0DE01119601900D928A95E1F7B0
:1016F0006E0181E2C80ED11C4FEDE42E4DE0F42EB8
:101700008E010F5E1F4F6FEE7DE0AE014F5F5F4FAA
:10171000EFECAE2EEDE0BE2E20E030E0F601819140
:101720009191A191B1916F01F70181939193A1934F
:10173000B1937F01F80181919191A191B1918F01B4
:10174000FB0181939193A193B193BF01FA01819120
:101750009191A191B191AF01F50181939193A193E1
:10176000B1935F012F5F3F4F24303105B9F680E020
:1017700090E0AAEFB4E48093C70D9093C80DA093B6
:10178000C90DB093CA0D8093C30D9093C40DA0935F
:10179000C50DB093C60D1092CB0D1092CC0D1092CA
:1017A000CD0D1092CE0D80E29EE4A0E0B0E08093DB
:1017B000FF0D9093000EA093010EB093020E1092B5
:1017C000B30D1092B40D1092B50D1092B60D80E0CD
:1017D00090E0A0EAB1E48093BF0D9093C00DA09378
:1017E000C10DB093C20D8DEC9CECACECBEE38093CC
:1017F000BB0D9093BC0DA093BD0DB093BE0D80E0CA
:1018000090E0A0EAB0E48093B70D9093B80DA09358
:10181000B90DB093BA0D1092410310924203109289
:1018200043031092440310923D0310923E03109222
:101830003F03109240031092390310923A03109222
:101840003B0310923C03EBEBF0E007C09091C0002B
:1018500095FFFCCF8093C600319684918111F6CF1D
:10186000E5E8F1E006C09091C00095FFFCCF8093C1
:10187000C60081918111F7CF8091C00085FFFCCF18
:101880008AE08093C600E0960FB6F894DEBF0FBEE4
:10189000CDBFDF91CF911F910F91FF90EF90DF901F
:1018A000CF90BF90AF90089507C03091C00035FF32
:1018B000FCCF2093C6000196FC0124912111F5CFA5
:1018C00022E030E08DE296E00C946E2D07C030915E
:1018D000C00035FFFCCF2093C6000196FC01249187
:1018E0002111F5CF22E030E08DE296E00C946E2DD0
:1018F00007C03091C00035FFFCCF2093C600019691
:10190000FC0124912111F5CF2AE030E08DE296E030
:101910000C94522CCF93DF93CBEBD0E0FE0107C0A9
:101920009091C00095FFFCCF8093C60031968491C2
:101930008111F6CFE8E3F4E007C09091C00095FF75
:10194000FCCF8093C600319684918111F6CF8091AF
:10195000C00085FFFCCF8AE08093C600FE01849121
:10196000EBEBF0E008C09091C00095FFFCCF8093B6
:10197000C600319684918111F6CF4091DF0D5091D0
:10198000E00D6091E10D7091E20D88E494E00E9419
:10199000540C4091E30D5091E40D6091E50D709170
:1019A000E60D80E594E00E94540C4091E70D5091C3
:1019B000E80D6091E90D7091EA0D83E594E00E94D5
:1019C000540C4091EB0D5091EC0D6091ED0D709128
:1019D000EE0D86E594E00E94540C8091C00085FFD6
:1019E000FCCF8AE08093C600FE018491EBEBF0E02F
:1019F00008C09091C00095FFFCCF8093C60031963F
:101A000084918111F6CFE9E5F4E007C09091C00020
:101A100095FFFCCF8093C600319684918111F6CF5B
:101A20008091C00085FFFCCF8AE08093C600FE0154
:101A30008491EBEBF0E008C09091C00095FFFCCFE3
:101A40008093C600319684918111F6CF4091EF0DBD
:101A50005091F00D6091F10D7091F20D83E794E0DB
:101A60000E94540C4091F30D5091F40D6091F50DCE
:101A70007091F60D8CE794E00E94540C4091F70DA4
:101A80005091F80D6091F90D7091FA0D8FE794E087
:101A90000E94540C4091FB0D5091FC0D6091FD0D86
:101AA0007091FE0D82E894E00E94540C8091C00079
:101AB00085FFFCCF8AE08093C600FE018491EBEBAA
:101AC000F0E008C09091C00095FFFCCF8093C60065
:101AD000319684918111F6CFE5E8F4E007C090914A
:101AE000C00095FFFCCF8093C60031968491811190
:101AF000F6CF8091C00085FFFCCF8AE08093C600BE
:101B0000FE018491EBEBF0E008C09091C00095FFDE
:101B1000FCCF8093C600319684918111F6CF40911D
:101B2000CF0D5091D00D6091D10D7091D20D83EAFF
:101B300094E00E94780C4091D30D5091D40D6091A7
:101B4000D50D7091D60D8CEA94E00E94780C4091EE
:101B5000D70D5091D80D6091D90D7091DA0D8FEAA3
:101B600094E00E94780C4091DB0D5091DC0D609167
:101B7000DD0D7091DE0D82EB94E00E94780C809177
:101B8000C00085FFFCCF8AE08093C600FE018491EF
:101B9000EBEBF0E008C09091C00095FFFCCF809384
:101BA000C600319684918111F6CFE5EBF4E007C0D1
:101BB0009091C00095FFFCCF8093C6003196849130
:101BC0008111F6CF8091C00085FFFCCF8AE0809321
:101BD000C600FE018491EBEBF0E008C09091C000DC
:101BE00095FFFCCF8093C600319684918111F6CF8A
:101BF0004091C70D5091C80D6091C90D7091CA0DEB
:101C00008AEE94E00E94540C4091C30D5091C40D93
:101C10006091C50D7091C60D83EF94E00E94540C45
:101C20008091C00085FFFCCF8AE08093C600FE0152
:101C30008491EBEBF0E008C09091C00095FFFCCFE1
:101C40008093C600319684918111F6CFE6EFF4E0DF
:101C500007C09091C00095FFFCCF8093C6003196DD
:101C600084918111F6CF8091C00085FFFCCF8AE07E
:101C70008093C600FE018491EBEBF0E008C09091E8
:101C8000C00095FFFCCF8093C600319684918111EE
:101C9000F6CF4091CB0D5091CC0D6091CD0D709150
:101CA000CE0D8FE895E00E94540C4091B30D5091F9
:101CB000B40D6091B50D7091B60D88E995E00E9464
:101CC000540C4091FF0D5091000E6091010E7091E7
:101CD000020E8BE995E00E94780C4091BF0D509167
:101CE000C00D6091C10D7091C20D8EE995E00E940A
:101CF000540C4091BB0D5091BC0D6091BD0D709185
:101D0000BE0D81EA95E00E94540C4091B70D5091B0
:101D1000B80D6091B90D7091BA0D84EA95E00E94FA
:101D2000540C8091C00085FFFCCF8AE08093C600F0
:101D3000FE018491EBEBF0E008C09091C00095FFAC
:101D4000FCCF8093C600319684918111F6CFE7EAEB
:101D5000F5E007C09091C00095FFFCCF8093C600CE
:101D6000319684918111F6CF8091C00085FFFCCF20
:101D70008AE08093C600FE018491EBEBF0E008C09E
:101D80009091C00095FFFCCF8093C600319684915E
:101D90008111F6CF4091390350913A0360913B0392
:101DA00070913C0389EB95E00E94540C40913D03F7
:101DB00050913E0360913F037091400382EC95E0A7
:101DC0000E94540C4091410350914203609143039F
:101DD0007091440385EC95E00E94540C8091C00002
:101DE00085FFFCCF8AE08093C600FE018491EBEB77
:101DF000F0E008C09091C00095FFFCCF8093C60032
:101E0000319684918111F6CFE8ECF5E007C090910E
:101E1000C00095FFFCCF8093C6003196849181115C
:101E2000F6CF8091C00085FFFCCF8AE08093C6008A
:101E3000FE01C491EBEBF0E008C08091C00085FF8B
:101E4000FCCFC093C6003196C491C111F6CF40912A
:101E50004C0150914D0160914E0170914F0186ED02
:101E600095E00E94540C25E93FEB46ED5DE360915F
:101E700048017091490180914A0190914B010E9463
:101E80006E6EAB01BC0180EE95E00E94660C25E908
:101E90003FEB46ED5DE36091440170914501809117
:101EA0004601909147010E943C71AB01BC0183EE59
:101EB00095E00E94660C8091C00085FFFCCF8AE00F
:101EC0008093C600DF91CF910895CF93DF9300D028
:101ED000CDB7DEB78091AD0E9091AE0E9E012F5F13
:101EE0003F4F009719F4235B3E4002C0281B390B7B
:101EF0003A83298389819A810F900F90DF91CF9146
:101F000008952091520430915304243031050CF08F
:101F10006AC0409154045091550460E6649F90015A
:101F2000659F300D1124BC01C9018A5A9B4F0E9444
:101F30005475EBEBF0E007C09091C00095FFFCCF2B
:101F40008093C600319684918111F6CFE1ECF0E0E8
:101F500007C09091C00095FFFCCF8093C6003196DA
:101F600084918111F6CF809154049091550420E61C
:101F7000289FF001299FF00D1124EA5AFB4F06C05B
:101F80009091C00095FFFCCF8093C6008191811194
:101F9000F7CFECECF0E007C09091C00095FFFCCFCC
:101FA0008093C600319684918111F6CF8091C00054
:101FB00085FFFCCF8AE08093C60080915404909105
:101FC0005504019664E070E00E94257290935504D8
:101FD00080935404809152049091530401969093FD
:101FE0005304809352040895CF92DF92EF92FF92B0
:101FF0000F931F93CF93DF9300D000D0CDB7DEB700
:1020000040E052EC61E070E08DE296E00E94662BC9
:10201000EEECF0E007C09091C00095FFFCCF8093FC
:10202000C600319684918111F6CF8091C00085FF62
:10203000FCCF8AE08093C6008BEB90E0FC0107C0E8
:102040003091C00035FFFCCF2093C600319624911B
:102050002111F6CF24B720FF14C0E4EDF0E007C053
:102060004091C00045FFFCCF3093C60031963491BB
:102070003111F6CF3091C00035FFFCCF3AE03093FC
:10208000C60021FF14C0ECEDF0E007C04091C00095
:1020900045FFFCCF3093C600319634913111F6CF15
:1020A0003091C00035FFFCCF3AE03093C60022FFEC
:1020B00014C0ECEEF0E007C04091C00045FFFCCF3B
:1020C0003093C600319634913111F6CF3091C00073
:1020D00035FFFCCF3AE03093C60023FF14C0EDEF8C
:1020E000F0E007C04091C00045FFFCCF3093C60030
:1020F000319634913111F6CF3091C00035FFFCCFCD
:102100003AE03093C60025FF14C0EDE0F1E007C0CF
:102110003091C00035FFFCCF2093C600319624914A
:102120002111F6CF2091C00025FFFCCF2AE020939B
:10213000C60014BEEDE1F1E007C03091C00035FFEC
:10214000FCCF2093C600319624912111F6CFE5E211
:10215000F1E007C03091C00035FFFCCF2093C600EE
:10216000319624912111F6CF2091C00025FFFCCF9C
:102170002AE02093C600FC012491EBEBF0E008C0BC
:102180003091C00035FFFCCF2093C60031962491DA
:102190002111F6CFEBE2F1E007C03091C00035FF2E
:1021A000FCCF2093C600319624912111F6CFEBE3AA
:1021B000F1E007C03091C00035FFFCCF2093C6008E
:1021C000319624912111F6CFE6E4F1E007C0309179
:1021D000C00035FFFCCF2093C60031962491211119
:1021E000F6CFE2E5F1E007C03091C00035FFFCCF4B
:1021F0002093C600319624912111F6CF2091C00082
:1022000025FFFCCF2AE02093C600FC018491EBEB74
:10221000F0E008C09091C00095FFFCCF8093C6000D
:10222000319684918111F6CFE7E5F1E007C09091F6
:10223000C00095FFFCCF8093C60031968491811138
:10224000F6CF0E94650F4AE050E0BC018DE296E0B7
:102250000E94762CE6E6F1E007C09091C00095FF61
:10226000FCCF8093C600319684918111F6CF4AE06D
:1022700050E060ED74E08DE296E00E94762C809153
:10228000C00085FFFCCF8AE08093C6001092D6057F
:102290001092D7051092D8051092D90580E00E94BF
:1022A0004B0BFFECCF2EFDE0DF2EAFEDEA2EADE0C5
:1022B000FA2E03EA1DE0F6016191719181919191ED
:1022C0006F01F70121913191419151917F01298352
:1022D0003A834B835C830E94076F29813A814B814B
:1022E0005C810E943C710E94DB6EF80161937193E6
:1022F000819391938F01FFEDCF16FDE0DF06D9F6B4
:102300000E945C5B0E94B7420F900F900F900F905D
:10231000DF91CF911F910F91FF90EF90DF90CF90C1
:102320000C9434568091E0059091E10560E070E0F6
:1023300001960C949D728091E0059091E1054AE030
:1023400050E060E070E001960C94EA734091DA0589
:102350005091DB0590E6949F9001959F300D1124DC
:10236000682F70E0C9018A5A9B4F0E94497590936B
:10237000E1058093E00521E0892B09F420E0822F1C
:1023800008950E94C2296093F2057093F30580932B
:10239000F4059093F505E091DA05F091DB05EA523A
:1023A000FA4F8081811114C0EEEEF5E007C09091E4
:1023B000C00095FFFCCF8093C600319684918111B7
:1023C000F6CF8091C00085FFFCCF8AE08093C600E5
:1023D00008958DE296E00E94AB2BE6EEF5E007C093
:1023E0009091C00095FFFCCF8093C60031968491F8
:1023F0008111F6CF4091E6055091E7056091E8051F
:102400007091E9054F5F5F4F6F4F7F4F2AE030E0DB
:102410008DE296E00E94652C8091C00085FFFCCF84
:102420008AE08093C6000C94C1112F923F924F9284
:102430005F926F927F928F929F92AF92BF92CF9254
:10244000DF92EF92FF920F931F93CF93DF93CDB75D
:10245000DEB76F970FB6F894DEBF0FBECDBF40E674
:10246000B42E54E0C52ED12CEEE3F2E094906AE055
:10247000A62EEBE3F2E08490332433948091AE06F1
:102480009091AF062091B0063091B106821B930B5C
:102490008F779927892B09F007C237C38D3051F008
:1024A0008A3321F49091DD05992321F02F353105F0
:1024B0000CF4DDC12115310509F4A2C28091540448
:1024C00090915504B89E8001B99E100D1124F80119
:1024D000E20FF31FEA5AFB4F10822091DD05211114
:1024E000C1C11092DD05FC01EA52FA4F108236E5B7
:1024F000E32E34E0F32EE00EF11E6EE470E0C7012F
:102500000E944975009709F404C19093E1058093F6
:10251000E0058E199F09800F911F4AE050E060E0AE
:1025200070E0895A9B4F0E94EA736093E2057093B2
:10253000E3058093E4059093E5054090E60550900F
:10254000E7056090E8057090E905930182010F5F4F
:102550001F4F2F4F3F4F6017710782079307C1F13D
:102560002091540430915504B29EC001B39E900D49
:1025700011246DE971E08A5A9B4F0E947875892B6E
:1025800039F5E2E9F1E007C09091C00095FFFCCF7A
:102590008093C600319684918111F6CFE9E9F1E08C
:1025A00007C09091C00095FFFCCF8093C600319684
:1025B00084918111F6CF2AE030E0B301A2018DE2CF
:1025C00096E00E94652C8091C00085FFFCCF8AC0F8
:1025D0008091540490915504B89E7001B99EF00CFE
:1025E000112487010A5A1B4F6AE270E0C8010E9459
:1025F0004975009721F450C063262F5F02C020E088
:10260000612CF701E20FF11DEA5AFB4F30813A329B
:1026100099F79093E1058093E005801B910B8E0D57
:102620009F1D60E070E0895A9B4F0E949D720E943E
:10263000D66E262D30E02617370709F459C0E2E997
:10264000F1E007C09091C00095FFFCCF8093C600D9
:10265000319684918111F6CFEBECF1E007C09091B7
:10266000C00095FFFCCF8093C60031968491811104
:10267000F6CF4091E6055091E7056091E80570912D
:10268000E9052AE030E08DE296E00E94652C809119
:10269000C00085FFFCCF26C0E2E9F1E007C09091C1
:1026A000C00095FFFCCF8093C600319684918111C4
:1026B000F6CFE9EEF1E007C09091C00095FFFCCFA6
:1026C0008093C600319684918111F6CF2AE030E0E4
:1026D000B301A2018DE296E00E94652C8091C000BA
:1026E00085FFFCCF8AE08093C6000E94E91147C0B5
:1026F0008091E2059091E305A091E405B091E50594
:102700008093E6059093E705A093E805B093E9056B
:102710003BC06AE270E0C7010E944975892BA1F1B4
:10272000E2E9F1E007C09091C00095FFFCCF8093F3
:10273000C600319684918111F6CFE2E1F2E007C044
:102740009091C00095FFFCCF8093C6003196849194
:102750008111F6CF4091E6055091E7056091E805BB
:102760007091E9052AE030E08DE296E00E94652C48
:102770008091C00085FFFCCF8AE08093C600109254
:10278000DF051092DE05EFC180915404909155044D
:10279000B89E8001B99E100D112426E5E22E24E09A
:1027A000F22EE00EF11E67E470E0C7010E94497549
:1027B000009709F442C09093E1058093E0058E19DB
:1027C0009F09800F911F60E070E0895A9B4F0E9423
:1027D0009D720E94D66E6430710578F580912A034F
:1027E000811117C080915C03811127C0882DEBE314
:1027F000F2E008C09091C00095FFFCCF8093C60026
:10280000319684918111F6CF8091C00085FFFCCF75
:1028100012C0892DEEE3F2E008C09091C00095FF50
:10282000FCCF8093C600319684918111F6CF8091C0
:10283000C00085FFFCCFA092C60080915404909107
:1028400055040196B6010E94257290935504809319
:102850005404809152049091530401969093530430
:10286000809352041092DF051092DE0507CE8B3361
:1028700011F43092DD059091DD059111FFCD40916D
:10288000540450915504B49EF001B59EF00D1124EE
:10289000E20FF31FEA5AFB4F80832F5F3F4F3093C5
:1028A000DF052093DE05EACD809152049091530418
:1028B00004970CF42FC129C18091DE059091DF05AA
:1028C000892B09F4E8C04FC14D3081F04A3321F41F
:1028D0002091DD05222351F02091DE053091DF05A6
:1028E0002F3531051CF4019609F0B8C04091480419
:1028F0005091490460914A0470914B0480914004C6
:1029000090914104A0914204B091430448175907A3
:102910006A077B0708F46DC0842DE6EBF2E008C07F
:102920009091C00095FFFCCF8093C60031968491B2
:102930008111F6CF8091C00085FFFCCF5092C60078
:102940000E94C2296093EA057093EB058093EC0521
:102950009093ED052091EE053091EF054091F00543
:102960005091F105621B730B840B950BA701960127
:102970000E943972CA01B901A50194010E943972FD
:102980007F936F933F932F9382EA91E09F938F936E
:102990001F930F930E9492758F8D0FB6F894DEBF30
:1029A0000FBECDBFEBEBF0E008C09091C00095FFEB
:1029B000FCCF8093C600319684918111F6CFF80147
:1029C00006C09091C00095FFFCCF8093C600819116
:1029D0008111F7CF8091C00085FFFCCF5092C600D7
:1029E0008CE593E00E94BE6A61E08CE593E00E9472
:1029F000B7692091DE053091DF052115310519F405
:102A00001092DD05B0C08091540490915504789ED9
:102A1000F001799EF00D1124E20FF31FEA5AFB4FEB
:102A20001082FC01EA52FA4F6082209152043091E8
:102A300053042F5F3F4F3093530420935204019669
:102A4000B1010E9425729093550480935404109212
:102A5000DD051092DF051092DE053BC04B3311F40B
:102A60006092DD058091DD05811133C080915404B1
:102A700090915504789EF001799EF00D1124E20F9B
:102A8000F31FEA5AFB4F40832F5F3F4F3093DF0520
:102A90002093DE051EC0B0E67B2E6624639414E00E
:102AA000212E312CE6EBF2E044900AE0502E88EE25
:102AB000C82E83E0D82EE12CF12C9CE3892E912C9A
:102AC000A12CB12C8E010F5F1F4FEBEBF0E0349186
:102AD0003F8F409148045091490460914A0470919D
:102AE0004B048091400490914104A0914204B09124
:102AF0004304481759076A077B07A8F580915204D9
:102B0000909153040497A4F02EC080915D0381112D
:102B1000D3CE29C08DE296E00E948F2B8093DC05F6
:102B20002091DE053091DF058A3009F0B7CCC2CCA8
:102B300080912D0490912E04A0912F04B091300427
:102B40008093480490934904A0934A04B0934B04A3
:102B500085E294E00E940530482F8093DC058A309E
:102B600009F0B2CEC3CE6F960FB6F894DEBF0FBE9B
:102B7000CDBFDF91CF911F910F91FF90EF90DF902C
:102B8000CF90BF90AF909F908F907F906F905F900D
:102B90004F903F902F9008958F929F92AF92BF9247
:102BA000CF92DF92EF92FF920F931F93CF93DF9319
:102BB0007CE5E72E72E0F72E05E413E0CAEFD5E0DE
:102BC000E8E5CE2EE3E0DE2EF70181917F010E9441
:102BD000A611882319F10E9492114B015C01F601A4
:102BE0008081811103C060910A0601C061E070E03C
:102BF00080E090E00E94096FF801208131814281DC
:102C000053810E943C719B01AC01C501B4010E943B
:102C10008E6D688379838A839B8309C0F8018081E4
:102C20009181A281B38188839983AA83BB830C5F3E
:102C30001F4F2496FFEFCF1ADF0A80E6E81682E0E6
:102C4000F80611F686E40E94A6118823D9F00E94A6
:102C500092116B017C0160931406709315068093AA
:102C600016069093170620E030E0A9010E946A70D2
:102C7000181644F4C0922601D0922701E092280150
:102C8000F0922901DF91CF911F910F91FF90EF906A
:102C9000DF90CF90BF90AF909F908F9008950E944B
:102CA000CC1589E40E94A611882359F00E94921144
:102CB000609318067093190680931A0690931B066A
:102CC00008C0109218061092190610921A06109257
:102CD0001B068AE40E94A611882359F00E949211D3
:102CE00060931C0670931D0680931E0690931F062A
:102CF000089510921C0610921D0610921E06109246
:102D00001F060895CF92DF92EF92FF92CF93DF9349
:102D1000EC01C0902D03D0902E03E0902F03F09093
:102D20003003A7019601688179818A819B810E9485
:102D3000676E87FF04C0C882D982EA82FB82C09096
:102D40003103D0903203E0903303F0903403A701B5
:102D500096016C817D818E819F810E94676E87FFC5
:102D600004C0CC82DD82EE82FF82C0903503D09019
:102D70003603E0903703F0903803A7019601688589
:102D800079858A859B850E94676E87FF04C0C88607
:102D9000D986EA86FB86C0900601D0900701E090B4
:102DA0000801F0900901A7019601688179818A8163
:102DB0009B810E946A70181624F4C882D982EA8224
:102DC000FB82C0900A01D0900B01E0900C01F090C2
:102DD0000D01A70196016C817D818E819F810E94EA
:102DE0006A70181624F4CC82DD82EE82FF82C090D5
:102DF0000E01D0900F01E0901001F0901101A70199
:102E00009601688579858A859B850E946A70181667
:102E100024F4C886D986EA86FB86DF91CF91FF909D
:102E2000EF90DF90CF900895CF92DF92EF92FF92D4
:102E30000F931F938AEF95E00E9482160E94C22989
:102E40006093F2057093F3058093F4059093F50574
:102E50002091FA053091FB054091FC055091FD054C
:102E60006091450370914603809147039091480318
:102E70000E94676E811173C02091FE053091FF059D
:102E800040910006509101066091490370914A03F8
:102E900080914B0390914C030E94676E81115FC03B
:102EA00020E030E040E752E4609126017091270174
:102EB00080912801909129010E946E6EFCE2CF2E34
:102EC000F3E0DF2E7B018C0126E036E042E056E0A5
:102ED0006EEF75E08AEF95E00E947B448091FA05E1
:102EE0009091FB05A091FC05B091FD0580934503F1
:102EF00090934603A0934703B09348038091FE0547
:102F00009091FF05A0910006B091010680934903BE
:102F100090934A03A0934B03B0934C038091020615
:102F200090910306A0910406B091050680934D038D
:102F300090934E03A0934F03B093500380910606E5
:102F400090910706A0910806B0910906809351035D
:102F500090935203A0935303B09354031FC0609106
:102F6000140170911501882777FD8095982F0E9494
:102F7000096F20912601309127014091280150913D
:102F800029010E943C7120E030E040E752E40E94B9
:102F90006E6E20E030E048EC52E48ECF1F910F912E
:102FA000FF90EF90DF90CF900895AF92BF92CF92B5
:102FB000DF92EF92FF920F931F93CF93DF93D82F5F
:102FC00020911C0630911D0640911E0650911F064F
:102FD000609118067091190680911A0690911B064F
:102FE0000E947770C62F172F082FF92E60911401B9
:102FF00070911501882777FD8095982F0E94096FA1
:1030000020912601309127014091280150912901FA
:103010000E943C7120E030E040E752E40E946E6E76
:1030200020E030E048EC52E40E946E6E20912C03C8
:103030002F93DF93FF920F931F93CF935B016C014C
:10304000A2E0EA2E01E020E048E156E06AEF75E0F8
:1030500085E493E00E94263B8091FA059091FB0560
:10306000A091FC05B091FD05809345039093460324
:10307000A0934703B09348038091FE059091FF050C
:10308000A0910006B09101068093490390934A03F2
:10309000A0934B03B0934C038091020690910306DA
:1030A000A0910406B091050680934D0390934E03C2
:1030B000A0934F03B09350038091060690910706AA
:1030C000A0910806B0910906809351039093520392
:1030D000A0935303B09354030E94C2296093F20556
:1030E0007093F3058093F4059093F5050F900F907E
:1030F0000F900F900F900F90DF91CF911F910F9134
:10310000FF90EF90DF90CF90BF90AF900895F8942C
:103110000E94C15B5A985A985A985A98E2E9F1E08D
:1031200007C09091C00095FFFCCF8093C6003196F8
:1031300084918111F6CFE1EFF5E007C09091C000D6
:1031400095FFFCCF8093C600319684918111F6CF14
:103150008091C00085FFFCCF8AE08093C600FFCF3E
:10316000CF92DF92EF92FF920F931F930E94C2299A
:1031700000910C0610910D0620910E0630910F065D
:10318000C090F205D090F305E090F405F090F505BD
:103190006C197D098E099F0906171707280739073B
:1031A00030F4012B022B032B11F00E948718809121
:1031B0002B0190912C01A0912D01B0912E01892B12
:1031C0008A2B8B2B09F10E94C2290091F2051091E4
:1031D000F3052091F4053091F505601B710B820B0E
:1031E000930B00912B0110912C0120912D01309116
:1031F0002E01061717072807390730F49091C108E8
:103200008091C008981721F00E9430441EBA05C072
:103210005A985A985A985A98F7CF1F910F91FF9041
:10322000EF90DF90CF9008950E94C15B80912A03B8
:10323000811134C081E080932A038091E60590914A
:10324000E705A091E805B091E905809310069093F9
:103250001106A0931206B0931306E2E9F1E007C04D
:103260009091C00095FFFCCF8093C6003196849169
:103270008111F6CFE2E1F6E007C09091C00095FF22
:10328000FCCF8093C600319684918111F6CF809156
:10329000C00085FFFCCF8AE08093C600089580912E
:1032A0002A030895CF93DF93EC0180912C03809340
:1032B0000B0684E50E94A611811102C080E055C072
:1032C0000E9492110E94DB6E60930B066623B1F39D
:1032D000EBEBF0E007C09091C00095FFFCCF80932E
:1032E000C600319684918111F6CFC936D10551F0CF
:1032F000CD36D10521F0C836D10539F506C0E1EB50
:10330000F1E020C0E8ECF1E013C0EFEDF1E006C021
:103310009091C00095FFFCCF8093C60081918111F0
:10332000F7CF13C09091C00095FFFCCF8093C600EB
:1033300081918111F7CF09C09091C00095FFFCCF1A
:103340008093C60081918111F7CF40E050E06091F9
:103350000B068DE296E00E945E2C8091C00085FFF6
:10336000FCCF8AE08093C60081E0DF91CF91089581
:103370002F923F924F925F926F927F928F929F9285
:10338000AF92BF92CF92DF92EF92FF920F931F9373
:10339000CF93DF93CDB7DEB7A2970FB6F894DEBF19
:1033A0000FBECDBF87E40E94A611882309F49FC2F7
:1033B0000E9492110E94D66E64307105D9F144F4D6
:1033C0006230710521F15CF577FF17C00C94D327AB
:1033D0006A35710509F437C234F46C31710511F0A6
:1033E0000C94D32769C06B35710509F430C26C3574
:1033F000710511F00C94D3272FC280912A038111FB
:1034000006C00E94CC150E9414170C94AF2880911E
:103410002A03811104C00E944F1681E007C08091E9
:103420002A03811107C00E944F1680E00E94D51721
:103430000C94AF2880E50E94A611882339F00E94E1
:1034400092110E94DB6E6B017C0103C0C12CD12C58
:10345000760183E50E94A611882361F00E949211F3
:1034600020E030E04AE754E40E943C710E94DB6EA9
:103470006B017C010E9480560E94C2294B015C01B5
:103480008C0C9D1CAE1CBF1C0E94C2296093F205CF
:103490007093F3058093F4059093F50504C00E94A2
:1034A000D3580E94B0180E94C229681579058A0570
:1034B0009B05A8F30C94D3278091260190912701B6
:1034C000A0912801B09129018093F6059093F7050A
:1034D000A093F805B093F90580911401909115011E
:1034E000909357038093560384E690E090931501E0
:1034F000809314010E94C2296093F2057093F30532
:103500008093F4059093F50581E00E9433508091FB
:10351000450390914603A0914703B09148038093DF
:10352000FA059093FB05A093FC05B093FD058091EF
:10353000490390914A03A0914B03B0914C038093AF
:10354000FE059093FF05A0930006B09301068091BD
:103550004D0390914E03A0914F03B091500380937F
:10356000020690930306A0930406B093050680918B
:10357000510390915203A0915303B091540380934F
:10358000060690930706A0930806B09309061092CA
:10359000260110922701109228011092290188E536
:1035A0000E94A611882311F090E00AC089E50E94CC
:1035B000A6118111F9CF8AE50E94A61191E0982702
:1035C00090932A0191110C94D62788E50E94A611A8
:1035D000882309F487C089E50E94A61181110C9403
:1035E000D62780C0C0922601D0922701E092280100
:1035F000F092290120E030E040E752E4609126019A
:103600007091270180912801909129010E946E6E8E
:10361000ACE2CA2EA3E0DA2E7B018C0126E036E074
:1036200042E056E06EEF75E08AEF95E00E947B4441
:103630000E94805680E090E00E94C40981E090E002
:103640000E94C40921E533E04DE453E069E473E0EE
:1036500085E493E00E94E44E8091450390914603F7
:10366000A0914703B09148038093FA059093FB051E
:10367000A093FC05B093FD058091490390914A0306
:10368000A0914B03B0914C038093FE059093FF05EE
:10369000A0930006B093010620E030E040E752E43A
:1036A0006091260170912701809128019091290154
:1036B0000E946E6E7B018C0126E036E042E056E00F
:1036C0006EEF75E08AEF95E00E947B441092260130
:1036D0001092270110922801109229010E94805611
:1036E0000E942C5080912A0181110C94262888E593
:1036F0000E94A61181110C94262880912A01811123
:103700000C942C2889E50E94A61181110C942C2878
:1037100080912A0181110C9432288AE50E94A61119
:1037200081110C94322888E50E94A6118823D1F0DB
:103730000E949B11672B682B692BA1F00E949211AC
:103740002091390330913A0340913B0350913C035F
:103750000E948E6D609345037093460380934703E8
:103760009093480389E50E94A6118823D1F00E9416
:103770009B11672B682B692BA1F00E94921120915D
:103780003D0330913E0340913F03509140030E941E
:103790008E6D6093490370934A0380934B0390931B
:1037A0004C038AE50E94A6118823D1F00E949B1148
:1037B000672B682B692BA1F00E9492112091410385
:1037C0003091420340914303509144030E948E6D17
:1037D00060934D0370934E0380934F039093500377
:1037E00021E533E04DE453E069E473E085E493E0E0
:1037F0000E94E44E80E00E9433508091F605909143
:10380000F705A091F805B091F905809326019093F2
:103810002701A0932801B09329018091560390912C
:10382000570390931501809314010E94C22960935D
:10383000F2057093F3058093F4059093F5050E94CB
:103840002C500C94D32710920A060C94D32781E0B5
:1038500080930A060C94D32785E40E94A611811157
:1038600002C00E948056ECE5CE2EE2E0DE2EF9E3A7
:10387000EF2EF3E0FF2E05E413E0B12CF601819169
:103880006F010E94A611882339F1F3E0BF120CC02A
:103890000E949211F801608371838283938381E592
:1038A00093E00E94804F18C00E949211F70120817E
:1038B0003181428153810E948E6DF8016083718352
:1038C0008283938321E533E04DE453E069E473E0C0
:1038D00085E493E00E94E44EB394F4E0EF0EF11C13
:1038E0000C5F1F4F24E0B212C9CF0C94D3278DE494
:1038F0000E94A611882311F40C9426270E9492118D
:103900000E94D66E6B36710509F405C60CF06FC0C7
:103910006C31710509F46FC19CF56631710509F4CC
:1039200027C1ACF46231710509F4FFC534F461318B
:10393000710511F00C94D327E4C06431710509F4CA
:10394000E6C06531710511F00C94D3270BC16931C4
:10395000710509F436C154F46731710509F40EC1DB
:103960006831710511F00C94D3271BC16A317105C0
:1039700009F42DC16B31710511F00C94D32735C1B9
:103980006435710509F4D1C5CCF46A32710509F4C6
:103990003BC254F46E31710509F462C16F31710597
:1039A00011F00C94D3279AC16235710509F4B6C59C
:1039B0006335710511F00C94D327B3C568367105D2
:1039C00009F45EC254F46535710509F4E9C56C3536
:1039D000710511F00C94D327F9C56936710509F406
:1039E00094C26A36710511F00C94D3276DC56D3CF5
:1039F000710511F40C945325D4F56937710509F458
:103A00005BC7CCF46337710509F46AC654F46D36AC
:103A1000710509F433C36237710511F00C94D32793
:103A20006DC66737710509F469C06837710511F013
:103A30000C94D3273FC7693C710511F40C94DD2425
:103A400054F46C38710509F44CC26E3B710511F0E9
:103A50000C94D3279DC46B3C710511F40C9417256D
:103A60006C3C710511F00C94D3270C9433256F3204
:103A700031E0730711F40C94CD26FCF46D3D710513
:103A800011F40C94DF2564F46E3C710511F40C9470
:103A9000B1256C3D710511F00C94D3270C94CD2504
:103AA0006D3291E0790711F40C94EE256E3271407D
:103AB00011F00C94D3270C94C926663FF1E07F07E0
:103AC00011F40C940A276CF4603931E0730711F497
:103AD0000C940527653F714011F00C94D3270C948A
:103AE0000827673F91E0790711F40C940E27673E91
:103AF000734011F00C94D3270C941127E5E0F2E009
:103B0000E5C65A9A5A9A5A9A5A9A0C94D327E9ECCB
:103B1000F2E007C09091C00095FFFCCF8093C600F3
:103B2000319684918111F6CF8091C00085FFFCCF42
:103B30008AE08093C6008CE593E00E94A364E9EDDF
:103B4000F2E007C09091C00095FFFCCF8093C600C3
:103B5000319684918111F6CF8091C00085FFFCCF12
:103B60000C94D0278CE593E00E94E5640C94D32755
:103B70008CE593E00E94AE650C94D3270091E0059C
:103B80001091E1050C5F1F4F6AE270E0C8010E94CE
:103B90004975009719F0FC013197108241E0B80196
:103BA00059C08CE593E00E94B2650E94C2296093DF
:103BB000EE057093EF058093F0059093F1050C945A
:103BC000D3278CE593E00E94B9650C94D3278091AC
:103BD0005E03882311F40C94D32783E50E94A61179
:103BE00081110C9438280C94D3278CE593E00E9423
:103BF000F4680C94D3278091E0059091E1056AE286
:103C000070E004960E9449758C010097E1F02091C4
:103C1000DA053091DB0540E6429FC001439F900DDD
:103C200011246EE470E08A5A9B4F0E94497560E24D
:103C300070E00E94497501969093E1058093E0053C
:103C4000F801319710826091E0057091E1056C5F99
:103C50007F4F40E08CE593E00E94BE650C94D32733
:103C600080915E03882311F40C94D3278CE593E0B4
:103C70000E94AA6A8091E0059091E1056AE270E0F5
:103C800004960E9449758C010097E1F02091DA05B5
:103C90003091DB0540E6429FC001439F900D112407
:103CA0006EE470E08A5A9B4F0E94497560E270E0B2
:103CB0000E94497501969093E1058093E005F80113
:103CC000319710826091E0057091E1056C5F7F4F44
:103CD0008CE593E00E94AE670C94D3270E94C22922
:103CE0006093EA057093EB058093EC059093ED05E6
:103CF0000091EE051091EF052091F0053091F1054E
:103D0000601B710B820B930B28EE33E040E050E018
:103D10000E943972CA01B9012CE330E040E050E062
:103D20000E9439727F936F933F932F9382EA91E0C1
:103D30009F938F93CE0101969F938F930E949275CC
:103D4000EBEBF0E084910FB6F894DEBF0FBECDBF71
:103D500008C09091C00095FFFCCF8093C6003196BB
:103D600084918111F6CFFE01319606C09091C0007A
:103D700095FFFCCF8093C60081918111F7CF809190
:103D8000C00085FFFCCF8AE08093C6008091920D31
:103D9000882311F40C94D3271092920D60912C0378
:103DA000E62FF0E0EE0FFF1FE459F14F8081918183
:103DB0000E9409582091330130913401409135011E
:103DC000509136010E946A70181614F00C94D32793
:103DD00060912C03062F10E080E090E00E9439579C
:103DE000F801EE0FFF1FE459F14F91838083F80132
:103DF000EE0FFF1FEE0FFF1FEE59F14F10821182E1
:103E0000128213820C94D32783E50E94A611882383
:103E100011F40C94D3270E9492110E94D66E8B014C
:103E200080E50E94A611882311F40C94D32717FF74
:103E300002C00C94D3270F3F110509F014F40C9421
:103E400049280C94D327819191918E159F0511F4E7
:103E50000C94D32732E0E43DF307A9F7F7FE02C044
:103E60000C94D32761E08E2D0E94E12A602F8E2DC5
:103E70000E94FD2AB8018E2D0E94562A0C94D32749
:103E800088E690E00E94521981110C94D32783E5B3
:103E90000E94A611882309F1B0900B060E9492118E
:103EA0006B017C010B2D10E00E94D66EDC01CB0172
:103EB0006B2D0E943957F801EE0FFF1FE459F14FA7
:103EC00091838083F801EE0FFF1FEE0FFF1FEE5965
:103ED000F14FC082D182E282F3820E94C05B0C94D7
:103EE000D32783E50E94A611882311F40C94D327CD
:103EF0000E9492110E94D66ECB010E94BD579093F2
:103F00006B0E80936A0E0C94D32789E690E00E9492
:103F1000521981110C94D327E7EEF2E007C090917B
:103F2000C00095FFFCCF8093C6003196849181112B
:103F3000F6CF60910B06E62FF0E0EE0FFF1FE85979
:103F4000F14F808191810E940958AB01BC0121E0B1
:103F500030E08DE296E00E946E2DEDEEF2E007C0BB
:103F60009091C00095FFFCCF8093C600319684915C
:103F70008111F6CF60910B06E62FF0E0EE0FFF1FE8
:103F8000E459F14F808191810E940958AB01BC0135
:103F900021E030E08DE296E00E946E2DE0EFF2E04D
:103FA00007C09091C00095FFFCCF8093C60031966A
:103FB00084918111F6CF8091660E9091670E0E94D8
:103FC000C75AAB01BC0121E030E08DE296E00E94CF
:103FD0006E2DE4EFF2E007C09091C00095FFFCCF9A
:103FE0008093C600319684918111F6CF80916A0E3C
:103FF00090916B0E0E94C75AAB01BC0121E030E0EA
:104000008DE296E00E946E2DE7EFF2E007C09091FE
:10401000C00095FFFCCF8093C6003196849181113A
:10402000F6CF80910B0690E00E942E574AE050E0B8
:10403000BC018DE296E00E94762CEBEFF2E007C027
:104040009091C00095FFFCCF8093C600319684917B
:104050008111F6CF8FEF9FEF0E942E574AE050E07C
:10406000BC018DE296E00E94762C8091C00085FF15
:10407000FCCF8AE08093C6000C94AF288DE690E0D8
:104080000E94521981118FC71092920D83E50E94F0
:10409000A611882309F1B0900B060E9492116B01C2
:1040A0007C010B2D10E00E94D66EDC01CB016B2D44
:1040B0000E943957F801EE0FFF1FE459F14F918329
:1040C0008083F801EE0FFF1FEE0FFF1FEE59F14F37
:1040D000C082D182E282F38283E50E94A611882306
:1040E00051F00E94921160933301709334018093D8
:1040F00035019093360182E40E94A611882351F085
:104100000E949211609337017093380180933901B6
:1041100090933A0186E40E94A611882369F00E94D8
:10412000921160932F01709330018093310190932D
:10413000320181E08093920D0E94C05B0E94C229EF
:104140004B015C0180910B0690E0880F991FFC01E8
:10415000E459F14F2081318138A32F8FFC01E859B8
:10416000F14F808191819AA389A3CC24CA94DC2C3D
:104170007601E0E0F3E02490E3E0F3E03490E7E060
:10418000F3E004911AE093C7822DE0E0F3E008C069
:104190009091C00095FFFCCF8093C600319684912A
:1041A0008111F6CF60910B06E62FF0E0EE0FFF1FB6
:1041B000E859F14F808191810E940958AB01BC01FF
:1041C00021E030E08DE296E00E946E2D832DE3E049
:1041D000F3E008C09091C00095FFFCCF8093C6002B
:1041E000319684918111F6CF60910B064AE050E040
:1041F00070E08DE296E00E94762C802FE7E0F3E0FD
:1042000008C09091C00095FFFCCF8093C600319606
:1042100084918111F6CFF7FE03C0EEE1F2E029C0F0
:104220000E94C2294B015C01C701B6016854744F5A
:104230008F4F9F4F681979098A099B0928EE33E04F
:1042400040E050E00E94397249015A012AE030E012
:10425000B501A4018DE296E00E94522C8091C0002D
:1042600085FFFCCF0DC09091C00095FFFCCF8093DF
:10427000C60081918111F7CF8091C00085FFFCCFEE
:104280001093C6000E94C2294B015C010E94D358C2
:104290000E94B0189FEFC916D906E906F90689F5FC
:1042A00060910B06EF8DF8A129A13AA12E173F07C7
:1042B0000CF02DC7E62FF0E0EE0FFF1FE859F14F8D
:1042C000808191810E9409582B013C0160910B066D
:1042D000E62FF0E0EE0FFF1FE459F14F808191814E
:1042E0000E94095820E030E040E85FE30E948D6DB5
:1042F0009B01AC01C301B2010E946A7087FFD2C664
:1043000035C0F7FC33C060910B06E62FF0E0EE0FEE
:10431000FF1FE859F14F808191810E9409582B01BC
:104320003C0160910B06E62FF0E0EE0FFF1FE45911
:10433000F14F808191810E9409589B01AC01C3011A
:10434000B2010E948D6D0E94D66EAB01BC0177FF59
:1043500007C070956095509541955F4F6F4F7F4FA7
:1043600044305105610571050CF09CC63FEFC31642
:10437000D306E306F30609F49AC6F7FCA5C60E9425
:10438000C2296C197D09683B7B4008F490C69CC625
:1043900083E50E94A611882359F00E9492110E9481
:1043A000D66ECB010E94BD5790936B0E80936A0E20
:1043B0000E94C2296B017C01EBE0F3E01491EEE076
:1043C000F3E00491E2E1F3E0B4909AE0A92E6FC02B
:1043D0000E94C2296C197D098E099F09693E7340AC
:1043E0008105910508F45FC060912C03E62FF0E091
:1043F000EE0FFF1FE859F14F808191810E9409580B
:10440000AB01BC01812FEBE0F3E008C09091C0004C
:1044100095FFFCCF8093C600319684918111F6CF31
:1044200022E030E08DE296E00E946E2D802FEEE0DB
:10443000F3E008C09091C00095FFFCCF8093C600C8
:10444000319684918111F6CF60912C034AE050E0BF
:1044500070E08DE296E00E94762C8B2DE2E1F3E095
:1044600008C09091C00095FFFCCF8093C6003196A4
:1044700084918111F6CF8091660E9091670E0E9413
:10448000C75AAB01BC0121E030E08DE296E00E940A
:104490006E2D8091C00085FFFCCFA092C6000E94C7
:1044A000C2296B017C010E94D3580E94B018209150
:1044B0006A0E30916B0E8091660E9091670E821796
:1044C00093070CF485CF0AC683E50E94A6118823C2
:1044D000F1F00E94921120E030E0A9010E94676E85
:1044E00087FD0FC00E94921120E030E04FE753E4B7
:1044F0000E946A7018163CF00E9492110E94DB6EB6
:1045000003C060E001C06FEF60932B034CC58FEFD9
:1045100080932B0348C510922B0345C510925B0373
:1045200042C581E080935B033EC583E50E94A611EE
:10453000882399F00E94921120E030E04AE754E489
:104540000E943C710E94DB6E60932B0170932C01E2
:1045500080932D0190932E0126C588E50E94A61117
:104560008111CDC589E50E94A6118111C8C58AE5D2
:104570000E94A6118111C3C585E40E94A611811174
:10458000BEC5B7C55A9889E50E94A61181115A98EF
:104590008AE50E94A611882309F405C55A9803C527
:1045A00083E50E94A6110E94921120E030E04AE7C4
:1045B00054E40E943C710E94DB6E60930C06709381
:1045C0000D0680930E0690930F06EDC42CE532E0A5
:1045D00038A32F8F0FED1DE0AFEE8A2EADE09A2E9F
:1045E000B3EAAB2EBDE0BB2E712CEF8DF8A181910B
:1045F000F8A3EF8F0E94A611882309F464C0F3E0AA
:104600007F125AC00E9492116B017C0120E030E0C1
:1046100040EA51E40E94676E87FF48C0A7019601F7
:10462000F80160817181828193810E946E6E362EC5
:10463000472E582E692E762F272F342D452D562D97
:104640006091B70D7091B80D8091B90D9091BA0D30
:104650000E943C716093B70D7093B80D8093B90DB3
:104660009093BA0D232D342D452D562DF4016081E4
:104670007181828193810E943C71F4016083718316
:1046800082839383F50160817181828193810E948D
:10469000076F232D342D452D562D0E943C710E940D
:1046A000DB6EF5016083718382839383F801C0829E
:1046B000D182E282F38207C00E949211F8016083E6
:1046C00071838283938373940C5F1F4FF4E08F0E8A
:1046D000911C24E0A20EB11C34E0731286CF63C497
:1046E000E6E1F3E007C09091C00095FFFCCF809316
:1046F000C600319684918111F6CF55C4E1EBF3E009
:1047000007C09091C00095FFFCCF8093C600319602
:1047100084918111F6CF40914503509146036091F9
:1047200047037091480322E030E08DE296E00E945A
:104730006E2DE4EBF3E007C09091C00095FFFCCF35
:104740008093C600319684918111F6CF4091490340
:1047500050914A0360914B0370914C0322E030E08A
:104760008DE296E00E946E2DE7EBF3E007C090919A
:10477000C00095FFFCCF8093C600319684918111D3
:10478000F6CF40914D0350914E0360914F037091CD
:10479000500322E030E08DE296E00E946E2DEAEBBD
:1047A000F3E007C09091C00095FFFCCF8093C60056
:1047B000319684918111F6CF40915103509152036B
:1047C000609153037091540322E030E08DE296E053
:1047D0000E946E2DEDEBF3E007C09091C00095FFB5
:1047E000FCCF8093C600319684918111F6CF0E9450
:1047F000D9560E94096F2091DF0D3091E00D409154
:10480000E10D5091E20D0E946E6EAB01BC0122E001
:1048100030E08DE296E00E946E2DE7ECF3E007C0F9
:104820009091C00095FFFCCF8093C6003196849193
:104830008111F6CF81E00E94D9560E94096F209124
:10484000E30D3091E40D4091E50D5091E60D0E948D
:104850006E6EAB01BC0122E030E08DE296E00E947A
:104860006E2DEAECF3E007C09091C00095FFFCCFFD
:104870008093C600319684918111F6CF82E00E9428
:10488000D9560E94096F2091E70D3091E80D4091B3
:10489000E90D5091EA0D0E946E6EAB01BC0122E061
:1048A00030E08DE296E00E946E2D8091C00085FF81
:1048B000FCCF76C380E001C081E00E94335073C317
:1048C0009091C00095FFFCCF8093C600819181112B
:1048D000F7CF8091C00085FFFCCF8AE08093C600AF
:1048E000EDECF3E007C09091C00095FFFCCF809302
:1048F000C600319684918111F6CF189903C0E6EF76
:10490000F1E009C0E0E0F2E006C09091C00095FF40
:10491000FCCF8093C60081918111F7CF8091C000B8
:1049200085FFFCCF8AE08093C600E5EDF3E007C089
:104930009091C00095FFFCCF8093C6003196849182
:104940008111F6CF199903C0E6EFF1E009C0E0E06C
:10495000F2E006C09091C00095FFFCCF8093C600A6
:1049600081918111F7CF8091C00085FFFCCF8AE053
:104970008093C600EDEDF3E007C09091C00095FF75
:10498000FCCF8093C600319684918111F6CF1A999D
:1049900003C0E6EFF1E009C0E0E0F2E006C090916C
:1049A000C00095FFFCCF8093C60081918111F7CFA5
:1049B0008091C00085FFFCCFF3C2FCE5EF2EF2E052
:1049C000FF2E00E010E0F70181917F010E94A61107
:1049D000882339F10E9492115FECC52E5DE0D52E3F
:1049E000C00ED11E0E94DB6EF6016083718382834C
:1049F00093830E949211E3EACE2EEDE0DE2EC00EEC
:104A0000D11EF801E152F24F208131814281538160
:104A10000E943C710E94DB6EF60160837183828389
:104A200093830C5F1F4F0031110569F6BCC20CE582
:104A300012E04FEEE42E4DE0F42EF80181918F014B
:104A40000E94A611882339F00E949211F701608319
:104A5000718382839383F4E0EF0EF11C22E0003631
:104A6000120759F7A0C283E50E94A611882351F0CE
:104A70000E9492116093C70D7093C80D8093C90D69
:104A80009093CA0D84E50E94A611882309F48BC275
:104A90000E9492116093C30D7093C40D8093C50D55
:104AA0009093C60D80C283E50E94A611882351F021
:104AB0000E9492116093CB0D7093CC0D8093CD0D1D
:104AC0009093CE0D84E50E94A611882351F00E9498
:104AD00092116093B30D7093B40D8093B50D9093C4
:104AE000B60D82E40E94A611882361F00E94921103
:104AF0000E94DB6E6093FF0D7093000E8093010E99
:104B00009093020E88E50E94A611882351F00E941E
:104B100092116093BF0D7093C00D8093C10D90935F
:104B2000C20D8AE50E94A611882351F00E949211BD
:104B30006093BB0D7093BC0D8093BD0D9093BE0D23
:104B400085E40E94A611882309F42DC20E949211C7
:104B50006093B70D7093B80D8093B90D9093BA0D13
:104B600022C20CE512E039E3E32E33E0F32EF80124
:104B700081918F010E94A611882339F00E94921121
:104B8000F7016083718382839383F4E0EF0EF11C5D
:104B900022E00F35120759F706C283E50E94A611DD
:104BA000882309F400C20E9492110E94D66E70936D
:104BB00015016093140181E080935503F4C183E5EE
:104BC0000E94A611882309F4EEC10E9492110E944E
:104BD000D66E7093130160931201E5C180E50E94C7
:104BE000A611882351F00E94921160934C0170939A
:104BF0004D0180934E0190934F0189E40E94A611CC
:104C0000882381F00E94921125E93FEB46ED5DE398
:104C10000E943C71609348017093490180934A015E
:104C200090934B0184E40E94A611882381F00E9496
:104C3000921125E93FEB46ED5DE30E946E6E6093B5
:104C4000440170934501809346019093470183E4AA
:104C50000E94A611882351F00E9492116093400196
:104C60007093410180934201909343010E94175732
:104C7000E0E2F2E006C09091C00095FFFCCF809387
:104C8000C60081918111F7CFE3E2F2E006C0909176
:104C9000C00095FFFCCF8093C60081918111F7CFB2
:104CA00040914C0150914D0160914E0170914F0126
:104CB00022E030E08DE296E00E946E2DE7E2F2E025
:104CC00006C09091C00095FFFCCF8093C6008191F3
:104CD0008111F7CF25E93FEB46ED5DE36091480197
:104CE0007091490180914A0190914B010E946E6E32
:104CF000AB01BC0122E030E08DE296E00E946E2D17
:104D0000EBE2F2E006C09091C00095FFFCCF8093EB
:104D1000C60081918111F7CF25E93FEB46ED5DE3B8
:104D20006091440170914501809146019091470145
:104D30000E943C71AB01BC0122E030E08DE296E0C4
:104D40000E946E2DEFE2F2E006C09091C00095FF48
:104D5000FCCF8093C60081918111F7CF25E93FEB0D
:104D600046ED5DE360914001709141018091420107
:104D7000909143010E943C71AB01BC0122E030E004
:104D80008DE296E00E946E2D8091C00085FFFCCFE1
:104D900007C181E00E949A4F06C185E40E94A611D6
:104DA000882341F00E9492110E94D66E8B0177FDFC
:104DB0000AC002C000E010E0C12CD12C26E1E22E96
:104DC00023E4F22E06C0C12CD12C9CE8E92E92E4FB
:104DD000F92E83E50E94A611882321F00E949211EA
:104DE0006B017C0183E40E94A611882331F00E94AC
:104DF00092110E94D66E9B0102C025E030E0A8010E
:104E0000C701B6010E94F25BCEC00E948056CBC0A3
:104E100080E001C081E00E944B0BC5C00E948A0C5B
:104E2000C2C010922A038091100690911106A091A1
:104E30001206B09113068093E6059093E705A093C0
:104E4000E805B093E9050E94E911ADC084E50E9430
:104E5000A611882309F463C00E9492110E94DB6EA0
:104E600060930B06662391F1EBEBF0E007C09091A5
:104E7000C00095FFFCCF8093C600319684918111CC
:104E8000F6CFE3E3F2E006C09091C00095FFFCCFBF
:104E90008093C60081918111F7CF40E050E060918E
:104EA0000B068DE296E00E945E2CE5E3F2E006C080
:104EB0009091C00095FFFCCF8093C6008191811135
:104EC000F7CF8091C00085FFFCCF6AC010922C0301
:104ED000EBEBF0E007C09091C00095FFFCCF809312
:104EE000C600319684918111F6CFE6E4F2E006C067
:104EF0009091C00095FFFCCF8093C60081918111F5
:104F0000F7CF60912C034AE050E070E08DE296E02C
:104F10000E94762C8091C00085FFFCCF41C0EBEB56
:104F2000F0E007C09091C00095FFFCCF8093C600D1
:104F3000319684918111F6CFE5EEF3E007C09091B0
:104F4000C00095FFFCCF8093C600319684918111FB
:104F5000F6CF8091DA059091DB0520E6289FF001DD
:104F6000299FF00D1124EA5AFB4F06C09091C00012
:104F700095FFFCCF8093C60081918111F7CFE7EFB9
:104F8000F3E007C09091C00095FFFCCF8093C6006E
:104F9000319684918111F6CF8091C00085FFFCCFBE
:104FA0008AE08093C6000E94C111D9C010924503C7
:104FB000109246031092470310924803109249033F
:104FC00010924A0310924B0310924C0321E533E0F8
:104FD0004DE453E069E473E085E493E00E94E44E1D
:104FE00080E090ECA9E9B3EC8093FA059093FB057F
:104FF000A093FC05B093FD058093FE059093FF05FB
:10500000A0930006B093010620911601309117017C
:1050100040911801509119012093260130932701E6
:105020004093280150932901C0901A01D0901B0190
:10503000E0901C01F0901D01C701B6010E94676E4F
:1050400087FF02C00C94F21A0C94FA1A80E090E0E8
:105050000E94120A0C947D1B81E090E00E94120ACB
:105060000C94881B82E090E00E94120A0C94931B1F
:105070000E949B11AB0160934804509349048093B4
:105080004A0490934B04BC0185E294E00E94E13015
:105090008ACF0E9492110E94D66E7B01E0E6F2E078
:1050A0000C94231F0E94C2296B017C015FC90E94DE
:1050B000C229681979098A099B09693E73408105EB
:1050C000910508F061C8E2C80E94C2296093EE050C
:1050D0007093EF058093F0059093F1050E94C2292B
:1050E0006093F2057093F3058093F4059093F505B2
:1050F0005ACF0E9480565A980E94ED5654CF0E9473
:10510000805688E50E94A61181113CCA3CCAE62F50
:10511000F0E0EE0FFF1FE859F14F808191810E946E
:1051200009582B013C0160910B06E62FF0E0EE0FD1
:10513000FF1FE459F14F808191810E94095820E0BE
:1051400030E040E85FE30E948E6D9B01AC01C3013B
:10515000B2010E94676E18160CF0A4CF07C9A29680
:105160000FB6F894DEBF0FBECDBFDF91CF911F9178
:105170000F91FF90EF90DF90CF90BF90AF909F90F6
:105180008F907F906F905F904F903F902F900895F9
:10519000CF93DF938091520490915304039714F4BA
:1051A0000E94151260E08CE593E00E94B76980913F
:1051B000520490915304892B09F460C080915C03E0
:1051C000882309F443C08091DA059091DB0520E63D
:1051D000289FE001299FD00D1124CA5ADB4F68E5B2
:1051E00072E0CE010E947875892BB9F4BE018CE57E
:1051F00093E00E944969EDE7F1E007C09091C0009B
:1052000095FFFCCF8093C600319684918111F6CF33
:105210008091C00085FFFCCF15C08CE593E00E9413
:10522000AA6AE0E8F1E007C09091C00095FFFCCFCA
:105230008093C600319684918111F6CF8091C00091
:1052400085FFFCCF8AE08093C60002C00E94B81997
:10525000809152049091530401979093530480934A
:1052600052048091DA059091DB05019664E070E0CC
:105270000E9425729093DB058093DA050E94D35833
:105280000E94B018DF91CF910C949D4F0E941B2A71
:105290000E94F40F0E94C828FDCF2EE932E0FC01E5
:1052A000318320832581222319F002960C94C83182
:1052B0000895CF93DF93EC0189539F4F0E944D29AE
:1052C000CE0189579F4F0E944D29CE0186599F4F8D
:1052D0000E944D29CE01835B9F4F0E944D29CE0134
:1052E0008E96DF91CF910C944D298CE593E00C9430
:1052F000A8628CE593E00C9459291F920F920FB687
:105300000F9211242F933F938F939F93AF93BF934B
:105310008091240690912506A0912606B09127063B
:1053200030912C06232F2A592D3720F02D57019626
:10533000A11DB11D20932C06809324069093250671
:10534000A0932606B09327068091280690912906FF
:10535000A0912A06B0912B060196A11DB11D809344
:10536000280690932906A0932A06B0932B06BF9196
:10537000AF919F918F913F912F910F900FBE0F9002
:105380001F9018950F931F938FB7F89400912406E0
:105390001091250620912606309127068FBFB8016F
:1053A000C9011F910F9108959FB7F8944091280665
:1053B0005091290660912A0670912B0686B5A89B0C
:1053C00006C08F3F21F04F5F5F4F6F4F7F4F9FBFF2
:1053D0002227342F452F562F280F311D411D511DD7
:1053E000A3E0B0E00E9402720895CF92DF92EF92A4
:1053F000FF92CF93DF936B017C010E94D429EB01D4
:105400000EC00E94D4296C1B7D0B683E734038F09F
:1054100081E0C81AD108E108F108C851DC4FC11475
:10542000D104E104F10469F7DF91CF91FF90EF908F
:10543000DF90CF900895789484B5826084BD84B560
:10544000816084BD85B5826085BD85B5816085BD7F
:10545000EEE6F0E0808181608083E1E8F0E0108298
:10546000808182608083808181608083E0E8F0E0D9
:10547000808181608083E1EBF0E0808184608083C3
:10548000E0EBF0E0808181608083EAE7F0E08081FA
:10549000846080838081826080838081816080835A
:1054A0008081806880831092C10008951F93CF93FC
:1054B000DF93182FEB0161E00E94E12A209711F49D
:1054C00060E004C0CF3FD10539F461E0812FDF9166
:1054D000CF911F910C94FD2AE12FF0E0E059FD4E91
:1054E000E491E330B9F028F4E13051F0E230B1F565
:1054F0000CC0E63019F1E73049F1E43079F514C019
:1055000084B5806884BDC7BD2EC084B5806284BD6B
:10551000C8BD29C080918000806880938000D093AE
:105520008900C09388001FC08091800080628093B2
:105530008000D0938B00C0938A0015C08091B0008A
:1055400080688093B000C093B3000DC08091B0001C
:1055500080628093B000C093B40005C0C038D1050C
:105560000CF0B3CFADCFDF91CF911F910895833071
:1055700069F028F48130A1F0823011F514C0863032
:10558000B1F08730C1F08430D9F404C0809180003C
:105590008F7703C0809180008F7D80938000089575
:1055A00084B58F7702C084B58F7D84BD08958091C6
:1055B000B0008F7703C08091B0008F7D8093B000E2
:1055C000089590E0FC01E057FD4E2491FC01E05568
:1055D000FD4EE491EE2381F0F0E0EB52FD4EA491FC
:1055E000B0E09FB7F8948C91611103C0209582239D
:1055F00001C0822B8C939FBF08950F931F93CF936D
:10560000DF931F92CDB7DEB7A82FB0E0FD01E059C0
:10561000FD4E8491FD01E057FD4E1491FD01E055D2
:10562000FD4E04910023B9F0882321F069830E9484
:10563000B72A6981E02FF0E0E053FD4EA491B0E07D
:105640009FB7F8948C91611103C01095812301C01C
:10565000812B8C939FBF0F90DF91CF911F910F9162
:1056600008951F920F920FB60F9211242F933F931C
:105670004F935F936F938F939F93EF93FF936091FB
:10568000C6002091AE063091AF06C90101968F7712
:1056900099274091B0065091B1068417950741F0C3
:1056A000F901E25DF94F60839093AF068093AE06F7
:1056B000FF91EF919F918F916F915F914F913F91EA
:1056C0002F910F900FBE0F901F9018959A01AB016C
:1056D00082E08093C00060E47BE48CE490E00E9470
:1056E0005B722150310941095109CA01B90122E017
:1056F00030E040E050E00E945B72832F9927809356
:10570000C5002093C400E1ECF0E0808180618083DB
:105710008081886080838081806880830895809103
:10572000B0069091B1062091AE063091AF062817D1
:10573000390769F0FC01E25DF94F208101968F770E
:1057400099279093B1068093B00630E002C02FEF06
:105750003FEFC90108958091B0069091B1069093F2
:10576000AF068093AE0608954F925F926F927F923C
:105770008F929F92AF92BF92CF92DF92EF92FF9261
:105780000F931F93CF93DF93CDB7DEB7A0970FB6DC
:10579000F894DEBF0FBECDBF8C01411551056105E8
:1057A0007105F1F420E030E040E350E060E070E0AB
:1057B000A0960FB6F894DEBF0FBECDBFDF91CF919C
:1057C0001F910F91FF90EF90DF90CF90BF90AF901F
:1057D0009F908F907F906F905F904F900C94652C6E
:1057E000EE24E394F12CEC0EFD1E812C912C54013F
:1057F000422E512C612C712CCB01BA01A3019201D4
:105800000E943972FA01D7016D937D01BFEF8B1AA7
:105810009B0AAB0ABB0AA901BF01411551056105ED
:10582000710551F7CC24CA94DC2C7601C80CD91C24
:10583000EA1CFB1C1AC0E1E0F0E0EC0FFD1FEC0DD0
:10584000FD1D8081482F8A3010F4405D01C0495C05
:1058500050E060E070E020E030E0C8010E94652C7C
:1058600081E0C81AD108E108F108AFEFCA16DA06DC
:10587000EA06FA0601F7A0960FB6F894DEBF0FBE4F
:10588000CDBFDF91CF911F910F91FF90EF90DF90EF
:10589000CF90BF90AF909F908F907F906F905F90D0
:1058A0004F9008952115310539F48091C00085FF8E
:1058B000FCCF4093C60008950C94B42B9A01462F58
:1058C00050E060E070E00C94522C2115310539F461
:1058D0008091C00085FFFCCF4093C60008952A3018
:1058E000310511F40C94A22C0C94B42B9A01AB0149
:1058F000662757FD6095762F0C94652CCF93DF9328
:10590000EC0120E030E04DE050E060E070E00E940B
:10591000652C20E030E04AE050E060E070E0CE012D
:10592000DF91CF910C94652CCF93DF93EC019A011A
:10593000AB0160E070E00E94522CCE01DF91CF916C
:105940000C947E2CCF92DF92EF92FF92CF93DF9355
:10595000EC016A017B0177FF10C020E030E04DE2EE
:1059600050E060E070E00E94652CF094E094D094E8
:10597000C094C11CD11CE11CF11C2AE0B701A60196
:10598000CE01DF91CF91FF90EF90DF90CF900C94FC
:10599000B42B9F92AF92BF92CF92DF92EF92FF9281
:1059A0000F931F93CF93DF93EC016A017B01122FBA
:1059B00020E030E0A901C701B6010E94676E87FFB1
:1059C0000DC020E030E04DE250E060E070E0CE013C
:1059D0000E94652CF7FAF094F7F8F09400E060E08C
:1059E00070E080E09FE307C020E030E040E251E457
:1059F0000E946E6E0F5F0113F7CF262F372F482FAF
:105A0000592FC701B6010E948E6D962EA72EB82E73
:105A1000C92E0E94DB6ED62EE72EF82E092F0E948B
:105A2000076F9B01AC01692D7A2D8B2D9C2D0E9457
:105A30008D6DC62EB72EA82E992E2AE04D2D5E2DE7
:105A40006F2D702FCE010E94B42B1123C9F1E3EF0B
:105A5000F2E006C09091C00095FFFCCF8093C60095
:105A600081918111F7CF2CC020E030E040E251E479
:105A70006C2D7B2D8A2D992D0E943C71962EA72E80
:105A8000B82E092F902F0E94D66E6B01EE24D7FC02
:105A9000E094FE2CB701A601CE010E94A22CC70102
:105AA000B6010E94096F9B01AC01692D7A2D8B2DE7
:105AB000902F0E948D6DC62EB72EA82E992E1150B4
:105AC0001111D2CFDF91CF911F910F91FF90EF90E5
:105AD000DF90CF90BF90AF909F9008950C94C92C09
:105AE000CF93DF93EC019C012C5F3F4F41E050E0EE
:105AF00060E070E0898D9A8D0E947F388823A1F044
:105B00004D895E896F89788D452B462B472B71F423
:105B10004C815D816E817F814D8B5E8B6F8B788F29
:105B200089818068898302C080E001C081E0DF91C3
:105B3000CF910895CF92DF92EF92FF921F93CF9370
:105B4000DF93EC0189899A89AB89BC89803E9F4F9C
:105B5000AF41B10508F06DC0CE010E94702D8823C1
:105B600009F467C00E949236882309F462C0E98D67
:105B7000FA8DCC80DD80EE80FF8032E0C31AD10840
:105B8000E108F108058404C0CC0CDD1CEE1CFF1CF0
:105B90000A94D2F786859785A089B189C80ED91E47
:105BA000EA1EFB1E81E08093B806C092BB08D0922B
:105BB000BC08E092BD08F092BE0880E092E0EBEBFA
:105BC000F6E0DF019C011D9221503040E1F711E029
:105BD00011C0B701A601410F511D611D711D2BEBB5
:105BE00036E08091B9069091BA060E94436D8823F1
:105BF00001F11F5FE98DFA8D8481181750F380E061
:105C000092E0A0E0B0E0058404C0880F991FAA1FAD
:105C1000BB1F0A94D2F749895A896B897C89480F3E
:105C2000591F6A1F7B1F498B5A8B6B8B7C8B81E0C2
:105C300001C080E0DF91CF911F91FF90EF90DF9046
:105C4000CF900895CF93DF93EC0141E0611101C043
:105C500040E06C857D858E859F850E94CD368823AA
:105C600041F0288980E2289F900111242554394F62
:105C700002C020E030E0C901DF91CF910895CF93B9
:105C8000FB0120E030E231932F5F2B30E1F7DC01A4
:105C900030E0C7E01CC0CA3051F138E0CAE017C09C
:105CA000E21729F1FC010196E491E111F9CFC31744
:105CB000F0F02132E0F02F37D0F4FB01E30FF11DBB
:105CC000822F81568A3108F4205220833F5FCD0114
:105CD0002D91211109C0FA018083918381E0FB019C
:105CE0009081903259F403C02F3219F4F4CF80E040
:105CF00005C02E3281F28AE896E0D4CFCF91089584
:105D00000F931F93CF93DF93EC018B018B8188233B
:105D100011F080E044C0FB018789803131F528C053
:105D200083E08B83F801428D538D648D758D4D8B8F
:105D30005E8B6F8B788F9E012F5E3F4FC8010E9454
:105D40008737882331F31A8F098F81E089831C827A
:105D50001D821E821F82188619861A861B861C8643
:105D60001D861E861F86188A1AC0803291F6D8CFEB
:105D700082E08B831D8A1E8A1F8A188EFB01408D4C
:105D8000518D60E070E085E0440F551F661F771F5E
:105D90008A95D1F7498B5A8B6B8B7C8BD4CFDF9153
:105DA000CF911F910F9108952F923F924F925F9242
:105DB0006F927F928F929F92AF92BF92CF92DF921B
:105DC000EF92FF920F931F93CF93DF9300D000D0F9
:105DD000CDB7DEB79C838B83962E872E5A01DC01CC
:105DE00013968C91811103C02FEF3FEFF6C0EB812A
:105DF000FC81818180FFF8CFC0C05A01A81AB90A7E
:105E00006501092D182D8B819C8104969A838983C5
:105E1000612CB2E07B2EABC0AB81BC8118964D915A
:105E20005D916D917C911B97DB01CA019170AA274E
:105E3000BB274C01EB81FC8123811A012B01A9E0D6
:105E40005694479437942794AA95D1F7818D928DD3
:105E5000223061F4DC015A966D917D918D919C9177
:105E60005D97620D731D841D951D4BC0FC01F48070
:105E7000FA94F2208114910401F5F1101EC0452B13
:105E8000462B472B59F4EB81FC8185899689A7899C
:105E9000B08D84839583A683B7830FC0AB81BC810B
:105EA00014964D915D916D917C91179729813A815E
:105EB0000E940637882309F497CFAB81BC8159969D
:105EC000ED91FC915A9714966D917D918D919C91D5
:105ED00017976250710981099109058404C0660F02
:105EE000771F881F991F0A94D2F726853785408926
:105EF0005189620F731F841F951F6F0D711D811DC6
:105F0000911D93012819390976012C153D0508F4D6
:105F10007901E114B2E0FB0609F059C02091BB08F9
:105F20003091BC084091BD085091BE0862177307BC
:105F30008407950709F03FC04AC0C4018554994FB2
:105F4000A701BC01C8010E9435750E0D1F1DEB8114
:105F5000FC8180859185A285B3858E0D9F1DA11D35
:105F6000B11D80879187A287B387CE18DF08C1143F
:105F7000D10409F051CF950130C0AB81BC8151965D
:105F80004D915D916D917C91549718968D919D9155
:105F90000D90BC91A02D6501E12CF12C8A019B0193
:105FA000081B190B2A0B3B0BC016D106E206F306A1
:105FB00008F023CF25CF9801AB01BC018091B90631
:105FC0009091BA060E94206C8111BFCF0DCF40E0A6
:105FD0000E94CD368111B1CF07CFC9010F900F902C
:105FE0000F900F90DF91CF911F910F91FF90EF9045
:105FF000DF90CF90BF90AF909F908F907F906F90E9
:106000005F904F903F902F900895CF93DF931F9212
:10601000CDB7DEB741E050E0BE016F5F7F4F0E9419
:10602000D42E019719F4298130E002C02FEF3FEF01
:10603000C9010F90DF91CF910895CF92DF92EF9237
:10604000FF920F931F93CF93DF936C01EB017A01C3
:10605000FC018381823008F461C0008511852285AE
:1060600033850F71112722273327012B022B032B96
:1060700009F054C055C0F70110821DE040E250E025
:10608000BE01C6010E94D42E8032910529F0892BD1
:1060900009F044C080E04EC028812223D9F3253E78
:1060A00069F32E3259F33B853F733F3099F5E11484
:1060B000F104D9F52FC02F7130E02115310551F1D0
:1060C000233031053CF521503109129FC001139F47
:1060D000900D1124F701E80FF91F298120832B81EE
:1060E00021832D8122832F812383298524832E855B
:1060F0002583288926832A8927832C8920872E892E
:106100002187288D22872C8D23872E8D2487288117
:1061100026FD15862B8523FDB1CF0CC08FEF0AC05D
:106120004115510509F0A7CFA8CF4A8D5B8D452BAE
:1061300011F2F0CFDF91CF911F910F91FF90EF906F
:10614000DF90CF900895CF92DF92EF92FF92CF939E
:10615000DF93EC018B81823018F420E030E029C01D
:10616000C884D984EA84FB8485E0F694E794D794C4
:10617000C7948A95D1F78FE0C822DD24EE24FF244E
:10618000CE010E94053097FDE8CF488559856A8584
:106190007B85415E5F4F6F4F7F4F488759876A8786
:1061A0007B879601C5E0220F331FCA95E1F725547E
:1061B000394FC901DF91CF91FF90EF90DF90CF90E1
:1061C00008958F929F92AF92BF92CF92DF92EF92FB
:1061D000FF920F931F93CF93DF93EC014A015B0172
:1061E0002B81222309F475C089899A89AB89BC89DE
:1061F00084179507A607B70708F46BC06CC0811415
:106200009104A104B10449F41C821D821E821F82E4
:10621000188619861A861B865AC0488559856A854C
:106220007B85E98DFA8D258530E0275F3F4FDB01C7
:10623000CA010197A109B109022E04C0B695A7951C
:10624000979587950A94D2F7CC24CA94DC2C7601D2
:10625000C80CD91CEA1CFB1C04C0F694E794D79424
:10626000C7942A95D2F7C816D906EA06FB0620F08D
:10627000452B462B472B49F48D899E89AF89B88DD4
:106280008C839D83AE83BF8316C0C81AD90AEA0ADD
:10629000FB0A11C04C815D816E817F819801898DDF
:1062A0009A8D0E94063791E0C91AD108E108F108D9
:1062B000811104C014C08E010C5F1F4FC114D104A2
:1062C000E104F10439F788869986AA86BB8681E0C5
:1062D00006C080E004C0223009F091CFF4CFDF91F6
:1062E000CF911F910F91FF90EF90DF90CF90BF90D3
:1062F000AF909F908F9008950F931F93CF93DF934C
:10630000EC018B818823E1F1898187FF33C061E053
:10631000CE010E94222E8C01009791F1FC01808118
:10632000853E71F18B81823040F449895A896B89AD
:106330007C89448F558F668F778F4D895E896F89F1
:10634000788DF801538F428F758B648BE091B20684
:10635000F091B306309759F0B8016A5E7F4FC801DB
:1063600048960995F801808D918D938B828B898158
:106370008F778983DF91CF911F910F910C94923683
:1063800081E0888380E0DF91CF911F910F91089584
:10639000CF93DF93EC010E947C311B82DF91CF9180
:1063A0000895FC01238121110C94C83108954F9266
:1063B0005F926F927F92AF92BF92CF92DF92EF92F5
:1063C000FF920F931F93CF93DF9300D000D0CDB7F0
:1063D000DEB75C016A017B01FC018381813009F039
:1063E00083C0818181FF80C081C0892B8A2B8B2B48
:1063F00009F478C0F5014084518462847384B70144
:10640000A601C5010E94E130811101C06DC0F501F6
:10641000818D928DC114D104E104F10479F4458990
:1064200056896789708D0E949739882309F45CC06A
:10643000F501158A168A178A108E3AC0F501448133
:106440005581668177819E012F5F3F4F0E940637FD
:10645000882309F449C049815A816B817C81F50107
:10646000818D928DFC012789203139F4483FFFEF5F
:106470005F0761057105E0F407C0483F2FEF520741
:1064800062072FE07207A0F40E949739882361F118
:10649000F50144815581668177810FEF1FEF2FEF62
:1064A0003FE0818D928D0E94EF37811101C01CC0A9
:1064B000F501C18AD28AE38AF48A81818068818366
:1064C000C5010E947C31882379F0B701A6014C14E4
:1064D0005D046E047F0410F4B301A201C5010E94A3
:1064E000E13010C081E00EC080E00CC0F501818970
:1064F0009289A389B48984179507A607B70708F07E
:1065000074CFF2CF0F900F900F900F90DF91CF913B
:106510001F910F91FF90EF90DF90CF90BF90AF90C1
:106520007F906F905F904F900895CF93DF93EC0131
:1065300040E050E0BA010E94D731882371F061E059
:10654000CE010E94222E009741F025EEFC0120830F
:106550001B82DF91CF910C94923680E0DF91CF9136
:1065600008951F93CF93DF93EC01142F80E2689F6F
:10657000F0011124E554F94F8385817121F0842FB6
:10658000827109F05AC08091BB089091BC08A0911B
:10659000BD08B091BE088C879D87AE87BF87688B8A
:1065A0004489558960E070E0BA0155274427828DFF
:1065B000938DA0E0B0E0482B592B6A2B7B2B4D8BA1
:1065C0005E8B6F8B788F8385887151F4848D958D68
:1065D000A68DB78D898B9A8BAB8BBC8B81E00CC061
:1065E000803159F59E012F5E3F4F898D9A8D0E9413
:1065F0008737882311F184E08B83812F8F70898303
:106600001C821D821E821F82188619861A861B868E
:1066100014FF16C040E050E0BA01CE010E94D7310D
:1066200081110EC010C049895A896B897C89CE01BD
:10663000DF91CF911F910C94E1301B8280E003C069
:1066400015FDF1CF81E0DF91CF911F910895AF92B9
:10665000BF92CF92DF92EF92FF920F931F93CF934F
:10666000DF937C01EB016A01B22E898D9A8DF701CF
:10667000928F818F40E050E0BA01CE010E94E1305C
:10668000A12C34C045E036952795179507954A9576
:10669000D1F70F70CE010E94A330009709F493C088
:1066A000FC012081222311F0253EB9F4A11010C075
:1066B0004091BB085091BC086091BD087091BE0824
:1066C000F7014487558766877787008BAA24A394B0
:1066D000FC01808181110AC071C04BE050E0BC0117
:1066E000C6010E942875009709F46BC008851985BA
:1066F0002A853B8589899A89AB89BC89081719073E
:106700002A073B0708F4BECF59C0B1FE5CC0AA20DF
:1067100051F0F701008961E0C7010E94222EEC01CF
:10672000009771F450C08B81823009F44CC0CE01C7
:106730000E949A2D882309F446C0CBEBD6E000E0F6
:1067400080E2FE0111928A95E9F78BE0F601DE0105
:1067500001900D928A95E1F7E091B206F091B306AF
:10676000309739F0BE01625F7F4FCE0140960995A8
:1067700008C081E298E2998B888B80E098E09F873F
:106780008E87888999899B8B8A8B998F888F8E8534
:106790009F859F8B8E8B0E9492368823A1F04B2D74
:1067A000602FC701DF91CF911F910F91FF90EF9064
:1067B000DF90CF90BF90AF900C94B132B6FCA5CFD4
:1067C00002C0B7FEECCF80E0DF91CF911F910F9117
:1067D000FF90EF90DF90CF90BF90AF9008955F92C1
:1067E0006F927F928F929F92AF92BF92CF92DF92E1
:1067F000EF92FF920F931F93CF93DF93CDB7DEB746
:10680000C354D1090FB6F894DEBF0FBECDBF5C01F3
:106810006B0124965FAF4EAF2497622E1C8E1F8EA5
:1068200019821C826115710511F410E078C0FC0119
:1068300083818111FACF2496EEADFFAD249780813C
:106840008F3239F0760117C031962496FFAFEEAF44
:1068500024972496EEADFFAD249780818F32A1F36B
:10686000F60183818250823068F4ECCFEE24E39409
:10687000F12CEC0EFD1E8E01045E1F4F4801502EC0
:10688000712E0DC0F601618D728DCE0101960E94B0
:10689000802E8111EBCFC9CF7801052D172DAE01C8
:1068A0004E5B5F4FBE01695C7F4F24968EAD9FADFE
:1068B00024970E943F2E811106C0B7CF31962496AF
:1068C000FFAFEEAF24972496EEADFFAD2497808105
:1068D0008F32A1F38823D1F021E0AE01495C5F4FF4
:1068E000B701C8010E942733882309F49ECFEC1416
:1068F000FD0419F0C7010E94C8310815190561F699
:106900008E010F5F1F4FE52CF72CC9CF262DAE014E
:10691000495C5F4FB701C5010E942733182FCE0194
:1069200001960E94D131CE014C960E94D131812F27
:10693000CD5BDF4F0FB6F894DEBF0FBECDBFDF914A
:10694000CF911F910F91FF90EF90DF90CF90BF906C
:10695000AF909F908F907F906F905F9008951F935E
:10696000CF93DF93CDB7DEB76B970FB6F894DEBF4A
:106970000FBECDBFAB0119821C8222E0BC01CE014B
:1069800001960E94EF33882331F0CE0101960E94D8
:106990009532182F01C010E0CE0101960E94D1312E
:1069A000812F6B960FB6F894DEBF0FBECDBFDF917F
:1069B000CF911F9108952F923F924F925F926F92C5
:1069C0007F928F929F92AF92BF92CF92DF92EF927F
:1069D000FF920F931F93CF93DF9300D000D01F92AD
:1069E000CDB7DEB78C01D62EC72E3A01DC01139647
:1069F0008C911397813009F055C111968C9181FFCC
:106A000051C156C1F80141895289638974898085D1
:106A10009185A285B38584179507A607B70721F44A
:106A20005301ED2CFC2C04C1C8010E94E1308111FE
:106A3000F7CF38C1D80159968D919C915A97FC0196
:106A4000F481F1501A012B01E9E0569447943794F0
:106A50002794EA95D1F7F221FD83517066277727B5
:106A60004A01F11146C04115510509F042C0149682
:106A70004D915D916D917C9117974115510561057F
:106A8000710559F455968D919D910D90BC91A02D55
:106A90000097A105B10541F521C09E012F5F3F4F31
:106AA0000E940637882309F4FDC089819A81AB8151
:106AB000BC81F801218D328DF9012789203139F40B
:106AC000883FFFEF9F07A105B10540F40DC0883F47
:106AD0002FEF9207A2072FE0B20730F0C8010E9403
:106AE000702D811106C0DEC0F80184839583A683D2
:106AF000B78380E092E08819990965018A159B05A2
:106B000008F46C01D8015996ED91FC915A971496AE
:106B10002D903D904D905C901797B2E02B1A310864
:106B200041085108058404C0220C331C441C551C28
:106B30000A94D2F786859785A089B189280E391ED7
:106B40004A1E5B1EED812E0E311C411C511CC114CE
:106B5000F2E0DF0631F58091BB089091BC08A0916E
:106B6000BD08B091BE0882159305A405B50569F46A
:106B70001092B8068FEF9FEFDC018093BB089093D3
:106B8000BC08A093BD08B093BE089701B201A10153
:106B90008091B9069091BA060E94436D811137C069
:106BA00081C08114910419F5D80118964D915D9119
:106BB0006D917C911B9751968D919D910D90BC91FB
:106BC000A02D481759076A077B0788F00E94923664
:106BD000882309F467C081E08093B8062092BB083F
:106BE0003092BC084092BD085092BE0808C041E0F7
:106BF000C201B1010E94CD36882309F453C094012B
:106C00002554394FA601B701C9010E943575F80115
:106C100080859185A285B3858C0D9D1DA11DB11D1B
:106C200080879187A287B387EC0CFD1CAC18BD0848
:106C3000D80118964D915D916D917C911B97A1148F
:106C4000B10409F0F7CE51968D919D910D90BC91B4
:106C5000A02D84179507A607B70748F4F801418BC4
:106C6000528B638B748B81818068818310C080918B
:106C7000B2069091B306892B51F06114710439F07A
:106C8000D80111968C911197806811968C93F80118
:106C9000818183FD02C093010EC0C8010E947C3136
:106CA0008111F9CF81E0D8018C932FEF3FEF03C022
:106CB00082FDA8CEB5CEC9010F900F900F900F9016
:106CC0000F90DF91CF911F910F91FF90EF90DF9088
:106CD000CF90BF90AF909F908F907F906F905F907C
:106CE0004F903F902F900895DB010D900020E9F721
:106CF000AD0141505109461B570B02960C94DB34F1
:106D0000CF93DF931F92CDB7DEB7698341E050E0A8
:106D1000BE016F5F7F4F02960E94DB340F90DF91C0
:106D2000CF9108958091B8068823A9F14091BB08BE
:106D30005091BC086091BD087091BE082BEB36E005
:106D40008091B9069091BA060E94436D811102C0EC
:106D500080E008954091B4065091B5066091B60662
:106D60007091B706411551056105710591F02BEB46
:106D700036E08091B9069091BA060E94436D88234F
:106D800039F31092B4061092B5061092B60610921E
:106D9000B7061092B80681E00895CF92DF92EF9285
:106DA000FF92CF936B017C01C42F8091BB0890911F
:106DB000BC08A091BD08B091BE088C159D05AE051C
:106DC000BF05D1F00E949236811102C080E018C048
:106DD0002BEB36E0B701A6018091B9069091BA0677
:106DE0000E94206C882391F3C092BB08D092BC080B
:106DF000E092BD08F092BE0881E0C1118093B80610
:106E0000CF91FF90EF90DF90CF9008958F929F9257
:106E1000AF92BF92CF92DF92EF92FF920F931F93A8
:106E2000CF93DF93EC016A017B01890189859A8503
:106E3000AB85BC850196A11DB11D84179507A607DA
:106E4000B70710F480E056C08F89803129F4992764
:106E5000872F762F652F0BC08032A1F7CB01BA01A7
:106E600027E096958795779567952A95D1F78B8832
:106E70009C88AD88BE88680D791D8A1D9B1D8090F9
:106E8000BB089090BC08A090BD08B090BE086815E3
:106E900079058A059B0521F48F898031A1F406C00C
:106EA00040E00E94CD368111F7CFCCCFDD24EE2417
:106EB000FF24F601EE0FFF1FE554F94F8081918109
:106EC000A0E0B0E011C0E894C7F8DD24EE24FF2470
:106ED000F601EE0FFF1FEE0FFF1FE554F94F808103
:106EE0009181A281B381BF70F80180839183A283D5
:106EF000B38381E0DF91CF911F910F91FF90EF90CD
:106F0000DF90CF90BF90AF909F908F9008954F9259
:106F10005F926F927F92AF92BF92CF92DF92EF9289
:106F2000FF920F931F93CF93DF9300D000D0CDB784
:106F3000DEB78C0149835A836B837C835901C12C52
:106F4000D12C7601412C42E0542E612C712C4981C8
:106F50005A816B817C819E012F5F3F4FC8010E9447
:106F60000637882341F1D301C201F801058404C02A
:106F7000880F991FAA1FBB1F0A94D2F7C80ED91EEB
:106F8000EA1EFB1E89819A81AB81BC812789203151
:106F900031F4883F9F4FA105B10530F4D8CF883F29
:106FA0009F4FAF4FBF4098F2F501C082D182E2827D
:106FB000F38281E001C080E00F900F900F900F905E
:106FC000DF91CF911F910F91FF90EF90DF90CF90C5
:106FD000BF90AF907F906F905F904F9008954F92C9
:106FE0005F926F927F928F929F92AF92BF92CF9259
:106FF000DF92EF92FF920F931F93CF93DF93EC01F9
:107000004A015B01280139014230510561057105D2
:1070100008F463C089859A85AB85BC850196A11D5E
:10702000B11D84179507A607B70708F456C08F89C6
:10703000803129F4C52ED62EE72EFF240CC08032D5
:1070400009F04BC06A017B0177E0F694E794D7948E
:10705000C7947A95D1F78B899C89AD89BE89C80E72
:10706000D91EEA1EFB1E41E0C701B6010E94CD36C3
:10707000882399F18F89803159F49924AA24BB245B
:10708000F401EE0FFF1FE554F94F5182408210C00A
:10709000E89487F89924AA24BB24F401EE0FFF1F7B
:1070A000EE0FFF1FE554F94F4082518262827382D6
:1070B0008A89823080F08D819E81AF81B8858C0D68
:1070C0009D1DAE1DBF1D8093B4069093B506A09381
:1070D000B606B093B70681E001C080E0DF91CF91A2
:1070E0001F910F91FF90EF90DF90CF90BF90AF90E6
:1070F0009F908F907F906F905F904F9008952F9208
:107100003F924F925F926F927F929F92AF92BF9207
:10711000CF92DF92EF92FF920F931F93CF93DF9363
:10712000CDB7DEB760970FB6F894DEBF0FBECDBF08
:107130005C014D875E876F87788B1901DC0119969A
:107140002D913D914D915C911C972F5F3F4F4F4F7B
:107150005F4F29873A874B875C87F10140805180D8
:1071600062807380411451046104710431F0FFEFB7
:107170004F1A5F0A6F0A7F0A10C0DC014D905D90C4
:107180006D907C90992493942D853E854F855889E8
:10719000213031054105510509F0912C730162013F
:1071A0001D821E821F821886F50181859285A38526
:1071B000B4852D813E814F815885281739074A07AC
:1071C0005B0708F056C089859A85AB85BC858C1510
:1071D0009D05AE05BF0550F4F2E0CF2ED12CE12C79
:1071E000F12CA2E04A2E512C612C712C9E012F5FB4
:1071F0003F4FB701A601C5010E9406378823C9F198
:1072000049815A816B817C81D701C6010196A11DFC
:10721000B11D452B462B472B19F02C013D010DC00C
:1072200084199509A609B7092D853E854F8558898A
:1072300082179307A407B50789F08D819E81AF81DE
:10724000B8850196A11DB11D8D839E83AF83B8873C
:107250009FEFC91AD90AE90AF90AA6CF0FEF1FEF63
:107260002FEF3FE0A601B701C5010E94EF37811162
:107270001BC080E044C0A70196012150310941099B
:1072800051092D833E834F835887970186014D8195
:107290005E816F817885C5010E94EF37882349F3AD
:1072A000CD80DE80EF80F8844C145D046E047F0492
:1072B00010F3D1014D915D916D917C914115510576
:1072C0006105710541F4F10140825182628273824D
:1072D000911009C013C093018201C5010E94EF37CC
:1072E0008111F1CFC6CFFFEF4F1A5F0A6F0A7F0AF5
:1072F000D5014D925D926D927C92139781E06096DC
:107300000FB6F894DEBF0FBECDBFDF91CF911F91B6
:107310000F91FF90EF90DF90CF90BF90AF909F9034
:107320007F906F905F904F903F902F900895AF9215
:10733000BF92CF92DF92EF92FF920F931F93CF9362
:10734000DF9300D000D0CDB7DEB75C016A017B01CE
:1073500082E090E0A0E0B0E0F50180839183A28319
:10736000B3839E012F5F3F4FB701A601C5010E9465
:107370000637811102C080E023C000E010E09801D0
:10738000B701A601C5010E94EF378823A1F3C98088
:10739000DA80EB80FC80F5018789803141F4F8EFD9
:1073A000CF16FFEFDF06E104F10448F4DACF88EFEF
:1073B000C8168FEFD806E8068FE0F80690F281E055
:1073C0000F900F900F900F90DF91CF911F910F9121
:1073D000FF90EF90DF90CF90BF90AF9008958F9285
:1073E0009F92AF92BF92CF92DF92EF92FF921F9344
:1073F000CF93DF93EC01142F7093BA066093B90614
:107400001F8A82E090E0A0E0B0E088839983AA839D
:10741000BB831092B8061092B4061092B506109273
:10742000B6061092B7068FEF9FEFDC018093BB0882
:107430009093BC08A093BD08B093BE08442351F1BB
:10744000453008F0DFC040E060E070E0CB010E9412
:10745000CD36882309F4D6C020E1129FF001112413
:10746000E759F74F80818F7709F0CCC084859585E7
:10747000A685B78584369105A105B10508F4C2C07B
:10748000C084D184E284F384C114D104E104F10402
:1074900021F4B8C0C12CD12C760140E0C701B6015F
:1074A0000E94CD36882309F4ADC08091C606909124
:1074B000C7068115924009F0A5C03091CB06332351
:1074C00009F4A0C08091C9069091CA06892B09F4DD
:1074D00099C02091C806222309F494C03A8B2C83CA
:1074E0001D8630E041E050E006C0812F8F5F8D8720
:1074F000183008F087C01D85CA01012E02C0880F10
:10750000991F0A94E2F72817390779F72091D106D5
:107510003091D2062115310519F040E050E008C045
:107520002091DF063091E0064091E1065091E2069D
:107530002D833E834F8358878091C9069091CA0658
:1075400046015701880E991EA11CB11C8B8A9C8A8A
:10755000AD8ABE8AE091CC06F091CD06F98FE88F16
:10756000A091CB06B0E00E940272680D791D8A1DC1
:107570009B1D6A8F7B8F8C8F9D8FB5E0EE0FFF1F59
:10758000BA95E1F7E150FE4FEF2FFF27E695DC01BA
:10759000CB018E0F9F1FA11DB11D8E879F87A88BCA
:1075A000B98B8090CE069090CF068114910419F08B
:1075B000A12CB12C08C08090DB069090DC06A09036
:1075C000DD06B090DE06A7019601281B390B4A0B99
:1075D0005B0BDA01C901880D991DAA1DBB1D04C0F2
:1075E000B695A795979587951A95D2F789879A8723
:1075F000AB87BC87853F3FE09307A105B10520F429
:107600008CE08F8B80E016C0853F9F4FA105B105B0
:1076100010F480E10DC08091E7069091E806A091FA
:10762000E906B091EA068A8F9B8FAC8FBD8F80E20E
:107630008F8B81E0DF91CF911F91FF90EF90DF90D2
:10764000CF90BF90AF909F908F9008952F923F92D0
:107650004F925F926F927F928F929F92AF92BF9262
:10766000CF92DF92EF92FF920F931F93CF93DF930E
:10767000CDB7DEB7CA54D1090FB6F894DEBF0FBE3E
:10768000CDBF3C017E8B6D8B4A012FA309A7EBAACE
:10769000ACAABDAACEAADFAA34E0239F80011124A0
:1076A000400F511F58AB4FA7DA01CD90DD90ED9000
:1076B000FC90FC01E00FF11F208131814281538158
:1076C000C701B6010E948E6D68AF79AF8AAF9BAFDC
:1076D000E9A5B4E0EB9F200111249401240D351D90
:1076E0003AAB29ABD9018D909D90AD90BC90F30140
:1076F000E40DF51D2081318142815381C501B40122
:107700000E948E6D6CAF7DAF8EAF9FAFEBA9B4E0E2
:10771000EB9FC0011124F301E80FF91F2081318193
:10772000428153812F8B388F498F5A8FED89FE8983
:10773000E80FF91F60817181828193810E948D6DB4
:10774000462F572F682F792F4D8F5E8F6F8F78A31D
:10775000AD89BE891C968D919D910D90BC91A02DF7
:107760008BA79CA7ADA7BEA7D3011C962D913D91D9
:107770004D915C911F9729A33AA34BA35CA3A7014A
:1077800096015058298B3A8B4B8B5C8BB7FAB0948F
:10779000B7F8B094ED89FE89E00FF11F78AD69ADBF
:1077A0009AAD8BAD272F362F492F582F60817181CD
:1077B000828193810E948D6D162F072F382E292EDE
:1077C000ED89FE89E40DF51D7CAD6DAD9EAD8FADEF
:1077D000272F362F492F582F608171818281938105
:1077E0000E948D6D762E672E582E492EB801C1014C
:1077F000272F362F492F582F69897A898B899C89A1
:107800000E943C716B017C01B301C201272F362F0E
:10781000492F582FC501B4010E943C719B01AC0156
:10782000C701B6010E948E6D6B017C01B301C201DC
:10783000272F362F492F582F69897A898B899C8960
:107840000E943C712B013C01B801C101272F362F4A
:10785000492F582FC501B4010E943C719B01AC0116
:10786000C301B2010E948D6DA70196010E94016EB5
:10787000562E472E782E692E20E030E0A901D20145
:10788000F3016B2F7A2F8F2F9E2F0E94676E87FF39
:1078900010C02BED3FE049EC50E4D201F3016B2F17
:1078A0007A2F8F2F9E2F0E948E6D562E472E782E68
:1078B000692EA4968FADA497882381F02BED3FE02D
:1078C00049EC50E4D201F3016B2F742D8F2F962DCC
:1078D0000E948D6D562E472E782E692ECD8CDE8C13
:1078E000EF8CF8A0E894F7F8A3962CAD3DAD4EAD23
:1078F0005FADA397D201F3016B2F742D8F2F962DBF
:107900000E943C71A70196010E9477706B017C0177
:107910002FE632E143E85AE30E94676E87FD23C2F7
:10792000C701B6010E94446F0E94DB6E7EA36DA367
:107930006115710521F481E090E09EA38DA3ADA1B6
:10794000BEA1BD0180E090E00E94076F6B017C0149
:107950009B01AC01D201F3016B2F742D8F2F962D5B
:107960000E946E6E6B8F7C8F1C01A70196016D8D3E
:107970007E8D8F8D98A10E946E6E24966FAF249796
:1079800025967FAF259726968FAF269727969FAF90
:10799000279729A13AA14BA15CA16BA57CA58DA538
:1079A0009EA50E948D6DA70196010E946E6E28967D
:1079B0006FAF289729967FAF29972A968FAF2A977E
:1079C0002B969FAF2B9720E030E040E05FE3BB8D2C
:1079D000AC8D6B2F7A2F822D932D0E943C71BB8D25
:1079E000AC8D2B2F3A2F422D532D0E943C719B01C1
:1079F000AC0160E070E080E89FE30E948D6D6BA7B2
:107A000021967FAF219722968FAF229723969FAF23
:107A10002397CE010196FC012BA9B4E02B9FE00D2A
:107A2000F11D11242F89388D498D5A8D2083318382
:107A30004283538329A13AA14BA15CA12D873E87A4
:107A40004F87588B512C41E050E0588F4F8B81E08D
:107A500090E08C0F9D1FBFA1A4E0BA9F800D911DE7
:107A6000112498A78FA321E030E02C0F3D1F59A5CA
:107A700044E0549F200D311D11243AA729A7FAA3F1
:107A8000E9A350C188E185150CF45EC07B8D6C8D37
:107A9000272F362F422D532D69897A898B899C890E
:107AA0000E943C716B017C017BA521966FAD2197F3
:107AB00022969FAD229723968FAD2397272F362F9F
:107AC000492F582FC501B4010E943C719B01AC01A4
:107AD000C701B6010E948E6D7B018C017BA52196AA
:107AE0006FAD219722969FAD229723968FAD239756
:107AF000272F362F492F582F69897A898B899C899E
:107B00000E943C713B016C017B8D6C8D272F362FC1
:107B1000422D532DC501B4010E943C719B01AC0163
:107B2000662D772D8C2D9D2D0E948D6D462F572F04
:107B3000682F792F498B5A8B6B8B7C8B53948E2CAF
:107B40009F2CA02EB12E6FC0AF89B88DBD0180E0F3
:107B500090E00E94076FBB8DAC8D2B2F3A2F422DEA
:107B6000532D0E943C717B018C017F2D802F912F22
:107B70000E946B6E6D8F7E8F8F8F98A36E2D7F2DE1
:107B8000802F912F0E949F714B015C01EFA5F8A9F6
:107B9000C080D180E280F380F7FAF094F7F8F09497
:107BA000A9A9BAA94D905D906D907C902D8D3E8DC8
:107BB0004F8D58A1C701B6010E943C71698B7A8B29
:107BC0008B8B9C8BA5019401C301B2010E943C7177
:107BD0009B01AC0169897A898B899C890E948E6D91
:107BE000462F572F682F792F498B5A8B6B8B7C8BA5
:107BF000A5019401C701B6010E943C716B017C0193
:107C00002D8D3E8D4F8D58A1C301B2010E943C7154
:107C10009B01AC01C701B6010E948D6D862E972E87
:107C2000A82EB92E512C29893A894B895C89B8AD87
:107C3000A9ADFAADEBAD6B2F7A2F8F2F9E2F0E943F
:107C40008E6DEFA1F8A56083718382839383A50174
:107C50009401BCADADADFEADEFAD6B2F7A2F8F2F84
:107C60009E2F0E948E6DA9A5BAA56D937D938D93CD
:107C70009C93139724967FAD249725966FAD2597F7
:107C800026969FAD269727968FAD2797272F362FBD
:107C9000492F582FE9A1FAA16081718182819381D6
:107CA0000E948E6DA9A1BAA16D937D938D939C9333
:107CB000139728967FAD289729966FAD29972A9616
:107CC0009FAD2A972B968FAD2B97272F362F492FB5
:107CD000582F6D857E858F8598890E948E6D6D8762
:107CE0007E878F87988BCE0101960E94821694E63C
:107CF000C92ED12CCC0EDD1EECA8FDA80EA91FA903
:107D00009E01235F3F4FAE01475F5F4FBE016B5F38
:107D10007F4FCE0101960E947B44EF89F88D31960A
:107D2000F88FEF8B2F89388D4DA15EA12417350771
:107D300008F4A8CE2D893E89245F3F4F4D895E8986
:107D4000485F5F4F6D897E896C5F7F4F84E6C82EE8
:107D5000D12CCC0EDD1EECA8FDA80EA91FA98D8983
:107D60009E890E947B44C65BDF4F0FB6F894DEBF4E
:107D70000FBECDBFDF91CF911F910F91FF90EF907C
:107D8000DF90CF90BF90AF909F908F907F906F903B
:107D90005F904F903F902F9008952F923F924F9277
:107DA0005F926F927F928F929F92AF92BF92CF928B
:107DB000DF92EF92FF920F931F93CF93DF93CDB794
:107DC000DEB768970FB6F894DEBF0FBECDBF1C01BB
:107DD0002A013B0168017901DC01D8966D917D9102
:107DE0008D919C91DB970E94076F4B015C01A30171
:107DF00092010E943C710E94546E0E94DB6E698366
:107E00007A838B839C83A7019601C501B4010E94EC
:107E10003C710E94546E0E94DB6E6D837E838F8363
:107E2000988729813A814B815C812837310541054A
:107E3000510540F488E790E0A0E0B0E089839A83A0
:107E4000AB83BC832D813E814F8158852837310516
:107E50004105510540F488E790E0A0E0B0E08D8353
:107E60009E83AF83B88791012C5B3F4FD9018D91E1
:107E70009D910D90BC91A02D8D879E87AF87B88B6B
:107E8000BC01CD010E94096F69877A878B879C8727
:107E9000F10164AD75AD86AD97AD0E94076F698B3A
:107EA0007A8B8B8B9C8B20E030E0A90169857A85E9
:107EB0008B859C850E94676E882339F1A50194010A
:107EC000C501B4010E943C712B013C0129893A890A
:107ED0004B895C89CA01B9010E943C719B01AC01CC
:107EE000C301B2010E948D6D2B013C0129853A85A9
:107EF0004B855C85CA01B9010E948E6D9B01AC0166
:107F0000C301B2010E946E6E04C060E070E080E0C8
:107F100090E00E94546E0E94D66E6B017C016D85CC
:107F20007E858F85988990958095709561957F4F16
:107F30008F4F9F4F0E94096F2B013C01F101E05CC4
:107F4000FF4F60817181828193810E94076F6D87ED
:107F50007E878F87988B20E030E0A901C301B201B2
:107F60000E94676E882349F12D853E854F8558898B
:107F7000CA01B9010E943C716D8B7E8B8F8B988FEB
:107F8000A5019401C501B4010E943C719B01AC01A3
:107F90006D897E898F89988D0E948D6D4B015C0162
:107FA000A3019201C301B2010E948E6D9B01AC013D
:107FB000C501B4010E946E6E04C060E070E080E014
:107FC00090E00E94446FD10150964D905D906D906D
:107FD0007C905397530142018C189D08AE08BF084E
:107FE0000E94D66E861A970AA80AB90AB7FE6CC014
:107FF00020E030E0A90169857A858B859C850E9407
:10800000676E882309F447C029853A854B855C85CE
:10801000CA01B9010E948E6D4B015C01C301B2011E
:108020000E94076F9B01AC01C501B4010E943C7125
:108030004B015C0129893A894B895C89CA01B901E4
:108040000E943C719B01AC01C501B4010E948D6D81
:108050004B015C012D853E854F855889CA01B901C8
:108060000E943C719B01AC01C501B4010E948E6D60
:108070004B015C0120E030E040E850E469857A85FE
:108080008B859C850E943C719B01AC01C501B401AC
:108090000E946E6E04C060E070E080E090E00E949C
:1080A000546E0E94D66E6B017C01F7FE03C0C12C9A
:1080B000D12C7601C414D504E604F70410F0730142
:1080C0006201812C912C54018FB7F894F101E45B8B
:1080D000FF4F9081911121C0F101C48AD58AE68AAF
:1080E000F78A8C0C9D1CAE1CBF1CD101808E918E1A
:1080F000A28EB38E29813A814B815C8124AF35AF4A
:1081000046AF57AFA05CBF4F2D813E814F81588550
:108110002D933D934D935C9313978FBF68960FB645
:10812000F894DEBF0FBECDBFDF91CF911F910F91AD
:10813000FF90EF90DF90CF90BF90AF909F908F9087
:108140007F906F905F904F903F902F9008958F9207
:108150009F92AF92BF92CF92DF92EF92FF920F93D6
:108160001F93CF93DF93EB016A01209709F46CC052
:108170004115510509F468C0EAA4FBA40CA51DA58E
:108180002E2D3F2D402F512F6EA17FA188A599A59F
:108190000E94676E882309F457C08FA9811146C0D9
:1081A000F60186A097A0A0A4B1A4A50194016E2D0C
:1081B0007F2D802F912F0E946A701816BCF5A501A3
:1081C0009401C501B4010E943C714B015C018AA974
:1081D0009BA9ACA9BDA9BC01CD0190589B01AC01E4
:1081E0000E948E6D2EA53FA548A959A90E943C71F9
:1081F0009B01AC01C501B4010E948D6D0E94A97163
:108200005B016C01762F272F3B2D4C2D5D2D6E2DA4
:108210007F2D802F912F0E94676E87FF02C057012C
:1082200068015A2D4B2D3C2D2D2D04C05E2D4F2D58
:10823000302F212F852F942FA32FB22F8EA39FA3F2
:10824000A8A7B9A781E08EABDF91CF911F910F91C5
:10825000FF90EF90DF90CF90BF90AF909F908F9066
:108260000895CF92DF92EF92FF920F931F93CF93D7
:10827000DF931F92CDB7DEB78091C1088FB7F89416
:10828000F090C0088FBF8091C10890E08F199109CC
:108290008F709927049704F12091C10823502F7003
:1082A00040E050E000E010E08DE4E82E13C0211122
:1082B00001C020E12150E29E6001112482EC98E08F
:1082C000C80ED91EB801C60129830E94A740A80183
:1082D000860129812F11EBCF0F90DF91CF911F9154
:1082E0000F91FF90EF90DF90CF9008954F925F92A3
:1082F0006F927F92AF92BF92CF92DF92EF92FF92F6
:108300000F931F93CF93DF938C01EB01009709F438
:1083100060C0FC0187A981115CC046A057A060A481
:1083200071A4AEA0BFA0C8A4D9A42A2D3B2D4C2D6A
:108330005D2DC301B2010E94676E87FF4AC0A30191
:108340009201C301B2010E943C712B013C01F80172
:1083500082A993A9A4A9B5A9BC01CD0190589B01FC
:10836000AC010E948E6DF80126A537A540A951A940
:108370000E943C719B01AC01C301B2010E948D6D52
:108380000E94A9717B018C01762F272F3F2D402F52
:10839000512F6A2D7B2D8C2D9D2D0E94676E87FF9E
:1083A00002C0750186012E2D3F2D402F512F6A2DC1
:1083B0007B2D8C2D9D2D0E94676E882351F08E2D74
:1083C0009F2DA02FB12F8EA39FA3A8A7B9A781E0AF
:1083D0008EABDF91CF911F910F91FF90EF90DF90C7
:1083E000CF90BF90AF907F906F905F904F90089527
:1083F000EF92FF920F931F93CF93DF93F090C008FB
:10840000C0E0D0E080E090E02DE4E22E11C0EF9CCF
:10841000800111240E53174FA801BE010E9476411E
:108420008F2D8F5F803109F480E0F82ECE01E801B6
:108430002091C108F212EBCF40E050E0BE01DF9185
:10844000CF911F910F91FF90EF900C9476414F9236
:108450005F926F927F928F929F92AF92BF92CF92D4
:10846000DF92EF92FF920F931F93CF93DF93909041
:10847000C008C0E0D0E03DE4832E37C0889E5001A4
:10848000899EB00C112482EC98E0A80EB91E2097AA
:1084900031F18EA9811104C0F50186A98823F9F074
:1084A000CAA0DBA0ECA0FDA0A7019601F50166A182
:1084B00077A180A591A50E946E6E2B013C01A701BA
:1084C00096016EA17FA188A599A50E946E6EAB0151
:1084D000BC0193018201CE010E94CD3E1EAA93945D
:1084E000F0E19F1201C0912CE501892D992787FDAC
:1084F00090952091C10830E08217930709F0BECF14
:108500002097F1F0CAA0DBA0ECA0FDA0A701960186
:108510006DEC7CEC8CE49DE30E946E6E4B015C0183
:10852000A70196016EA17FA188A599A50E946E6EF4
:10853000AB01BC0195018401CE010E94CD3E1EAA73
:10854000DF91CF911F910F91FF90EF90DF90CF902F
:10855000BF90AF909F908F907F906F905F904F9063
:1085600008950E9431410E94F8410C9427421092D4
:10857000C1081092C00880E1E3E9FDE0DF011D922F
:108580008A95E9F71092030E1092040E1092050ED0
:108590001092060E1092070E1092080E1092090EFD
:1085A00010920A0E10920B0E10920C0E10920D0EDD
:1085B00010920E0E10920F0E1092100E1092110EBD
:1085C0001092120E1092130E1092140E1092150E9D
:1085D0001092160E08954F925F926F927F928F9233
:1085E0009F92AF92BF92CF92DF92EF92FF920F9342
:1085F0001F93CF93DF938091920D882309F41FC1BD
:1086000060E080916C0E90916D0E0E94095800916F
:10861000330110913401D0913501C091360120E031
:1086200030E040E050E40E948E6DFE01202F312F9B
:108630004F2F5E2F0E94676E87FD01C1D090C0084A
:10864000912CA12CB12CC12C4DE4842E5CC02D2D7D
:1086500030E0829EF001839EF00D1124EE53F74F1F
:1086600080819181A281B381892B8A2B8B2B81F40C
:1086700084819581A681B781892B8A2B8B2B41F42C
:1086800080859185A285B385892B8A2B8B2BC1F19F
:10869000829E7001839EF00C112482EC98E0E80E1B
:1086A000F91EF70164857585868597850E94096F97
:1086B0002B013C01F70160897189828993890E94AD
:1086C000076F9B01AC01C301B2010E946E6EF701FE
:1086D00022A133A144A155A10E943C713B017C0120
:1086E000292D3A2D4B2D5C2D662D772D8E2D9F2D0E
:1086F0000E946A70181624F4962CA72CBE2CCF2C3E
:10870000D394FFE0DF228091C108D812A0CF20913E
:108710002F01309130014091310150913201692D8A
:108720007A2D8B2D9C2D0E943C719B01AC01FE018A
:10873000602F712F8F2F9C2F0E948E6D6B017C01FB
:10874000CE01202F312F492F5C2F6C2D7D2D8E2DAA
:108750009F2D0E94676E87FD03C08601DE2DCF2D01
:10876000C0903701D0903801E0903901F0903A0183
:108770002C2D3D2D4E2D5F2DFE01602F712F8F2F43
:108780009C2F0E946A7018161CF06801ED2EFC2EBA
:108790008090170E9090180EA090190EB0901A0E9F
:1087A0002C2D3D2D4E2D5F2DC501B4010E946A7008
:1087B0001816F4F420E037ED43EA5CE36C2D7D2DD0
:1087C0008E2D9F2D0E943C718B01D82FC92F28E43C
:1087D00031EE4AE75FE3C501B4010E943C71FE013E
:1087E000202F312F4F2F5E2F0E948E6D6B017C0149
:1087F0008C2D9D2DAE2DBF2D8093170E9093180EAE
:10880000A093190EB0931A0E6C2D7D2D8E2D9F2DD9
:108810000E94D66EDC01CB0160E00E943957909334
:108820006D0E80936C0E8C2D9D2DAE2DBF2D8093E3
:10883000620E9093630EA093640EB093650EDF9169
:10884000CF911F910F91FF90EF90DF90CF90BF904D
:10885000AF909F908F907F906F905F904F90089512
:10886000CF939091C0088091C108981709F1209189
:10887000C0088DE4289FF0011124E65FF64FC08107
:1088800030E04DE410C0429FF0011124E65FF64F46
:1088900080819181A281B381892B8A2B8B2B09F056
:1088A0003F5F2F5F2F708091C1082813ECCF0AC063
:1088B00060912B03662321F070E08EE00E94562A1F
:1088C000C0E030E080912B03811107C0311105C059
:1088D00060E070E08EE00E94562A80912B0388238E
:1088E00039F0CC2329F06C2F70E08EE00E94562ADC
:1088F000CF910C94EB422F923F924F925F926F92E6
:108900007F928F929F92AF92BF92CF92DF92EF921F
:10891000FF920F931F93CF93DF93CDB7DEB7C85667
:10892000D1090FB6F894DEBF0FBECDBF2C013B01BD
:108930004A015901EBA6FBAA0CA719ABDEAACDAAE6
:108940002091C1082F5F61962FAF6197203119F4F4
:1089500061961FAE619761963FAD6197032F112716
:1089600007FD109504C00E94D3580E94B018809152
:10897000C00890E080179107B1F32091DF0D30918E
:10898000E00D4091E10D5091E20DD2016D917D918C
:108990008D919C910E943C710E940C716CAF7DAFD7
:1089A0008EAF9FAF2091E30D3091E40D4091E50D26
:1089B0005091E60DF30160817181828193810E9463
:1089C0003C710E940C7121966FAF219722967FAF68
:1089D000229723968FAF239724969FAF24972091B9
:1089E000E70D3091E80D4091E90D5091EA0DD40169
:1089F0006D917D918D919C910E943C710E940C71B2
:108A000025966FAF259726967FAF269727968FAF2F
:108A1000279728969FAF28972091EB0D3091EC0D6A
:108A20004091ED0D5091EE0DF501608171818281D3
:108A300093810E943C710E940C7168AF79AF8AAF3C
:108A40009BAF80919F0D9091A00DA091A10DB09131
:108A5000A20D28AD39AD4AAD5BAD281739074A07DD
:108A60005B07C1F160912C03E62FF0E0EE0FFF1FD2
:108A7000E859F14F808191810E94095820E030E04F
:108A800046E153E40E94676E87FF24C08091BF08CF
:108A9000811120C00C94BA4E9091C00095FFFCCF7C
:108AA0008093C600319684918111F6CFE0EAF6E01A
:108AB00007C09091C00095FFFCCF8093C60031960F
:108AC00084918111F6CF8091C00085FFFCCF8AE0B0
:108AD0008093C60080919F0D9091A00DA091A10D53
:108AE000B091A20D28AD39AD4AAD5BAD281B390B55
:108AF0004A0B5B0BCA01B90157FF07C090958095DF
:108B0000709561957F4F8F4F9F4F0E94096F6B014A
:108B10007C0120E030E04DEC53E46091EB0D70916E
:108B2000EC0D8091ED0D9091EE0D0E943C719B013A
:108B3000AC01C701B6010E946A7018166CF548AD09
:108B400059AD6AAD7BAD40939F0D5093A00D6093DE
:108B5000A10D7093A20DEAE9F6E007C09091C00064
:108B600095FFFCCF8093C600319684918111F6CF9A
:108B7000EAEBF6E007C09091C00095FFFCCF809330
:108B8000C600319684918111F6CF8091C00085FF97
:108B9000FCCF8AE08093C6008091C1085DE4859F88
:108BA0001001112462EC78E0260E371EF101E45B1F
:108BB000FF4F10828091930D9091940DA091950D8F
:108BC000B091960D8BA39CA3ADA3BEA38CAC9DAC22
:108BD000AEACBFAC881A990AAA0ABB0AB7FE08C095
:108BE000B094A09490948094811C911CA11CB11C01
:108BF000D1018D929D92AD92BC9213972091970DC9
:108C00003091980D4091990D50919A0D2FA338A74E
:108C100049A75AA72496CCACDDACEEACFFAC2497A8
:108C2000C21AD30AE40AF50AF7FE08C0F094E094E9
:108C3000D094C094C11CD11CE11CF11CD10114962C
:108C4000CD92DD92ED92FC92179740909B0D509043
:108C50009C0D60909D0D70909E0D28968CAD9DADE5
:108C6000AEADBFAD289784199509A609B709B7FF1E
:108C700007C0B095A095909581959F4FAF4FBF4F7E
:108C8000182F092FAFAB6296BFAF6297F1018087B3
:108C90009187A287B38720919F0D3091A00D4091BD
:108CA000A10D5091A20D2DA73EA74FA758ABA091A3
:108CB0001201B091130128AD39AD4AAD5BAD6DA580
:108CC0007EA58FA598A9261B370B480B590B57FF7C
:108CD00007C050954095309521953F4F4F4F5F4FBE
:108CE0000E940D7224E630E040E050E00E945B728A
:108CF000D1011C962D933D934D935C931F97812F2B
:108D0000902FAFA96296BFAD62978C159D05AE05F9
:108D1000BF0514F4D701C60182179307A407B5074E
:108D200014F4DA01C901B501A40188169906AA064E
:108D3000BB0614F4AC01BD01F101408B518B628B79
:108D4000738B463051056105710510F40C94CA4EC1
:108D5000E85BFF4F80912B0390E0A0E0B0E08083C0
:108D60009183A283B3832CAD3DAD4EAD5FAD6BA1BE
:108D70007CA18DA19EA1261737074807590724F02B
:108D8000D10190961C9203C081E0F10180A324964A
:108D90002CAD3DAD4EAD5FAD24976FA178A589A5F3
:108DA0009AA526173707480759073CF4D101909632
:108DB0008C919097826090968C9328962CAD3DADC7
:108DC0004EAD5FAD289724153505460557053CF493
:108DD000D10190968C919097846090968C9328AD59
:108DE00039AD4AAD5BAD6DA57EA58FA598A92617B7
:108DF0003707480759073CF4D10190968C9190971A
:108E0000886090968C93EDA9FEA98081D1019196FE
:108E10008C9389288A288B2809F05A9AF101848139
:108E20009581A681B781892B8A2B8B2B09F05A9AC1
:108E3000F10180859185A285B385892B8A2B8B2BA7
:108E400009F05A9AF10184859585A685B785892B05
:108E50008A2B8B2B09F05A9AD1011C962D913D91AA
:108E60004D915C911F976B962CAF3DAF4EAF5FAFAE
:108E70006B97232B242B252BE9F48090B30D909036
:108E8000B40D0091B50D1091B60D282D392D402F40
:108E9000512FBBA5ABA9FCA5E9A96B2F7A2F8F2F6A
:108EA0009E2F0E94676E87FD0EC08BA49BA80CA509
:108EB00019A909C08090CB0D9090CC0D0091CD0DDB
:108EC0001091CE0DE2CF6CAD7DAD8EAD9FAD2BA1DF
:108ED0003CA14DA15EA1621B730B840B950B0E94FC
:108EE000096F2091DF0D3091E00D4091E10D50911F
:108EF000E20D0E946E6E6BA37BA78BAB9CA7472FE6
:108F0000382F292F862F942FA32FB22F898B9A8B3E
:108F1000AB8BBC8B24966CAD7DAD8EAD9FAD249795
:108F20002FA138A549A55AA5621B730B840B950B7D
:108F30000E94096F2091E30D3091E40D4091E50D01
:108F40005091E60D0E946E6E6FA379AB8DAB9FAB17
:108F5000472F382F292F862F942FA32FB22F8D8B99
:108F60009E8BAF8BB88F28966CAD7DAD8EAD9FADCF
:108F7000289764197509860997090E94096F20913D
:108F8000E70D3091E80D4091E90D5091EA0D0E94F6
:108F90006E6E762E672E582E492EA3019201852FD4
:108FA000942FA32FB22F898F9A8FAB8FBC8FA09055
:108FB0001201B090130168AD79AD8AAD9BAD2DA5BE
:108FC0003EA54FA558A9621B730B840B950B0E94FD
:108FD000096F2091EB0D3091EC0D4091ED0D50910A
:108FE000EE0D0E946E6E6B017C01B501882777FD46
:108FF0008095982F0E94096F9B01AC01C701B601B3
:109000000E943C7120E030E048EC52E40E946E6E19
:10901000F62FE72F382F292F862F9E2FA32FB22F21
:109020004F2F5E2F632F722F4D8F5E8F6F8F78A320
:10903000F101408151816281738160964CAF5DAFD7
:109040006EAF7FAF60974630510561057105C4F47E
:1090500044815581668177814630510561057105EE
:109060007CF44085518562857385463051056105E4
:10907000710534F4BF7786A797A7A0ABB1AB3BC00F
:109080005BA14BA53BA92CA5652F742F832F922F95
:109090000E94E7716B017C015FA149A93DA92FA93D
:1090A000652F742F832F922F0E94E7719B01AC01D3
:1090B000C701B6010E948E6DF62EE72ED82EC92E5E
:1090C000A3019201652F762D832F942D0E94E771C5
:1090D0009B01AC01D701F6016B2F7A2F8F2F9E2FAA
:1090E0000E948E6D0E94A971D1019E966D937D9311
:1090F0008D939C93D197D1019E962D913D914D9149
:109100005C91D19765962CAF3DAF4EAF5FAF659741
:1091100060E070E080E89FE30E946E6E9B01AC010E
:10912000682D792D802F912F0E943C716DAB7FAB04
:109130008C019091C1088091C008E92FF0E0E81BF4
:10914000F109EF70FF27FCABEBAB762F6FA9272F50
:10915000362F402F512F60E074E284E799E40E949B
:109160006E6E0E940C71B62EA72E982E892E2BA9FA
:109170003CA9223031050CF44BC06901EE24D7FC28
:10918000E094FE2CC701B6010E94096F20E030E098
:1091900040E051E40E94676E87FF3AC04B2C5A2C86
:1091A000692C782C8091FF0D9091000EA091010EFA
:1091B000B091020E481659066A067B0648F5BC01B6
:1091C000CD016419750986099709660F771F881FF5
:1091D000991FA70196010E943972CA01B9010E9424
:1091E000076F0E940C71AB01BC01CB01BA01640D89
:1091F000751D861D971D0E94076F9B01AC0160E0E5
:1092000074E284E799E40E946E6E6DAB7FAB8C01D3
:109210007DA96FA9272F362F402F512F65966CAD52
:109220007DAD8EAD9FAD65970E943C71A0966FAFEE
:10923000A097A4967FAFA497A5968FAFA597A69663
:109240009FAFA697472F382F292F862F942FA32F14
:10925000B22FF10182A393A3A4A3B5A3608971895E
:10926000828993890E94076F6BA37CA38DA39EA321
:109270007DA96FA9272F362F402F512F6BA17CA1DD
:109280008DA19EA10E943C710E94546E0E94DB6ED3
:109290006B017C01D101D8966D937D938D939C9346
:1092A000DB97FE0171962A96FFAFEEAF2A979E01DB
:1092B0002F5F3F4F3AAB29AB4FEE5DE06D965FAF4E
:1092C0004EAF6D97BE016F5D7F4F7AA369A367961E
:1092D0003FAF2EAF67971FA21DA670E87BA78FE355
:1092E0008CA72A96AEADBFAD2A976D917D918D91D9
:1092F0009D912A96BFAFAEAF2A97BDA9AFA92B2FDC
:109300003A2F402F512F0E943C712B013C01679650
:10931000EEADFFAD6797419251926192719267965F
:10932000FFAFEEAF6797E89477F86D96AEADBFAD3F
:109330006D978D909D90AD90BD906D96BFAFAEAF87
:109340006D97A5019401C301B2010E946A701816BD
:1093500004F5A3019201C501B4010E946E6EB62E00
:10936000A72E982E892EB501C401272F362F492FFD
:10937000582FBFA1ADA5FBA5ECA56B2F7A2F8F2F82
:109380009E2F0E94676E87FD04C0BFA2ADA69BA65C
:109390008CA62A96EEADFFAD2A9729A13AA1E21735
:1093A000F30709F09ECF20E030E040E85FE3BFA183
:1093B000ADA5FBA5ECA56B2F7A2F8F2F9E2F0E94BA
:1093C000676E87FF54C08E010F5E1F4F7FA16DA592
:1093D0009BA58CA5272F362F492F582FA9A9BAA9AD
:1093E0006D917D918D919C910E943C71E9A9FAA9A2
:1093F0006193719381939193FAABE9ABE017F10715
:1094000029F77FA16DA59BA58CA5272F362F492F66
:10941000582FA096BFADA097A496AFADA497A596E0
:10942000FFADA597A696EFADA6976B2F7A2F8F2F3E
:109430009E2F0E943C71D10192966D937D938D93E6
:109440009C939597C701B6010E94076FBFA1ADA578
:10945000FBA5ECA52B2F3A2F4F2F5E2F0E943C71BE
:109460000E94DB6EF10160AF71AF82AF93AF659682
:109470002CAD3DAD4EAD5FAD65976BA17CA18DA1CF
:109480009EA10E946E6E762E672E582E492E6096F3
:109490002CAD3DAD4EAD5FAD6097232B242B252B1E
:1094A00079F5F10184819581A681B781892B8A2B79
:1094B0008B2B31F580859185A285B385892B8A2BED
:1094C0008B2BF1F42091C30D3091C40D4091C50D4B
:1094D0005091C60DD301F2016B2F7A2F8F2F9E2F43
:1094E0000E943C710E94546E81010C5B1F4F0E94D0
:1094F000DB6ED8016D937D938D939C931397FCC085
:109500002091C70D3091C80D4091C90D5091CA0DE1
:10951000D301F2016B2F762D8F2F942D0E943C7179
:109520000E94546E0E94DB6E81010C5B1F4FF8019C
:1095300060837183828393838090A30D9090A40DA8
:10954000A090A50DB090A60D0E94076F6B017C0145
:1095500060966CAD7DAD8EAD9FAD60970E94096F3A
:109560009B01AC01C701B6010E943C712BA13CA13B
:109570004DA15EA10E946E6E6B017C01C501B4011C
:109580000E94076F9B01AC01C701B6010E946A707F
:10959000181634F4D8018D929D92AD92BC92139717
:1095A0008090A70D9090A80DA090A90DB090AA0D45
:1095B000F80160817181828193810E94076F6B0144
:1095C0007C01D10114966D917D918D919C9117979D
:1095D0000E94096F9B01AC01C701B6010E943C715A
:1095E0002BA13CA14DA15EA10E946E6E6B017C017E
:1095F000C501B4010E94076F9B01AC01C701B60110
:109600000E946A7018162CF4F80180829182A2825E
:10961000B3828090AF0D9090B00DA090B10DB0903E
:10962000B20D81010C5B1F4FD8016D917D918D9121
:109630009C910E94076F6B017C016B966CAD7DADB8
:109640008EAD9FAD6B970E94096F9B01AC01C70166
:10965000B6010E943C712BA13CA14DA15EA10E94CC
:109660006E6E6B017C01C501B4010E94076F9B0106
:10967000AC01C701B6010E946A7018162CF4F801FB
:1096800080829182A282B3828090AB0D9090AC0DCB
:10969000A090AD0DB090AE0DD8016D917D918D91E2
:1096A0009C910E94076F6B017C01F10160857185BF
:1096B000828593850E94096F9B01AC01C701B601A9
:1096C0000E943C712BA13CA14DA15EA10E946E6E37
:1096D0006B017C01C501B4010E94076F9B01AC01C5
:1096E000C701B6010E946A70181634F4D8018D9231
:1096F0009D92AD92BC921397F101EC5BFF4F60819C
:109700007181828193810E94076F6B017C01B3019B
:10971000C201272F362D492F542DC701B6010E94B3
:109720006E6EF62FE72F382F292F862F9E2FA32F0F
:10973000B22FA9968CAF9DAFAEAFBFAFA9974F2FF9
:109740005E2F632F722FF10142AB53AB64AB75AB4D
:109750002DEB37E346E051E4C701B6010E943C71AE
:109760000E94D66ED1015C966D937D938D939C93F0
:109770005F978090BF0D9090C00DA090C10DB090EC
:10978000C20D20E030E040E05FE3C501B4010E947B
:109790003C716BA37FA38DA79BA729853A854B8539
:1097A0005C856F962CAF3DAF4EAF5FAF6F9740912A
:1097B000BB0D5091BC0D6091BD0D7091BE0D2C96EE
:1097C0004CAF5DAF6EAF7FAF2C9720E030E040E054
:1097D0005FE32C966CAD7DAD8EAD9FAD2C970E9456
:1097E0003C71F62EE72ED82EC92E6F966CAD7DAD4E
:1097F0008EAD9FAD6F979F77D701F6012B2F3A2F34
:109800004F2F5E2F0E946A701816B4F4B701C6017C
:10981000272F362F492F582FBBA1AFA1FDA5EBA5B0
:109820006B2F7A2F8F2F9E2F0E94676E87FD04C0AB
:10983000FBA2EFA2DDA6CBA66D857E858F859889DC
:10984000A3966CAF7DAF8EAF9FAFA397C090B70DBF
:10985000D090B80DE090B90DF090BA0D20E030E056
:1098600040E05FE3C701B6010E943C71762E672E8F
:10987000582E492EA3966CAD7DAD8EAD9FADA397AE
:109880009F77D301F2012B2F3A2F4F2F5E2F0E948B
:109890006A701816B4F4B301C201272F362F492F6E
:1098A000582FBBA1AFA1FDA5EBA56B2F7A2F8F2F52
:1098B0009E2F0E94676E87FD04C07BA26FA25DA6EB
:1098C0004BA6D1019296BC91BCA7F101F3A1F9ABD3
:1098D000D1019496BC91BDABF101F5A1FFAB7CA584
:1098E00069A9272F362F4B2F5F2FBBA1AFA1FDA555
:1098F000EBA56B2F7A2F8F2F9E2F0E94676E87FD0F
:1099000008C02CA52BA339A93FA34DA94DA75FA93A
:109910005BA76BA97CA9623071050CF434C170910E
:10992000130E7BAB8091140E2D968FAF2D979091D7
:10993000150E66969FAF6697A091160E6896AFAF0C
:10994000689727E137EB41ED58E36896EFAD6897EC
:10995000672F782F892F9E2F0E946A7018160CF09F
:1099600012C12091030E3091040E4091050E5091CA
:10997000060E69817A818B819C810E948D6D762E85
:10998000672E582E492E2091070E3091080E4091D7
:10999000090E50910A0E6D817E818F8198850E94FB
:1099A0008D6D162F072FA4968FAFA497A5969FAF06
:1099B000A597B301C201272F362F492F582FD30166
:1099C000F2016B2F7A2F8F2F9E2F0E943C712B015B
:1099D0003C01B801A4969FADA497A5968FADA5971D
:1099E000272F362F492F582FD801FC016B2F7A2FA4
:1099F0008F2F9E2F0E943C719B01AC01C301B201CD
:109A00000E948E6D0E94A9712B013C01A501940159
:109A10000E946A7018164CF4A3019201C501B401AA
:109A20000E946E6E3B018C0104C0612C712C00E819
:109A30001FE320910B0E30910C0E40910D0E5091B2
:109A40000E0E6F966CAD7DAD8EAD9FAD6F970E9483
:109A50008D6D4B015C01E894B7F82C962CAD3DADB3
:109A60004EAD5FAD2C97C501B4010E946A70181607
:109A700004F5A50194012C966CAD7DAD8EAD9FAD26
:109A80002C970E946E6EB62EA72E982E892EB501A9
:109A9000C401272F362F492F582F662D772D802F61
:109AA000912F0E94676E87FD04C06B2C7A2C092DC4
:109AB000182D20910F0E3091100E4091110E5091E3
:109AC000120EA3966CAD7DAD8EAD9FADA3970E9497
:109AD0008D6D4B015C01E894B7F8A7019601C501B3
:109AE000B4010E946A701816E4F4A5019401C7013C
:109AF000B6010E946E6EF62EE72ED82EC92EB70143
:109B0000C601272F362F492F582F662D772D802FEE
:109B1000912F0E94676E87FD04C06F2C7E2C0D2D47
:109B20001C2D262D372D402F512FBCA5A9A9FDA9ED
:109B3000EFA96B2F7A2F8F2F9E2F0E943C715B0114
:109B40008C01762F272F3B2D402F512FBBA92D960F
:109B5000AFAD2D976696FFAD66976896EFAD6897A7
:109B60006B2F7A2F8F2F9E2F0E94676E87FF0FC05B
:109B7000ABA82D96BFAC2D9766960FAD66976896ED
:109B80001FAD689704C0ABA0BFA00DA51BA58A2D73
:109B90009B2DA02FB12FF10182A793A7A4A7B5A752
:109BA000A9966CAD7DAD8EAD9FADA99790589B01E8
:109BB000AC010E948E6D65962CAD3DAD4EAD5FAD96
:109BC00065970E943C719B01AC016BE077ED83E2ED
:109BD0009BE30E948D6D0E94A9717B01D82EC92E36
:109BE000762FC601272F3F2D492F582F6A2D7B2D09
:109BF000802F912F0E94676E87FD03C057010D2DA6
:109C00001C2D8A2D9B2DA02FB12FF10186A397A388
:109C1000A0A7B1A7C6012E2D3F2D492F5C2DBCA5B5
:109C2000A9A9FDA9EFA96B2F7A2F8F2F9E2F0E9434
:109C3000676E18162CF081E0D101D7968C9302C084
:109C4000F10117AA81E0D101D6968C9380E1FE0143
:109C50003196A3E0BEE001900D928A95E1F75CA5F4
:109C600049A93DA92FA9852F942FA32FB22F809307
:109C7000130E9093140EA093150EB093160E252F6D
:109C8000342F4A2F5B2FBBA1AFA1FDA5EBA56B2FF6
:109C90007A2F8F2F9E2F0E946E6E6B017C017CA508
:109CA00069A99DA98FA9272F362F492F582F6A2DD3
:109CB0007B2D802F912F0E946E6EAB01BC0197010E
:109CC0008601C1010E94CD3E6196BFAD6197B09300
:109CD000C1082CAD3DAD4EAD5FAD2093930D3093DB
:109CE000940D4093950D5093960D24964CAD5DAD1B
:109CF0006EAD7FAD24974093970D5093980D609370
:109D0000990D70939A0D28966CAD7DAD8EAD9FAD7B
:109D1000289760939B0D70939C0D80939D0D90935D
:109D20009E0D88AD99ADAAADBBAD80939F0D90936C
:109D3000A00DA093A10DB093A20D0E94B142C859ED
:109D4000DF4F0FB6F894DEBF0FBECDBFDF91CF91CE
:109D50001F910F91FF90EF90DF90CF90BF90AF9049
:109D60009F908F907F906F905F904F903F902F903B
:109D70000C94365028AD39AD4AAD5BAD20939F0DA4
:109D80003093A00D4093A10D5093A20DEAE9F6E0A7
:109D90000C945345C859DF4F0FB6F894DEBF0FBE81
:109DA000CDBFDF91CF911F910F91FF90EF90DF908A
:109DB000CF90BF90AF909F908F907F906F905F906B
:109DC0004F903F902F900895EF92FF920F931F9323
:109DD000CF93DF937B018A01E9012091DF0D309160
:109DE000E00D4091E10D5091E20DFC016081718127
:109DF000828193810E943C710E940C71E3E9FDE035
:109E000060837183828393832091E30D3091E40D0D
:109E10004091E50D5091E60DF701608171818281DD
:109E200093810E943C710E940C71E7E9FDE0608320
:109E30007183828393832091E70D3091E80D4091E7
:109E4000E90D5091EA0DF801608171818281938161
:109E50000E943C710E940C71EBE9FDE0608371830C
:109E6000828393832091EB0D3091EC0D4091ED0DA9
:109E70005091EE0D688179818A819B810E943C71AD
:109E80000E940C71EFE9FDE060837183828393830C
:109E90009F014BE95DE067E97DE083E99DE00E9479
:109EA0008C561092130E1092140E1092150E1092E2
:109EB000160E1092030E1092040E1092050E1092C0
:109EC000060E1092070E1092080E1092090E1092B4
:109ED0000A0E10920B0E10920C0E10920D0E109294
:109EE0000E0E10920F0E1092100E1092110E109274
:109EF000120EDF91CF911F910F91FF90EF90089577
:109F00002091EB0D3091EC0D4091ED0D5091EE0D47
:109F1000FC0160817181828193810E943C710E9469
:109F20000C71EFE9FDE06083718382839383CF013D
:109F30000C94C8568093BF08089580912D0E81110E
:109F400088C080912C0E811184C080912B0E8111CC
:109F500080C008959091C00095FFFCCF8093C6000B
:109F6000319684918111F6CFEEEDF6E007C0909125
:109F7000C00095FFFCCF8093C6003196849181117B
:109F8000F6CF80912D0E8823D1F060912E0E709126
:109F90002F0E8091300E9091310E0E94096F20910A
:109FA000DF0D3091E00D4091E10D5091E20D0E94E6
:109FB0006E6EAB01BC018DEE96E00E94540C809158
:109FC0002C0E8823D1F06091320E7091330E809167
:109FD000340E9091350E0E94096F2091E30D30915F
:109FE000E40D4091E50D5091E60D0E946E6EAB01BF
:109FF000BC0181EF96E00E94540C80912B0E8823C7
:10A00000D1F06091360E7091370E8091380E90919C
:10A01000390E0E94096F2091E70D3091E80D4091B3
:10A02000E90D5091EA0D0E946E6EAB01BC0185EF07
:10A0300096E00E94540C8091C00085FFFCCF8AE01E
:10A040008093C60010922D0E10922C0E10922B0EA3
:10A050000895E8EDF6E085CF10922D0E10922C0EAB
:10A0600010922B0E089580933F010895EFE6F0E0E3
:10A0700080818260808308951F920F920FB60F92A5
:10A0800011240F931F932F933F934F935F936F93DD
:10A090007F938F939F93AF93BF93EF93FF938091A1
:10A0A0003E0E90913F0E892B09F056C19091C10848
:10A0B0008091C008981771F0E091C0088DE4E89F86
:10A0C000F0011124EE53F74FDF01A45BBF4F81E095
:10A0D0008C9302C0E0E0F0E0F0933F0EE0933E0E80
:10A0E000309709F433C1DF01A45BBF4F81E08C934B
:10A0F0001092400E1092410E1092420E1092430E9A
:10A1000060AD71AD613187E2780710F060E177E210
:10A1100081E08093440E6832710510F468E270E0CB
:10A1200068527109611588E07807D0F0872F992768
:10A13000880F991F880F991F8750994FFC013296FD
:10A1400045915491AA27659F9001649F210D3A1F64
:10A1500006942A1F3A1F1124FC01859194911DC079
:10A160009B01369527952C7F2750354FF901859116
:10A1700094912E5F3F4FF90145915491FB01E77097
:10A18000FF274E9F90014F9F300D5E9F300D112491
:10A19000A3E036952795AA95E1F7821B930B8436A9
:10A1A0009105A0F4E4EAF2E006C09091C00095FFAA
:10A1B000FCCF8093C60081918111F7CF4AE050E037
:10A1C0008DE296E00E94942C84E690E09093460EF7
:10A1D0008093450EE0913E0EF0913F0E94AD85AD1B
:10A1E0009093470E8093480E692F782F613187E254
:10A1F000780710F060E177E281E08093440E6832E6
:10A20000710510F468E270E068527109611588E028
:10A210007807E0F0872F9927880F991F880F991FDB
:10A220008750994FFC01329625913491AA27639F5C
:10A23000A001629F410D5A1F06944A1F5A1F112404
:10A24000FC0125913491241B350B1EC0CB01969542
:10A2500087958C7F8750954FFC012591349102960C
:10A26000FC0145915491FB01E770FF274E9FC0010F
:10A270004F9F900D5E9F900D112443E0969587951A
:10A280004A95E1F7281B390B24363105A0F4E4EA9E
:10A29000F2E006C09091C00095FFFCCF8093C6000D
:10A2A00081918111F7CF4AE050E08DE296E00E9463
:10A2B000942C24E630E0C901A0E0B0E08093490E80
:10A2C00090934A0EA0934B0EB0934C0E309389009E
:10A2D00020938800E0913E0EF0913F0E8089918995
:10A2E000A289B389B695A79597958795B095A095BE
:10A2F000909581959F4FAF4FBF4F80934D0E909398
:10A300004E0EA0934F0EB093500E8093510E90932B
:10A31000520EA093530EB093540E8093550E90930B
:10A32000560EA093570EB093580E8093590E9093EB
:10A330005A0EA0935B0EB0935C0E10923A0E1092E0
:10A340003B0E10923C0E10923D0E06C080ED97E041
:10A350009093890080938800E0913E0EF0913F0E2B
:10A36000309709F46EC480A180935D0E80FF3BC0DE
:10A3700016988FEF80933B0180913F018823B9F1BC
:10A3800023B1217031E0232759F180915E0E88239B
:10A3900039F180819181A281B381181619061A06BC
:10A3A0001B06F4F480911B0E90911C0EA0911D0EC3
:10A3B000B0911E0E80932E0E90932F0EA093300E10
:10A3C000B093310E30932D0E80899189A289B38983
:10A3D00080933A0E90933B0EA0933C0EB0933D0EAB
:10A3E00020935E0E04C0169A81E080933B01809119
:10A3F0005D0E81FF40C0149A8FEF80933C018091E5
:10A400003F018823E1F123B131E026952170232714
:10A4100079F180915F0E882359F1E0913E0EF09121
:10A420003F0E84819581A681B781181619061A06F8
:10A430001B06F4F480911F0E9091200EA091210E26
:10A44000B091220E8093320E9093330EA093340E6F
:10A45000B093350E30932C0E80899189A289B389EF
:10A4600080933A0E90933B0EA0933C0EB0933D0E1A
:10A4700020935F0E04C0149881E080933C0180918A
:10A480005D0E82FF41C046988FEF80933D01809121
:10A490003F018823E9F123B131E022FB222720F993
:10A4A000232779F18091600E882359F1E0913E0EC7
:10A4B000F0913F0E80859185A285B3851816190607
:10A4C0001A061B06F4F48091230E9091240EA0919D
:10A4D000250EB091260E8093360E9093370EA093E2
:10A4E000380EB093390E30932B0E80899189A28952
:10A4F000B38980933A0E90933B0EA0933C0EB09399
:10A500003D0E2093600E04C0469A81E080933D0189
:10A5100080915D0E83FF03C045988FEF02C0459A7E
:10A5200081E080933E0120E030E0BDC18091C00019
:10A5300087FF19C0E091C6004091AE065091AF066A
:10A54000CA0101968F7799276091B0067091B10684
:10A550008617970741F0DA01A25DB94FEC9390930B
:10A56000AF068093AE06E0913E0EF0913F0E8091D3
:10A570004D0E90914E0EA0914F0EB091500E408115
:10A58000518162817381840F951FA61FB71F80932D
:10A590004D0E90934E0EA0934F0EB093500E181682
:10A5A00019061A061B060CF4159A8091510E90910B
:10A5B000520EA091530EB091540E44815581668184
:10A5C0007781840F951FA61FB71F8093510E90931C
:10A5D000520EA093530EB093540E181619061A0675
:10A5E0001B060CF4139AE0913E0EF0913F0E809101
:10A5F000550E9091560EA091570EB091580E408571
:10A60000518562857385840F951FA61FB71F8093A0
:10A61000550E9093560EA093570EB093580E1816E1
:10A6200019061A061B060CF4479A8091590E909150
:10A630005A0EA0915B0EB0915C0E448555856685DF
:10A640007785840F951FA61FB71F8093590E90938F
:10A650005A0EA0935B0EB0935C0E181619061A06DC
:10A660001B060CF4179A80914D0E90914E0EA091FE
:10A670004F0EB091500E181619061A061B065CF5FF
:10A68000E0913E0EF0913F0E4089518962897389B5
:10A69000841B950BA60BB70B80934D0E90934E0E1B
:10A6A000A0934F0EB093500E40913B0180911B0E32
:10A6B00090911C0EA0911D0EB0911E0E840F911D45
:10A6C000A11DB11D80931B0E90931C0EA0931D0E17
:10A6D000B0931E0E15988091510E9091520EA0913C
:10A6E000530EB091540E181619061A061B065CF587
:10A6F000E0913E0EF0913F0E408951896289738945
:10A70000841B950BA60BB70B8093510E9093520EA2
:10A71000A093530EB093540E40913C0180911F0EB4
:10A720009091200EA091210EB091220E840F911DC8
:10A73000A11DB11D80931F0E9093200EA093210E9A
:10A74000B093220E13988091550E9091560EA091C1
:10A75000570EB091580E181619061A061B065CF50E
:10A76000E0913E0EF0913F0E4089518962897389D4
:10A77000841B950BA60BB70B8093550E9093560E2A
:10A78000A093570EB093580E40913D018091230E37
:10A790009091240EA091250EB091260E840F911D4C
:10A7A000A11DB11D8093230E9093240EA093250E1E
:10A7B000B093260E47988091590E90915A0EA09111
:10A7C0005B0EB0915C0E181619061A061B065CF596
:10A7D000E0913E0EF0913F0E408951896289738964
:10A7E000841B950BA60BB70B8093590E90935A0EB2
:10A7F000A0935B0EB0935C0E40913E018091270EBA
:10A800009091280EA091290EB0912A0E840F911DCF
:10A81000A11DB11D8093270E9093280EA093290EA1
:10A82000B0932A0E179880913A0E90913B0EA0910A
:10A830003C0EB0913D0E0196A11DB11D80933A0EC4
:10A8400090933B0EA0933C0EB0933D0E40913A0E78
:10A8500050913B0E60913C0E70913D0E2F5F3F4F2B
:10A86000E0913E0EF0913F0E80899189A289B389D3
:10A87000481759076A077B07B0F040913A0E50918C
:10A880003B0E60913C0E70913D0EE0913E0EF091BA
:10A890003F0E84899589A689B78984179507A607ED
:10A8A000B70748F4CBC08091440E90E028173907D1
:10A8B0000CF43CCEE2CF4091490E50914A0E60918B
:10A8C0004B0E70914C0E048D158D268D378DAA2759
:10A8D000419FB12D529FC001629F900D619F800DDD
:10A8E000911D429FB00D811D9A1F519FB00D811D7A
:10A8F0009A1F609FB00D811D9A1F509FB10D8A1F36
:10A900009A1FB6958A1F9A1F112444AD55AD480F62
:10A91000591F5093480E4093470E80AD91ADA2ADA4
:10A92000B3AD60E070E084179507A607B70720F481
:10A930009093480E8093470E6091470E7091480E99
:10A94000613187E2780710F060E177E281E080937F
:10A95000440E6832710510F468E270E068527109C3
:10A96000611588E07807E0F0872F9927880F991FF5
:10A97000880F991F8750994FFC0132962591349189
:10A98000AA27639FA001629F410D5A1F06944A1F88
:10A990005A1F1124FC0125913491241B350B1EC034
:10A9A000CB01969587958C7F8750954FFC0125911B
:10A9B00034910296FC0145915491FB01E770FF2709
:10A9C0004E9FC0014F9F900D5E9F900D1124A3E0FC
:10A9D00096958795AA95E1F7281B390B2436310502
:10A9E000A0F4E4EAF2E006C09091C00095FFFCCF2D
:10A9F0008093C60081918111F7CF4AE050E08DE24B
:10AA000096E00E94942C24E630E030938900209355
:10AA100088008091490E90914A0EA0914B0EB09102
:10AA20004C0E820F931FA11DB11D8093490E909370
:10AA30004A0EA0934B0EB0934C0EDEC040913A0EDE
:10AA400050913B0E60913C0E70913D0E808D918D2A
:10AA5000A28DB38D84179507A607B70708F0C4C069
:10AA60004091400E5091410E6091420E7091430E04
:10AA7000048D158D268D378DAA27419FB12D529FAC
:10AA8000C001629F900D619F800D911D429FB00D8E
:10AA9000811D9A1F519FB00D811D9A1F609FB00D9F
:10AAA000811D9A1F509FB10D8A1F9A1FB6958A1F4C
:10AAB0009A1F11242091470E3091480EE05CFF4F01
:10AAC0002817390718F42081318102C0281B390B5F
:10AAD00080819181A281B381A90160E070E0481773
:10AAE00059076A077B0708F49C01B901213187E205
:10AAF000380710F060E177E281E08093440E68321D
:10AB0000710510F468E270E068527109611588E01F
:10AB10007807E0F0872F9927880F991F880F991FD2
:10AB20008750994FFC01329625913491AA27639F53
:10AB3000A001629F410D5A1F06944A1F5A1F1124FB
:10AB4000FC0125913491241B350B1EC0CB01969539
:10AB500087958C7F8750954FFC0125913491029603
:10AB6000FC0145915491FB01E770FF274E9FC00106
:10AB70004F9F900D5E9F900D112443E09695879511
:10AB80004A95E1F7281B390B24363105A0F4E4EA95
:10AB9000F2E006C09091C00095FFFCCF8093C60004
:10ABA00081918111F7CF4AE050E08DE296E00E945A
:10ABB000942C24E630E03093890020938800809123
:10ABC000400E9091410EA091420EB091430E820F23
:10ABD000931FA11DB11D8093400E9093410EA09331
:10ABE000420EB093430E08C08091450E9091460EE0
:10ABF000909389008093880040913A0E50913B0ECB
:10AC000060913C0E70913D0EE0913E0EF0913F0E32
:10AC100080899189A289B389481759076A077B07F8
:10AC200080F010923F0E10923E0E9091C1088091DC
:10AC3000C008981731F08091C0088F5F8F708093A3
:10AC4000C008FF91EF91BF91AF919F918F917F913C
:10AC50006F915F914F913F912F911F910F910F90A5
:10AC60000FBE0F901F9018950E9A0C9A3E9A3D9A1F
:10AC70003B9A559A529A529A529A529A529A529A88
:10AC80002098289A2198299A22982A9A0D9A1598FC
:10AC90000B9A13983F9A47980F9A17983C9A4498A2
:10ACA0003B9A4398A1E8B0E08C918F7E8C938C9175
:10ACB00088608C93E0E8F0E080818D7F80838081E4
:10ACC0008E7F808380818F73808380818F7C80835F
:10ACD0008C91887F82608C9380E090E490938900CF
:10ACE000809388001092850010928400EFE6F0E0D7
:10ACF00080818260808381E080933F017894089511
:10AD00009091C1088091C008981729F00E94D358EB
:10AD10000E94B018F5CF0895CF93DF93EFB7F89462
:10AD2000EC0188819981AA81BB8180931B0E90934D
:10AD30001C0EA0931D0EB0931E0EEB01888199810D
:10AD4000AA81BB8180931F0E9093200EA093210EA9
:10AD5000B093220EEA0188819981AA81BB818093F8
:10AD6000230E9093240EA093250EB093260EE90196
:10AD700088819981AA81BB818093270E9093280EA8
:10AD8000A093290EB0932A0EEFBFDF91CF910895C3
:10AD90002FB7F894FC0180819181A281B3818093C7
:10ADA000270E9093280EA093290EB0932A0E2FBF42
:10ADB00008950F931F939FB7F89424E0829FF001AA
:10ADC0001124E55EF14F00811181228133819FBF03
:10ADD000B801C9011F910F9108950E9480565A9899
:10ADE0005A985A985A98089580916F008D7F809351
:10ADF0006F0006C08091C0088F5F8F708093C0087D
:10AE00009091C1088091C00898130AC010923F0E1B
:10AE100010923E0E80916F00826080936F000895C3
:10AE20009091C1088091C008981751F3E3CF209109
:10AE300048013091490140914A0150914B0160E035
:10AE400070E08FE793E40E946E6E6093700E7093D3
:10AE5000710E8093720E9093730E089597FF03C046
:10AE600080916E0E04C0FC01E159F14F808190E0A9
:10AE700008950F931F93CF93DF93EC01662309F49A
:10AE800061C0E6EEFFE007C09091C00095FFFCCFE7
:10AE90008093C600319684918111F6CF4AE050E04C
:10AEA00070E08DE296E00E94762CEDEEFFE007C0A8
:10AEB0009091C00095FFFCCF8093C600319684919D
:10AEC0008111F6CF8091C00085FFFCCF8AE080938E
:10AED000C6000E94871836C0C901880F991F880FC5
:10AEE000991FFC01E55FFF4E659174916C177D071A
:10AEF0003CF521503109220F331F220F331FF90176
:10AF0000E75FFF4E05911491255F3F4EF901459192
:10AF10005491FC01E75FFF4E25913491C41BD50B82
:10AF2000201B310BC29FC001C39F900DD29F900D7B
:10AF30001124641B750B0E942572600F711F13C0D2
:10AF40004F5F01C041E0242F30E0403209F0C4CF10
:10AF50002032310531F4E5E8F0E185919491BC01AE
:10AF600002C060E070E020EF3FE3261B370BC90111
:10AF7000DF91CF911F910F910895CF93DF9321E03F
:10AF800030E0A901440F551F440F551FFA01E55F3A
:10AF9000FF4E659174916817790744F52150310986
:10AFA000220F331F220F331FF901E75FFF4EC591B8
:10AFB000D491255F3F4EF901A591B491FA01E75F65
:10AFC000FF4E25913491AC014A1B5B0B2C1B3D0BB2
:10AFD000429FC001439F900D529F900D11246A1B08
:10AFE0007B0B0E9425726C0F7D1F0BC02F5F3F4FA4
:10AFF0002032310509F0C5CFE5E8F0E18591949163
:10B00000BC0120EF3FE3261B370BC901DF91CF9135
:10B0100008954F925F926F927F928F929F92AF921C
:10B02000BF92CF92DF92EF92FF920F931F93CF9335
:10B03000DF93EC01662351F1E6EEFFE007C090914B
:10B04000C00095FFFCCF8093C6003196849181119A
:10B05000F6CF4AE050E070E08DE296E00E94762C58
:10B06000E9E8F0E107C09091C00095FFFCCF809324
:10B07000C600319684918111F6CF8091C00085FF82
:10B08000FCCF8AE08093C6000E94871810EF612EE3
:10B090001FE3712E6C1A7D0A41E05EC09C01220FF5
:10B0A000331F220F331FF901E75FFF4E0591149103
:10B0B000601671060CF04FC00197880F991F880F1A
:10B0C000991FFC01E55FFF4EA590B490875F9F4EEE
:10B0D000FC01C591D491F901E55FFF4E85909490F4
:10B0E000B501882777FD8095982F0E94096F6B0125
:10B0F0007C01B3016C1B7D0B882777FD8095982F11
:10B100000E94096F2B013C01B4016A197B09882751
:10B1100077FD8095982F0E94096F9B01AC01C301B8
:10B12000B2010E943C714B015C01B8016C1B7D0BAC
:10B13000882777FD8095982F0E94096F9B01AC01AD
:10B14000C501B4010E946E6E9B01AC01C701B6013E
:10B150000E948E6D17C04F5F842F90E0403209F03F
:10B160009DCF809759F4E7E8F0E1659174918827C5
:10B1700077FD8095982F0E94096F04C060E070E011
:10B1800080E090E0DF91CF911F910F91FF90EF90C1
:10B19000DF90CF90BF90AF909F908F907F906F90F7
:10B1A0005F904F9008952F923F924F925F926F92CF
:10B1B0007F928F929F92AF92BF92CF92DF92EF9247
:10B1C000FF920F931F93CF93DF9300D0CDB7DEB7DD
:10B1D0008091610E882309F4C5C18FB7F89410924D
:10B1E000610E8FBF60E08091680E9091690E0E94A1
:10B1F00009586B017C019B01AC016091620E70915A
:10B20000630E8091640E9091650E0E948D6DB62E36
:10B21000A72E182F092FA5019801852F942FA32F52
:10B22000B22F8093740E9093750EA093760EB09308
:10B23000770E20E030E040E251E4D501F8016B2FB9
:10B240007A2F8F2F9E2F0E946A7018160CF41DC142
:10B2500020E030E040E251ECD501F8016B2F7A2F6D
:10B260008F2F9E2F0E94676E87FD0BC18091780EF5
:10B270008111FCC020914C0130914D0140914E0153
:10B2800050914F01D501F8016B2F7A2D8F2F902F00
:10B290000E943C71762E672E89839A83A301382FF2
:10B2A000292F852F942FA32FB22F80937D0E90935B
:10B2B0007E0EA0937F0EB093800E2091790E309178
:10B2C0007A0E40917B0E50917C0ED501F8016B2FC8
:10B2D0007A2D8F2F902F0E948E6D8B012C018090E4
:10B2E000810E9090820EA090830EB090840E282D37
:10B2F000392D4A2D5B2D602F712F842D952D0E94A5
:10B30000676E87FF9DC084012501802F912FA42D9A
:10B31000B52D8093790E90937A0EA0937B0EB09307
:10B320007C0E209148013091490140914A01509191
:10B330004B01602F712F842D952D0E943C714B0184
:10B340005C01862F992DAA2DBB2D8093850E90939D
:10B35000860EA093870EB093880E2091890E3091AF
:10B360008A0E40918B0E50918C0EC701B6010E943F
:10B370008D6D2091440130914501409146015091DD
:10B3800047010E943C7120ED3CEC4CE45DE30E94DF
:10B390003C711B012C0123E333E343E75FE360913E
:10B3A0008D0E70918E0E80918F0E9091900E0E9456
:10B3B0003C719B01AC01C201B1010E948E6D8B01F9
:10B3C0002C01862F912FA42DB52D80938D0E909357
:10B3D0008E0EA0938F0EB093900EC092890ED092D5
:10B3E0008A0EE0928B0EF0928C0E282D392D4A2D6C
:10B3F0005B2DD301F980EA806B2F762D8F2D9E2D4A
:10B400000E948E6D202F312F442D552D0E948D6D61
:10B410008B017C0120E030E0A901712F9F2D0E945B
:10B42000676E87FD3CC020E030E04FE753E4602FBB
:10B43000712F8E2D9F2D0E946A701816A4F528C0BA
:10B440008090700E9090710EA090720EB090730E5E
:10B45000282D392D4A2D5B2D602F712F842D952D90
:10B460000E946A7018160CF050CF4DCF1092790ED2
:10B4700010927A0E10927B0E10927C0E1092780E23
:10B48000F9CE81E08093780E0AC081E08093780E37
:10B4900000E010E08FE7E82E93E4F92E04C000E00E
:10B4A00010E0E12CF12C2091680E3091690E409152
:10B4B000910E5091920E421753071CF010926F0E8E
:10B4C00011C0409150015091510124173507B4F734
:10B4D000602F712F8E2D9F2D0E94D66E75956795CA
:10B4E00060936F0E0E94C2290091930E1091940EEA
:10B4F0002091950E3091960E601B710B820B930B71
:10B50000683873418105910568F10E94C2296093F2
:10B51000930E7093940E8093950E9093960E809157
:10B52000660E9091670E2091970E3091980E281715
:10B530003907ACF4209152013091530182179307DF
:10B5400074F420916A0E30916B0E821793071CF0F1
:10B5500010926E0E07C08FE780936E0E03C010929C
:10B560006E0E2C980F900F90DF91CF911F910F913D
:10B57000FF90EF90DF90CF90BF90AF909F908F9013
:10B580007F906F905F904F903F902F9008954F92D3
:10B590005F926F927F928F929F92AF92BF92CF9263
:10B5A000DF92EF92FF920F931F93CF93DF9360EFA1
:10B5B000662E6FE3762E681A790A81E090E09C018E
:10B5C000220F331F220F331FF901E75FFF4E059152
:10B5D0001491601671060CF04FC00197880F991FE7
:10B5E000880F991FFC01E55FFF4EA590B490875F1F
:10B5F0009F4EFC01C591D491F901E55FFF4E859006
:10B600009490B501882777FD8095982F0E94096F47
:10B610006B017C01B3016C1B7D0B882777FD809546
:10B62000982F0E94096F2B013C01B4016A197B0914
:10B63000882777FD8095982F0E94096F9B01AC01A8
:10B64000C301B2010E943C714B015C01B8016C1B4B
:10B650007D0B882777FD8095982F0E94096F9B01AD
:10B66000AC01C501B4010E946E6E9B01AC01C70123
:10B67000B6010E948E6D0FC001968032910509F0CF
:10B680009ECFE7E8F0E165917491882777FD80957A
:10B69000982F0E94096FDF91CF911F910F91FF901A
:10B6A000EF90DF90CF90BF90AF909F908F907F9062
:10B6B0006F905F904F9008951092810E1092820EBD
:10B6C0001092830E1092840E20914801309149010E
:10B6D00040914A0150914B0160E070E08FE793E4A4
:10B6E0000E946E6E6093700E7093710E8093720E56
:10B6F0009093730E239A549A249A569A87ED8093C6
:10B700007A00EEE7F0E010828081816080838081A2
:10B710008260808380818460808380818460808374
:10B7200080E888BDEEE6F0E08081846080836AEF87
:10B7300070E080E090E00E94F52960E085E090E014
:10B740000E9439579093920E8093910E60E083E1AE
:10B7500091E00E943957909351018093500185E008
:10B7600090E00E94BD579093980E8093970E86E9C3
:10B7700090E00E94BD579093530180935201089529
:10B78000089560E080E090E00E9439571092620EC8
:10B790001092630E1092640E1092650E80E090E09D
:10B7A0000E94BD5790936B0E80936A0E10926D0E9F
:10B7B00010926C0E10926F0E2B9810926F0E1092CA
:10B7C0006E0E1092700E5C981092710E1092700EA8
:10B7D0001092710E10926B0E10926A0E10926E0EF5
:10B7E0002C9808952F923F924F925F926F927F9282
:10B7F0008F929F92AF92BF92CF92DF92EF92FF9281
:10B800000F931F93CF93DF93CDB7DEB7E5970FB6B6
:10B81000F894DEBF0FBECDBF688B798B8A8B9B8B74
:10B820001A0139A728A70E94C2296C8B7D8B8E8BA9
:10B830009F8B22E0221631041CF4E8EBF2E017C0E3
:10B84000EBECF2E006C09091C00095FFFCCF809336
:10B85000C60081918111F7CF8091C00085FFFCCF98
:10B860002CC49091C00095FFFCCF8093C6008191BD
:10B870008111F7CF8091C00085FFFCCF8AE08093D3
:10B88000C6000E94C15B37FE04C08FE780936E0E36
:10B8900005C0F101E159F14F8FE780838C889D88C5
:10B8A000AE88BF888C869D86AE86BF868886998640
:10B8B000AA86BB863FE7C32ED12CE12CF12C4FE7A3
:10B8C000842E912CA12CB12C89AA9AAAABAABCAA2D
:10B8D00021E028A31F821E82A1014159514F5D8F93
:10B8E0004C8FE9EFFEE084908CA6E1E0FFE09490BD
:10B8F0009DA6E6E0FFE0A490AEA6EDE0FFE0B490E8
:10B90000BFA6E4E1FFE0849088AA5101AA0CBB1C09
:10B9100095012859314F3F8F2E8F8091610E8823DA
:10B9200009F4EEC28FB7F8941092610E8FBF37FE04
:10B9300007C08091660E9091670E0E94C75A07C09B
:10B94000622DAE8DBF8D8D919C910E9409586983A7
:10B950007A838B839C8379816A819B818C81272F59
:10B96000362F492F582FB88DA98DBA8CAB8C6B2FE1
:10B970007A2F8B2D9A2D0E946A70181644F08980B8
:10B98000888E9A80998EAB80AA8EBC80BB8E79817E
:10B990006A819B818C81272F362F492F582FBAA57A
:10B9A000AD816B2F7A2F802F912F0E94676E87FDBC
:10B9B00006C089808AA69A809D820B811C81A8A0DE
:10B9C000AA2009F47EC3788969899A898B89272FEF
:10B9D000362F492F582FB981AA81BB80AC806B2F9D
:10B9E0007A2F8B2D9A2D0E946A7018160CF088C23F
:10B9F0000E94C2298C849D84AE84BF846819790911
:10BA00008A099B09693873418105910508F478C258
:10BA100089A99AA9ABA9BCA98C199D09AE09BF092E
:10BA2000B595A7959795879537FE03C080936E0EC1
:10BA300003C0EC8DFD8D80830E94C22968877987C1
:10BA40008A879B874B015C012C853D854E855F85F0
:10BA5000821A930AA40AB50A8CA29DA2AEA2BFA222
:10BA60008888888E9988998EAA88AA8EBB88BB8E72
:10BA700028C30E94C22988849984AA84BB84681937
:10BA800079098A099B09693873418105910508F490
:10BA900036C20E94C2296C877D878E879F878E80E1
:10BAA0009F80892809F408C2DC01CB01888499842D
:10BAB000AA84BB8488199909AA09BB094CA05DA076
:10BAC0006EA07FA0480E591E6A1E7B1E8CA09DA0F2
:10BAD000AEA0BFA0881A990AAA0ABB0AC501B40180
:10BAE000A70196010E941572A30192010E945B7248
:10BAF00089A89AA8ABA8BCA8280D391D4A1D5B1DB2
:10BB000024313105410551052CF129AB3AAB4BAB42
:10BB10005CAB2C3E3105410551054CF0BBEE8B2E44
:10BB2000912CA12CB12C89AA9AAAABAABCAA29A9AA
:10BB30003AA94BA95CA92038310541055105CCF043
:10BB4000AEEFCA2ED12CE12CF12CC21AD30AE40A92
:10BB5000F50A13C0E4E18E2E912CA12CB12C89AAF8
:10BB60009AAAABAABCAAF4E1CF2ED12CE12CF12CDD
:10BB700004C0C9A8DAA8EBA8FCA88CA5E9EFFEE0F0
:10BB800008C09091C00095FFFCCF8093C60031960D
:10BB900084918111F6CF2AE030E049A95AA96BA916
:10BBA0007CA98DE296E00E94652C8DA5E1E0FFE086
:10BBB00008C09091C00095FFFCCF8093C6003196DD
:10BBC00084918111F6CF2AE030E0B701A6018DE221
:10BBD00096E00E94652C8EA5E6E0FFE008C09091FB
:10BBE000C00095FFFCCF8093C600319684918111EF
:10BBF000F6CF22E030E0FAA5ED814F2F5E2F602FC7
:10BC0000712F8DE296E00E946E2D8FA5EDE0FFE092
:10BC100008C09091C00095FFFCCF8093C60031967C
:10BC200084918111F6CF22E030E0F88DE98D9A8D74
:10BC30008B8D4F2F5E2F692F782F8DE296E00E941B
:10BC40006E2D8091C00085FFFCCF8AE08093C600F6
:10BC50002E813F81233031050CF42EC1C701B6017E
:10BC60000E94096F20E030E040E850E40E943C71FF
:10BC70004B015C017AA56D81272F362F402F512F64
:10BC8000B88DA98DEA8D1B8D6B2F7A2F8E2F912F5A
:10BC90000E948D6D20ED3FE049E450E40E943C712C
:10BCA00020E030E040E05FE30E943C719B01AC018A
:10BCB000C501B4010E946E6EB62EA72E182F092F53
:10BCC000C301B2010E94096F20E030E04AE754E46A
:10BCD0000E946E6E762E672E582E492E88A9E4E1BA
:10BCE000FFE008C09091C00095FFFCCF8093C60094
:10BCF000319684918111F6CF22E030E0F501C80140
:10BD00004F2F5A2D692F702F8DE296E00E946E2DD5
:10BD1000EAE1FFE007C09091C00095FFFCCF80935F
:10BD2000C600319684918111F6CF22E030E0F30114
:10BD3000C2014F2F562D692F742D8DE296E00E947F
:10BD40006E2D8091C00085FFFCCF8AE08093C600F5
:10BD50002AE939E949E15FE3D501F8016B2F7A2D32
:10BD60008F2F902F0E943C716DABB72E182F092F8B
:10BD7000762FC801272F3B2D492F582FF801672F09
:10BD80007B2D8F2F9E2F0E948E6DD301F2012B2FC2
:10BD9000362D4F2F542D0E946E6EA62E972E882E74
:10BDA0009BA7B301C201272F362D492F542DBDA9C2
:10BDB000F8016B2F7B2D8F2F9E2F0E943C7120E06E
:10BDC00030E040E05EE30E943C71762E672E582EF4
:10BDD000492EE0E2FFE007C09091C00095FFFCCF44
:10BDE0008093C600319684918111F6CF8091C00076
:10BDF00085FFFCCF8AE08093C600EDE2FFE007C03C
:10BE00009091C00095FFFCCF8093C600319684913D
:10BE10008111F6CF22E030E0FDA9C8014F2F5B2D44
:10BE2000692F702F8DE296E00E946E2D8091C000E8
:10BE300085FFFCCF8AE08093C600E3E3FFE007C004
:10BE40009091C00095FFFCCF8093C60031968491FD
:10BE50008111F6CF22E030E08BA54A2D592D682DB7
:10BE6000782F8DE296E00E946E2D8091C00085FFB4
:10BE7000FCCF8AE08093C600E9E3FFE007C0909121
:10BE8000C00095FFFCCF8093C6003196849181114C
:10BE9000F6CF22E030E0F301C2014F2F562D692F7B
:10BEA000742D8DE296E00E946E2D8091C00085FF7A
:10BEB000FCCF8AE08093C60089A99AA9ABA9BCA946
:10BEC0008C0D9D1DAE1DBF1DB595A79597958795AA
:10BED00037FE03C080936E0E03C0EC8DFD8D808312
:10BEE0002E813F812F5F3F4F3F832E8388888AA614
:10BEF00099889D820A891B8921E028A301C018A284
:10BF000020E030E040EA51E4B889A989BA88AB88DA
:10BF10006B2F7A2F8B2D9A2D0E948E6D9B01AC0179
:10BF2000B981AA81BB80AC806B2F7A2F8B2D9A2D83
:10BF30000E946A70181694F4EFE3FFE007C0909136
:10BF4000C00095FFFCCF8093C6003196849181118B
:10BF5000F6CF8091C00085FFFCCFAFC00E94C22900
:10BF60008C889D88AE88BF88681979098A099B09E1
:10BF7000613D77408105910508F452C037FE10C03D
:10BF800070906E0EE8E6FFE007C09091C00095FF4C
:10BF9000FCCF8093C600319684918111F6CF10C0FA
:10BFA000AC8DBD8D7C90EEE6FFE007C09091C000A7
:10BFB00095FFFCCF8093C600319684918111F6CF16
:10BFC00022E030E0F981EA819B818C814F2F5E2F46
:10BFD000692F782F8DE296E00E946E2DE4E7FFE056
:10BFE00007C09091C00095FFFCCF8093C6003196AA
:10BFF00084918111F6CF4AE050E0672D70E08DE228
:10C0000096E00E94762C8091C00085FFFCCF8AE0EC
:10C010008093C6000E94C2296C8B7D8B8E8B9F8B78
:10C020000E94C2292B013C010E94C2292C853D851A
:10C030004E855F8588849984AA84BB84280D391D28
:10C040004A1D5B1D421A530A640A750A460E571EA2
:10C05000681E791E21E842162FE4520622E162068C
:10C06000710490F0E8E7FFE007C09091C00095FFF1
:10C07000FCCF8093C600319684918111F6CF8091D8
:10C08000C00085FFFCCF19C08E809F80A8A4B9A4F2
:10C09000A814B9040CF041CCE5E9FFE007C0909189
:10C0A000C00095FFFCCF8093C6003196849181112A
:10C0B000F6CF8091C00085FFFCCF8AE08093C60058
:10C0C00015C0788969899A898B89272F362F492F3E
:10C0D000582FB981AA81BB80AC806B2F7A2F8B2D12
:10C0E0009A2D0E94676E87FDC4CC09CFE5960FB6E6
:10C0F000F894DEBF0FBECDBFDF91CF911F910F919E
:10C10000FF90EF90DF90CF90BF90AF909F908F9077
:10C110007F906F905F904F903F902F900895CF93B6
:10C12000DF931F92CDB7DEB789830E94C15B0E9467
:10C130004F19698181112FC0E6EEFFE007C08091A1
:10C14000C00085FFFCCF9093C60031969491911169
:10C15000F6CF4AE050E070E08DE296E00E94762C47
:10C160008091C00085FFFCCF8AE08093C600E6EA9C
:10C17000F0E107C09091C00095FFFCCF8093C6000E
:10C18000319684918111F6CF8091C00085FFFCCF5C
:10C190008AE08093C6000F90DF91CF910895CF93EE
:10C1A000DF931F92CDB7DEB789830E94C15B0E94E7
:10C1B0004F19698181112FC0E6EEFFE007C0809121
:10C1C000C00085FFFCCF9093C600319694919111E9
:10C1D000F6CF4AE050E070E08DE296E00E94762CC7
:10C1E0008091C00085FFFCCF8AE08093C600E3ED1C
:10C1F000F0E107C09091C00095FFFCCF8093C6008E
:10C20000319684918111F6CF8091C00085FFFCCFDB
:10C210008AE08093C6000F90DF91CF9108952C980B
:10C220000E944F19811121C0E6EEFFE007C09091F6
:10C23000C00095FFFCCF8093C60031968491811198
:10C24000F6CFE0E0F1E107C09091C00095FFFCCF90
:10C250008093C600319684918111F6CF8091C00001
:10C2600085FFFCCF8AE08093C60008951F920F924D
:10C270000FB60F9211242F933F934F935F936F93B9
:10C280007F938F939F93AF93BF93EF93FF9380918F
:10C29000540181110CC080916F0E8093990E811111
:10C2A0002B9A80916E0E80939A0E81112C9A909108
:10C2B000990E80915401891708F02B9890919A0E4D
:10C2C00080915401891708F02C988F5F8F778093A5
:10C2D000540180919B0E833009F445C020F48130D5
:10C2E000D1F0A8F50CC0853009F463C008F455C03E
:10C2F000863009F478C0873009F0A0C080C0109261
:10C300007B0080E480937C0080917A00806480933D
:10C310007A0081E019C020917800309179008091F5
:10C320009C0E90919D0EA0919E0EB0919F0E820F3B
:10C33000931FA11DB11D80939C0E90939D0EA09301
:10C340009E0EB0939F0E82E080939B0E77C010925A
:10C350007B0082E480937C0080917A0080648093EB
:10C360007A0083E0F1CF20917800309179008091BC
:10C37000A00E9091A10EA091A20EB091A30E820FDB
:10C38000931FA11DB11D8093A00E9093A10EA093A9
:10C39000A20EB093A30E84E0D7CF10927B0081E46D
:10C3A00080937C0080917A00806480937A0085E09D
:10C3B000CBCF20917800309179008091A40E90919C
:10C3C000A50EA091A60EB091A70E820F931FA11DDE
:10C3D000B11D8093A40E9093A50EA093A60EB093CA
:10C3E000A70E86E0B1CF10927B0082E480937C00A0
:10C3F00080917A00806480937A0087E0A5CF2091B5
:10C400007800309179008091A80E9091A90EA091AA
:10C41000AA0EB091AB0E820F931FA11DB11D809388
:10C42000A80E9093A90EA093AA0EB093AB0E1092F3
:10C430009B0E8091AC0E8F5F8093AC0E8091AC0E02
:10C44000803108F474C02FEF3FE380919C0E9091EF
:10C450009D0EA901481B590BCA015093690E4093C8
:10C46000680E4091A00E5091A10E241B350B309305
:10C47000670E2093660E21E02093610E1092AC0EA1
:10C4800010929C0E10929D0E10929E0E10929F0E76
:10C490001092A40E1092A50E1092A60E1092A70E46
:10C4A0001092A80E1092A90E1092AA0E1092AB0E26
:10C4B0001092A00E1092A10E1092A20E1092A30E36
:10C4C0002091500130915101821793074CF0109246
:10C4D0006D0E10926C0E80E00E948F600E94141905
:10C4E0002091680E3091690E8091910E9091920E7C
:10C4F000821793074CF010926D0E10926C0E80E034
:10C500000E94CF600E9414192091660E3091670E30
:10C5100080915201909153012817390744F01092ED
:10C520006B0E10926A0E0E940F610E941419FF9107
:10C53000EF91BF91AF919F918F917F916F915F919B
:10C540004F913F912F910F900FBE0F901F90189514
:10C55000CF93DF93FC0110AA13AA8EE992E097A76C
:10C5600086A7DF01A15BBF4F1C9213961C92DF01CF
:10C57000A35BBF4F8D939C93DF01A459BF4F1C92C7
:10C5800013961C92DF01A659BF4F8D939C93DF0138
:10C59000A757BF4F1C9213961C92DF01A957BF4F9C
:10C5A0008D939C93DF01AC55BF4F29E111962C93DD
:10C5B000119714961C92DF01A755BF4F57961C92F6
:10C5C000DF01A753BF4F1C9213961C92DF01A953A2
:10C5D000BF4F8D939C93DF01AC51BF4F1D921D92B5
:10C5E0001D921C921397DF01A451BF4F1D921D9203
:10C5F0001D921C921397118212821082EF01C85172
:10C60000DF4F188219821A821B82DF01A051BF4FAF
:10C6100081E08C9315A614A60E94C22968577C4E0F
:10C620008F4F9F4F688379838A839B83DF91CF915C
:10C630000895DB01FC0120E03EE24C91403229F0FC
:10C64000283009F431934C9141932F5F11962B3090
:10C65000A1F7108208952F923F924F925F926F92AE
:10C660007F928F929F92AF92BF92CF92DF92EF9282
:10C67000FF920F931F93CF93DF93CDB7DEB7C358CD
:10C68000D1090FB6F894DEBF0FBECDBF8C016B0190
:10C690007A01312C82E0E80EF11C2801E0E14E0E17
:10C6A000511C5801F1EFAF0EB11C480182EF880E0A
:10C6B000911C8EE3682E712C6C0E7D1EE2E06E0ED6
:10C6C000711CEAE3F1E1249006C19C85292F2871B1
:10C6D000203109F01BC1F5018081813009F416C1B8
:10C6E000823009F003C112C165EF72E0CE01855AB4
:10C6F0009F4F0E943E75B601CE01855A9F4F0E9402
:10C700003E75BE016B587F4FCE01855A9F4F0E94E8
:10C710003E7565EF72E0CE01855A9F4F0E943E75CF
:10C7200021961FAE219724961FAE24978EE992E0A2
:10C730009FAF8EAF21E0AE014B585F4FB701C301F1
:10C740000E94EF33811139C0F5018081811135C01C
:10C75000822DEAE3F1E108C09091C00095FFFCCF83
:10C760008093C600319684918111F6CFE7EFF2E015
:10C7700006C09091C00095FFFCCF8093C6008191C8
:10C780008111F7CF8091C00085FFFCCF8AE08093B4
:10C79000C600FE01EB58FF4F06C09091C00095FF08
:10C7A000FCCF8093C60081918111F7CF8091C000AA
:10C7B00085FFFCCF8AE08093C6008BE1FE01E05C40
:10C7C000FF4FDE01939601900D928A95E1F78EE975
:10C7D00092E09AA389A3AE014F5D5F4FBE01655AF7
:10C7E0007F4FC8010E942B63CE0181960E944D2984
:10C7F000CE01CE960E944D296EC0853E09F46BC0D5
:10C800008E3209F468C08F3509F465C093FD63C0AA
:10C8100081E0203109F080E0F80183A7811108C090
:10C820008985873409F057C08A858E3709F453C04B
:10C8300098012D5F3F4FBE016F5F7F4FC901CE57FB
:10C84000DF4F2883C258D040CD57DF4F3883C358BD
:10C85000D0400E941963F5018081CE57DF4F2881B7
:10C86000C258D040CD57DF4F3881C358D0408111D6
:10C870001EC0F60106C09091C00095FFFCCF8093CA
:10C88000C60081918111F7CFF90106C09091C000D7
:10C8900095FFFCCF8093C60081918111F7CF8091E5
:10C8A000C00085FFFCCF8AE08093C60014C08130B1
:10C8B00039F4F401808191810196918380830BC0CA
:10C8C000823049F4232D30E0F401808191812817D2
:10C8D0003907F9F03394A201BE016F5F7F4FC701A2
:10C8E0000E941D3018160CF4F0CE13C0BE016F5F0D
:10C8F0007F4FCE018B589F4F0E9419636C961FAEDD
:10C900006C97F60180818111F6CEEECE898181117E
:10C9100074CFCD57DF4F0FB6F894DEBF0FBECDBF3B
:10C92000DF91CF911F910F91FF90EF90DF90CF900B
:10C93000BF90AF909F908F907F906F905F904F903F
:10C940003F902F900895EF92FF920F931F93CF93F4
:10C95000DF93CDB7DEB76D970FB6F894DEBF0FBE8D
:10C96000CDBF8C01FC01EF50FF4F10827C0180E3B2
:10C97000E80EF11C40E050E0BA01C7010E94E1302E
:10C980008BE1F701DE01139601900D928A95E1F794
:10C990008EE992E09A838983AE014F5F5F4F67EB28
:10C9A00072E0C8010E942B63CE0101960E944D29BE
:10C9B0006D960FB6F894DEBF0FBECDBFDF91CF915D
:10C9C0001F910F91FF90EF900895EF92FF920F93B8
:10C9D0001F93CF93DF93EC011A828BA9882321F058
:10C9E000CE01C0960E94C8317E0184EAE80EF11C97
:10C9F0004BE060E0C7010E944D6C81111FC0EAE36B
:10CA0000F1E107C09091C00095FFFCCF8093C60074
:10CA1000319684918111F6CFE0E4F1E107C0909165
:10CA2000C00095FFFCCF8093C600319684918111A0
:10CA3000F6CF8091C00085FFFCCF76C08E010755F0
:10CA40001F4F41E0B701C8010E94EF39811126C094
:10CA500040E0B701C8010E94EF3981111FC0EDE429
:10CA6000F1E107C09091C00095FFFCCF8093C60014
:10CA7000319684918111F6CFE4E5F1E107C0909100
:10CA8000C00095FFFCCF8093C60031968491811140
:10CA9000F6CF8091C00085FFFCCF46C0B801CE0123
:10CAA000C0960E94802E81111FC0EDE4F1E107C005
:10CAB0009091C00095FFFCCF8093C6003196849181
:10CAC0008111F6CFE7E6F1E107C09091C00095FF34
:10CAD000FCCF8093C600319684918111F6CF80916E
:10CAE000C00085FFFCCF20C081E08A83EAE3F1E14A
:10CAF00007C09091C00095FFFCCF8093C60031968F
:10CB000084918111F6CFE7E7F1E107C09091C00071
:10CB100095FFFCCF8093C600319684918111F6CFAA
:10CB20008091C00085FFFCCF8AE08093C6008BE136
:10CB3000FE01F096DE01A15BBF4F01900D928A9538
:10CB4000E1F7FE01E55BFF4FAE96D183C083DF9135
:10CB5000CF911F910F91FF90EF900895FC011182EA
:10CB600012820895FC012281222311F021E0218309
:10CB70000895FC0121812111118208952F923F9285
:10CB80004F925F926F927F928F929F92AF92BF92DD
:10CB9000CF92DF92EF92FF920F931F93CF93DF9389
:10CBA000CDB7DEB7AB970FB6F894DEBF0FBECDBFE3
:10CBB0008C016B014BA7FC018281882309F4B5C16C
:10CBC0004801F9EC8F0E911CC4010E94C831F80194
:10CBD00011821B821E828EE992E09A83898318015A
:10CBE000FBE42F0E311CC8018E96F10191838083E6
:10CBF000F60180818F3209F08DC06FE270E0C601CE
:10CC00000E94497501967C0144244394512C4C0E9A
:10CC10005D1E7BC06FE270E0C7010E9449755C0138
:10CC2000009709F47EC0E816F90608F07AC03C01C6
:10CC30006E187F08A301B701CE014E960E94697558
:10CC4000EEE1F0E0EC0FFD1FE60DF71D10829EE116
:10CC5000E92EF12CEC0EFD1EF70106C09091C000EC
:10CC600095FFFCCF8093C60081918111F7CF809111
:10CC7000C00085FFFCCFFAE0F093C600F1016081AF
:10CC800071816115710519F06E5F7F4F02C060E020
:10CC900070E021E0AE01425E5F4FCE0103960E943C
:10CCA000EF3381112BC0E2E8F1E107C09091C000A1
:10CCB00095FFFCCF8093C600319684918111F6CF09
:10CCC00006C09091C00095FFFCCF8093C600F7018D
:10CCD00081917F018111F5CFE6E9F1E107C09091E3
:10CCE000C00095FFFCCF8093C600319684918111DE
:10CCF000F6CF8091C00085FFFCCF10C1F1015182B9
:10CD000040827501FFEFEF1AFF0AE114F10409F008
:10CD100081CF06C0C801835B9F4FF101918380835F
:10CD20007601F801E55BFF4F8BA560817181882357
:10CD300009F49CC06115710519F06E5F7F4F02C048
:10CD400060E070E021E0A701C4010E94EF33882376
:10CD500009F462C0F801EC51FF4FD801A753BF4F4F
:10CD600051968D919D910D90BC91A02D80839183C2
:10CD7000A283B383E8E9F1E107C09091C00095FF79
:10CD8000FCCF8093C600319684918111F6CFF701D4
:10CD900006C09091C00095FFFCCF8093C6008191A2
:10CDA0008111F7CFE5EAF1E107C09091C00095FF4E
:10CDB000FCCF8093C600319684918111F6CFF801A3
:10CDC000EC51FF4F40815181628173812AE030E054
:10CDD0008DE296E00E94522C8091C00085FFFCCF2E
:10CDE0008AE08093C600F801E451FF4F108211825F
:10CDF00012821382ECEAF1E107C09091C00095FF26
:10CE0000FCCF8093C600319684918111F6CF80913A
:10CE1000C00085FFFCCF82C0EAEBF1E107C0909132
:10CE2000C00095FFFCCF8093C6003196849181119C
:10CE3000F6CFF70106C09091C00095FFFCCF80931C
:10CE4000C60081918111F7CFEEECF1E107C090911E
:10CE5000C00095FFFCCF8093C6003196849181116C
:10CE6000F6CF8091C00085FFFCCF58C061157105D9
:10CE700019F06E5F7F4F02C060E070E026E5A70109
:10CE8000C4010E94EF3381112AC0E0EDF1E107C037
:10CE90009091C00095FFFCCF8093C600319684919D
:10CEA0008111F6CFF70106C09091C00095FFFCCF2D
:10CEB0008093C60081918111F7CFE4EEF1E107C0C4
:10CEC0009091C00095FFFCCF8093C600319684916D
:10CED0008111F6CF8091C00085FFFCCF1FC081E09B
:10CEE000F8018083E6EEF1E107C09091C00095FF64
:10CEF000FCCF8093C600319684918111F6CFF60164
:10CF000006C09091C00095FFFCCF8093C600819130
:10CF10008111F7CF8091C00085FFFCCF8AE080931C
:10CF2000C600CE0101960E944D29AB960FB6F8942B
:10CF3000DEBF0FBECDBFDF91CF911F910F91FF904C
:10CF4000EF90DF90CF90BF90AF909F908F907F90A9
:10CF50006F905F904F903F902F9008953F924F9227
:10CF60005F926F927F928F929F92AF92BF92CF9279
:10CF7000DF92EF92FF920F931F93CF93DF93CDB782
:10CF8000DEB7AA970FB6F894DEBF0FBECDBF7C0107
:10CF90006B01FC018281882309F40EC1C70187530C
:10CFA0009F4F0E94C831F70111821B821E828EE9B9
:10CFB00092E09A8389832701FBE44F0E511CC7013D
:10CFC0008E96F20191838083F60180818F3209F081
:10CFD0008CC06FE270E0C6010E9449758C010F5F42
:10CFE0001F4F3AE0332E66246394712C6C0E7D1E25
:10CFF00077C06FE270E0C8010E9449755C0100973C
:10D0000009F47AC00817190708F076C04C01801A95
:10D01000910AA401B801CE014E960E946975EEE115
:10D02000F0E0EC0FFD1FE80DF91D10828E01025E8D
:10D030001F4FF80106C09091C00095FFFCCF809370
:10D04000C60081918111F7CF8091C00085FFFCCF90
:10D050003092C600F201608171816115710519F08D
:10D060006E5F7F4F02C060E070E021E0AE01425E83
:10D070005F4FCE0103960E94EF3381112BC0E8EF82
:10D08000F1E107C09091C00095FFFCCF8093C600EE
:10D09000319684918111F6CF06C09091C00095FF22
:10D0A000FCCF8093C600F80181918F018111F5CFEB
:10D0B000ECE0F2E107C09091C00095FFFCCF8093B7
:10D0C000C600319684918111F6CF8091C00085FF12
:10D0D000FCCF6BC0F2017182608285010F5F1F4F30
:10D0E0000115110509F085CF06C0C701835B9F4F6D
:10D0F000F201918380838601F701E55BFF4F808118
:10D100009181009711F0029602C080E090E0B80192
:10D110000E94AF34882301F1EEE0F2E107C0909164
:10D12000C00095FFFCCF8093C60031968491811199
:10D13000F6CFF80106C09091C00095FFFCCF809318
:10D14000C60081918111F7CFF701E451FF4F1082A2
:10D150001182128213822CC0ECE1F2E107C090919F
:10D16000C00095FFFCCF8093C60031968491811159
:10D17000F6CFF80106C09091C00095FFFCCF8093D8
:10D18000C60081918111F7CFE4E3F2E107C09091ED
:10D19000C00095FFFCCF8093C60031968491811129
:10D1A000F6CF8091C00085FFFCCF8AE08093C60057
:10D1B000CE0101960E944D29AA960FB6F894DEBFC3
:10D1C0000FBECDBFDF91CF911F910F91FF90EF90D8
:10D1D000DF90CF90BF90AF909F908F907F906F9097
:10D1E0005F904F903F900895CF93DF93EC018A8139
:10D1F0008823C1F1E6E3F2E107C09091C00095FFFA
:10D20000FCCF8093C600319684918111F6CFFE0148
:10D21000E451FF4F40815181628173812AE030E007
:10D220008DE296E00E94522CE8E4F2E107C0909172
:10D23000C00095FFFCCF8093C60031968491811188
:10D24000F6CFCC51DF4F488159816A817B812AE03A
:10D2500030E08DE296E00E94522C8091C00085FF64
:10D26000FCCF11C0EAE4F2E107C09091C00095FF45
:10D27000FCCF8093C600319684918111F6CF8091C6
:10D28000C00085FFFCCF8AE08093C600DF91CF917C
:10D290000895CF92DF92EF92FF920F931F93CF9357
:10D2A000DF937C01EB01EC2FFD2FDF010D900020BF
:10D2B000E9F78D01015011090E1B1F0BF701E75310
:10D2C000FF4F10826EE470E0CE010E9449756C0140
:10D2D000009729F4F8013197EC0FFD1F0DC060E2B3
:10D2E00070E00E944975EC0121966AE270E0C60187
:10D2F0000E944975FC0131978DE081838AE0828329
:10D300001382BE01C70189539F4F0E947436F701F3
:10D31000E753FF4F8081882309F1EDE4F1E107C075
:10D320009091C00095FFFCCF8093C6003196849108
:10D330008111F6CFEAE5F2E107C09091C00095FFB8
:10D34000FCCF8093C600319684918111F6CF8091F5
:10D35000C00085FFFCCF8AE08093C600DF91CF91AB
:10D360001F910F91FF90EF90DF90CF9008953F9223
:10D370004F925F926F927F928F929F92AF92BF92E5
:10D38000CF92DF92EF92FF920F931F93CF93DF9391
:10D39000CDB7DEB7CC55D1090FB6F894DEBF0FBEBE
:10D3A000CDBF8C01662349F0F801E051FF4F108298
:10D3B000F8018281811118C031C0FC01E051FF4F9A
:10D3C0008081882309F4ADC0F801E851FF4FC08087
:10D3D000D180E280F3800E94C229C616D706E806F3
:10D3E000F90608F49EC0E0CFF80185A58F9384A5C7
:10D3F0008F938AE093E09F938F937E01FFE3EF0E7C
:10D40000F11CFF92EF920E9492750F900F900F9077
:10D410000F900F900F906701570110C0C8010E9434
:10D42000E564F80182818111DFCF7BC0F601808144
:10D4300090E00E940875F60181936F01F50101905B
:10D440000020E9F73197EA19FB098C2D8E198E1708
:10D450006CF34801F0E38F0E911C40E050E0BA01FC
:10D46000C4010E94E130312CEE24E394F12CEC0E47
:10D47000FD1E6E018FE3C80ED11C63E1662E63E0D2
:10D48000762E5E01E1E2AE0EB11C35C0F201808164
:10D4900090E00E940875F20181932F01F70101903D
:10D4A0000020E9F73197EE19FF09842D8E198E17A8
:10D4B0006CF38A858E37F9F045E050E0B601C7017C
:10D4C0000E945B750097B9F4DF92CF927F926F92C2
:10D4D000BF92AF920E949275C5010E94810F8AE1AE
:10D4E00093E00E94810F0F900F900F900F900F907C
:10D4F0000F903324339440E050E0B701C4010E9400
:10D500001D30181614F42701C9CF311004C08FEF55
:10D510009FEFF80104C0F80184A595A5019695A791
:10D5200084A7C45ADF4F0FB6F894DEBF0FBECDBF3D
:10D53000DF91CF911F910F91FF90EF90DF90CF90EF
:10D54000BF90AF909F908F907F906F905F904F9023
:10D550003F9008950F931F93CF93DF93EC018C01BD
:10D5600007531F4FC8010E947C31C8010E94C83177
:10D570001882DF91CF911F910F910895CF93DF9380
:10D58000EC010E9480560E94F45619828EE193E0CD
:10D590000E94810F8091920D8823A1F11092920D2B
:10D5A00060912C03E62FF0E0EE0FFF1FE459F14FDE
:10D5B000808191810E94095820913301309134017A
:10D5C00040913501509136010E946A701816D4F4CA
:10D5D00060912C03C62FD0E080E090E00E94395784
:10D5E000FE01EE0FFF1FE459F14F91838083FE018E
:10D5F000EE0FFF1FEE0FFF1FEE59F14F1082118249
:10D6000012821382DF91CF910895EF92FF920F93D0
:10D610001F93CF93DF937C01EB018A01060F171F45
:10D6200009C06991D701ED91FC910190F081E02D45
:10D63000C7010995C017D107A1F7DF91CF911F91BD
:10D640000F91FF90EF9008958FEF8EBD0DB407FE00
:10D65000FDCF8EB508958EBD0DB407FEFDCF0895A4
:10D6600061E0FC0180810C94FD2AFC014281242FA1
:10D6700030E03595279520652CBD40FD03C021E0A5
:10D68000463009F420E02DBD60E0FC0180810C945F
:10D69000FD2ACF92DF92EF92FF920F931F93CF93C9
:10D6A000DF93EC018B017A010E94C2296B0109C052
:10D6B0000E94C2296C197D096D32714010F081E120
:10D6C00008C00E94246B8B838F3F91F38E3F19F02B
:10D6D0008FE0898328C0E114F104E1F081E0E81AC9
:10D6E000F1088FEF8EBDF8012FEF06C00DB407FED5
:10D6F000FDCF8EB581932EBDCF01801B910B8E1572
:10D700009F05A0F30DB407FEFDCF8EB5F801EE0D19
:10D71000FF1D80830E94246B0E94246BCE010E9417
:10D72000306B81E004C0CE010E94306B80E0DF915D
:10D73000CF911F910F91FF90EF90DF90CF900895C0
:10D740000F931F93CF93DF93EB010E94C2298B01AC
:10D7500007C00E94C229601B710B6C177D0730F453
:10D760000E94246B8F3FA9F781E001C080E0DF9128
:10D77000CF911F910F910895CF92DF92FF920F9357
:10D780001F93CF93DF9300D000D0CDB7DEB76C01ED
:10D79000F62E29833A834B835C830E94356B6CE2BF
:10D7A00071E0C6010E94A06B8F2D80640E942B6BDC
:10D7B00008E110E05C814B813A812981DA01C901DD
:10D7C000002E04C0B695A795979587950A94D2F731
:10D7D00029833A834B835C830E942B6B0850110989
:10D7E00029813A814B815C81083F8FEF180731F71F
:10D7F000FF2029F0E8E0FE1621F08FEF03C085E955
:10D8000001C087E80E942B6BFCE0FF1202C00E945F
:10D81000246B10E00E94246BF601838387FF04C011
:10D820001F3F11F01F5FF6CF0F900F900F900F90DA
:10D83000DF91CF911F910F91FF90DF90CF900895CE
:10D840000F931F93CF93DF93EC0189018C81833079
:10D8500039F0B9E0440F551F661F771FBA95D1F70D
:10D860009A01AB0161E1CE010E94BC6B81110AC03B
:10D8700040E052E0B801CE01DF91CF911F910F91AE
:10D880000C94496B84E08983CE010E94306B80E068
:10D89000DF91CF911F910F910895BF92CF92DF92A8
:10D8A000EF92FF920F931F93CF93DF93EC01B62E6D
:10D8B0001C82198248830E94C2298B0161E0888101
:10D8C0000E94E12ACE010E94306B60E086E00E9457
:10D8D000E12A61E085E00E94E12A61E087E00E94A0
:10D8E000E12A61E084E00E94E12A61E084E00E9494
:10D8F000FD2A85E08A8382E58CBD1DBC2AE0F22EDC
:10D900008FEF0E942B6BFA94D9F709C00E94C229AD
:10D91000601B710B613D774010F081E058C020E042
:10D9200030E0A90160E0CE010E94BC6BF82E8B8331
:10D9300081E0F812EBCF2AEA31E040E050E068E005
:10D94000CE010E94BC6B82FF02C0FC820DC094E03D
:10D95000F92E0E94246B8B83FA94D9F78A3A11F03E
:10D9600082E035C082E08C838C81823031F4C12C1E
:10D97000D12CE12C80E4F82E0DC0C12CD12C7601E5
:10D9800009C00E94C229601B710B613D774010F0F5
:10D990008AE01DC020E030E0A90167E3CE010E94CB
:10D9A000BC6BA701960169E2CE010E94BC6B8B8320
:10D9B0008111E7CF8C818230C9F420E030E0A901E9
:10D9C0006AE3CE010E94BC6B882319F088E089834A
:10D9D00019C00E94246B807C803C11F483E08C830E
:10D9E0000E94246B0E94246B0E94246BCE010E9433
:10D9F000306B86E08B1518F488E1898306C0BA8203
:10DA000081E004C0CE010E94306B80E0DF91CF91B5
:10DA10001F910F91FF90EF90DF90CF90BF900895EE
:10DA2000CF93DF93EC016EBD20E030E00DB407FE34
:10DA3000FDCFFA01E20FF31F80818EBD0DB407FE0A
:10DA4000FDCF81818EBD2E5F3F4F211582E03807CB
:10DA500069F70DB407FEFDCF8FEF0E942B6B8FEFA0
:10DA60000E942B6B0E94246B8B838F71853039F061
:10DA700083E18983CE010E94306B80E001C081E0A8
:10DA8000DF91CF9108950F931F93CF93DF93EC0114
:10DA900089018C81833039F0E9E0440F551F661FFE
:10DAA000771FEA95D1F79A01AB0168E1CE010E9498
:10DAB000BC6B882311F086E029C0A8016EEFCE016F
:10DAC0000E94106D8823B9F068E572E0CE010E94D3
:10DAD000A06B811102C087E119C020E030E0A901EC
:10DAE0006DE0CE010E94BC6B81110FC00E94246BBF
:10DAF00081110BC005C0CE010E94306B80E008C0D0
:10DB0000CE010E94306B81E003C086E18983F3CFB0
:10DB1000DF91CF911F910F9108955058BB27AA27ED
:10DB20000ED076C23FD230F044D220F031F49F3F85
:10DB300011F41EF40FC20EF4E095E7FBDCC1E92FEF
:10DB400089D280F3BA17620773078407950718F024
:10DB500071F49EF5B8C20EF4E0950B2EBA2FA02DED
:10DB60000B01B90190010C01CA01A0011124FF278A
:10DB7000591B99F0593F50F4503E68F11A16F04085
:10DB8000A22F232F342F4427585FF3CF4695379584
:10DB90002795A795F0405395C9F77EF41F16BA0B49
:10DBA000620B730B840BBAF09150A1F0FF0FBB1FF7
:10DBB000661F771F881FC2F70EC0BA0F621F731F40
:10DBC000841F48F4879577956795B795F7959E3F9D
:10DBD00008F0B3CF9395880F08F09927EE0F97952B
:10DBE00087950895DFD158F080E891E009F49EEF21
:10DBF000E0D128F040E851E059F45EEF09C0AAC135
:10DC000062C2E92FE07826D268F3092E052AC1F313
:10DC1000261737074807590738F00E2E07F8E02572
:10DC200069F0E025E0640AC0EF6307F8009407FAA2
:10DC3000DB01B9019D01DC01CA01AD01EF935DD0AB
:10DC4000E7D10AD05F91552331F02BED3FE049E455
:10DC500050FD49EC63CF0895DF93DD27B92FBF77DF
:10DC600040E85FE31616170648075B0710F4D92F44
:10DC700096D29F938F937F936F93A9D3E0E7F0E0C1
:10DC80006CD1C6D12F913F914F915F9101D3DD238C
:10DC900049F09058A2EA2AED3FE049EC5FE3D078E2
:10DCA0005D274DDFDF91B4C1F7D180F09F3740F49D
:10DCB00091110EF409C260E070E080E89FE30895DE
:10DCC00026F01B16611D711D811D1BC135C1EFD0D2
:10DCD00008F481E0089575D1E395ABC10CD098C1EB
:10DCE00068D140F05FD130F021F45F3F19F003C1FB
:10DCF0005111EAC12FC1AED198F39923C9F355232D
:10DD0000B1F3951B550BBB27AA276217730784072E
:10DD100038F09F5F5F4F220F331F441FAA1FA9F3E4
:10DD200033D00E2E3AF0E0E830D091505040E695D6
:10DD3000001CCAF729D0FE2F27D0660F771F881F37
:10DD4000BB1F261737074807AB07B0E809F0BB0B26
:10DD5000802DBF01FF2793585F4F2AF09E3F51054A
:10DD600068F0C9C0B1C15F3FECF3983EDCF3869523
:10DD700077956795B795F7959F5FC9F7880F911DC0
:10DD80009695879597F90895E1E0660F771F881FAC
:10DD9000BB1F621773078407BA0720F0621B730B5F
:10DDA000840BBA0BEE1F88F7E095089504D06894B1
:10DDB000B1118AC1089556D188F09F5790F0B92FBC
:10DDC0009927B751A0F0D1F0660F771F881F991FD0
:10DDD0001AF0BA95C9F712C0B13081F074D1B1E030
:10DDE000089571C1672F782F8827B85F39F0B93F40
:10DDF000CCF3869577956795B395D9F73EF49095D2
:10DE00008095709561957F4F8F4F9F4F0895E8944F
:10DE100009C097FB3EF490958095709561957F4F72
:10DE20008F4F9F4F9923A9F0F92F96E9BB27939520
:10DE3000F695879577956795B795F111F8CFFAF430
:10DE4000BB0F11F460FF1BC06F5F7F4F8F4F9F4F61
:10DE500016C0882311F096E911C0772321F09EE8BF
:10DE6000872F762F05C0662371F096E8862F70E025
:10DE700060E02AF09A95660F771F881FDAF7880FFF
:10DE80009695879597F9089507D180F09F3740F4CC
:10DE900091110EF019C160E070E080E89FEB0895E9
:10DEA00026F41B16611D711D811D2BC045C0990FE5
:10DEB0000008550FAA0BE0E8FEEF16161706E80754
:10DEC000F907C0F012161306E407F50798F0621B75
:10DED000730B840B950B39F40A2661F0232B242B4A
:10DEE000252B21F408950A2609F4A140A6958FEF69
:10DEF000811D811D089597F99F6780E870E060E0BB
:10DF00000895882371F4772321F09850872B762F7A
:10DF100007C0662311F499270DC09051862B70E03D
:10DF200060E02AF09A95660F771F881FDAF7880F4E
:10DF30009695879597F908959F3F31F0915020F479
:10DF4000879577956795B795880F911D96958795D5
:10DF500097F908959FEF80EC0895DF93CF931F9377
:10DF60000F93FF92EF92DF927B018C01689405C0C2
:10DF7000DA2EEF018DD1FE01E894A591259135911E
:10DF800045915591AEF3EF01DADDFE019701A8014D
:10DF9000DA9479F7DF90EF90FF900F911F91CF9176
:10DFA000DF91089500240A9416161706180609062C
:10DFB000089500240A9412161306140605060895FF
:10DFC000C9CF50D0E8F3E894E0E0BB279F57F0F0CA
:10DFD0002AED3FE049EC06C0EE0FBB0F661F771F2E
:10DFE000881F28F0B23A62077307840728F0B25AF4
:10DFF000620B730B840BE3959A9572F7803830F4BB
:10E000009A95BB0F661F771F881FD2F7904896CF4F
:10E01000092E0394000C11F4882352F0BB0F40F436
:10E02000BF2B11F460FF04C06F5F7F4F8F4F9F4F76
:10E030000895EF93E0FF06C0A2EA2AED3FE049EC25
:10E040005FEB7DDDE5DF0F90039401FC9058EDE977
:10E05000F0E0C7C157FD9058440F551F59F05F3F7E
:10E0600071F04795880F97FB991F61F09F3F79F0FA
:10E0700087950895121613061406551FF2CF46957C
:10E08000F1DF08C0161617061806991FF1CF8695FE
:10E090007105610508940895E5DFA0F0BEE7B917A2
:10E0A00088F4BB279F3860F41616B11D672F782FB0
:10E0B0008827985FF7CF869577956795B11D9395DB
:10E0C0009639C8F30895E894BB2766277727CB01D4
:10E0D00097F90895ECDE08F48FEF089563DF19F0E7
:10E0E00068DF09F037CF07CFB901CA0125CF9F7785
:10E0F0005F77B0DF98F39923B9F35523B9F3FF277E
:10E10000951758F4E52FE91BED3070F75E3B10F0E2
:10E11000F1E41CC09034E0F40AC0E92FE51BED30B7
:10E1200028F79E3B10F0F1E411C0503488F4F9EA6E
:10E1300088232AF09A95660F771F881FDAF7442301
:10E140002AF05A95220F331F441FDAF79F1B5F1BDB
:10E15000FF931F930F93FF92EF9279018A01BB27E0
:10E16000AB2F9B01AC0196D09701A801BF937B0117
:10E170008C01AA27BA2FB901CA018CD0AF9197019F
:10E18000A801EF90FF900F911F91D9DC41DFE1D002
:10E190004F9140FF0895552747FD509509C09B01B9
:10E1A000AC0160E070E080E89FE398CDA4CEC4CEDF
:10E1B00059DFE8F39923D9F3940F511DBBF3915024
:10E1C000504094F059F0882332F0660F771F881F73
:10E1D00091505040C1F79E3F510544F7880F911D63
:10E1E0009695879597F908955F3FACF0983E9CF01F
:10E1F000BB27869577956795B79508F4B160939599
:10E20000C1F7BB0F58F711F460FFE8CF6F5F7F4F86
:10E210008F4F9F4FE3CF58CF25DF58F19E5758F1CE
:10E220009851A0F0E9F0983020F5092E9927660F53
:10E23000771F881F991F0A94D1F712C0062E672FE7
:10E24000782F8827985F11F4000C07C0993FB4F32A
:10E250008695779567959395D9F7611D711D811DF9
:10E260003EF490958095709561957F4F8F4F9F4FAD
:10E270000895689429CF27CF0BD0CACE93DE28F01B
:10E2800098DE18F0952309F036CE64CE11241CCF09
:10E29000E1DEA0F3959FD1F3950F50E0551F629FEB
:10E2A000F001729FBB27F00DB11D639FAA27F00DEF
:10E2B000B11DAA1F649F6627B00DA11D661F829F16
:10E2C0002227B00DA11D621F739FB00DA11D621FFB
:10E2D000839FA00D611D221F749F3327A00D611D18
:10E2E000231F849F600D211D822F762F6A2F1124FA
:10E2F0009F5750408AF0E1F088234AF0EE0FFF1F4D
:10E30000BB1F661F771F881F91505040A9F79E3F83
:10E31000510570F0F0CDD8CE5F3FECF3983EDCF3C2
:10E32000869577956795B795F795E7959F5FC1F7C0
:10E33000FE2B880F911D9695879597F908959F93C9
:10E3400040DE0F9007FCEE5F74CE11F40EF402CEA7
:10E35000F3CD88DED0F39923D9F3CEF39F57550B35
:10E3600087FF38D00024A0E640EA900180585695F7
:10E37000979528F4805C660F771F881F20F026177A
:10E380003707480730F4621B730B840B20293129AF
:10E390004A2BA69517940794202531254A2758F72C
:10E3A000660F771F881F20F026173707480730F4BD
:10E3B000620B730B840B200D311D411DA09581F75D
:10E3C000B901842F9158880F9695879508959B01E0
:10E3D000AC0152CF91505040660F771F881FD2F783
:10E3E00008959F938F937F936F93FF93EF939B0178
:10E3F000AC0142DFEF91FF91B0DD2F913F914F9142
:10E400005F913ACF0E947772A59F900DB49F900DB7
:10E41000A49F800D911D11240895B7FF0C940272E2
:10E420000E940272821B930B0895DB018F939F93CE
:10E430000E940272BF91AF91A29F800D911DA39F78
:10E44000900DB29F900D1124089597FB072E16F49E
:10E45000009407D077FD09D00E94837207FC05D095
:10E460003EF4909581959F4F0895709561957F4FEB
:10E470000895A1E21A2EAA1BBB1BFD010DC0AA1F05
:10E48000BB1FEE1FFF1FA217B307E407F50720F01D
:10E49000A21BB30BE40BF50B661F771F881F991F98
:10E4A0001A9469F760957095809590959B01AC01E1
:10E4B000BD01CF010895052E97FB16F4009407D0F7
:10E4C00057FD0DD00E94397207FC09D07EF490955B
:10E4D0008095709561957F4F8F4F9F4F0895509510
:10E4E0004095309521953F4F4F4F5F4F0895A29F24
:10E4F000B001B39FC001A39F01D0B29F700D811DD9
:10E500001124911D0895AA1BBB1B51E107C0AA1F2E
:10E51000BB1FA617B70710F0A61BB70B881F991FC4
:10E520005A95A9F780959095BC01CD010895EE0FFD
:10E53000FF1F0590F491E02D0994A0E0B0E0E3EA1C
:10E54000F2E70C9439787B016115710521F0DB014C
:10E550008C9311969C93EC01C9908E018C2D90E0C8
:10E560000E940075892BC1F7BDE2CB1206C0FE01E7
:10E57000C1908F01DD24D39407C0FBE2CF1203C00A
:10E58000DE01CD908D01D12CE801219743E050E0D0
:10E590006AED72E1CE010E941075892BC9F4E80181
:10E5A000229645E050E06DED72E1CE010E941075BB
:10E5B000892B11F4E8012796E114F10419F0F70111
:10E5C000D183C083812C912C90E8D110F3C0F7C087
:10E5D00043E050E062EE72E1CE010E941075892B9B
:10E5E00051F4E114F10409F4E7C00E5F1F4FD701A5
:10E5F0000D931C93E1C060E070E0CB01C0E0D0E07F
:10E60000EC2DE053EA3020F5FD2DF2602D2D287021
:10E61000D2FE04C0211122C0219620C021112197D1
:10E62000A5E0B0E09B01AC010E940272660F771F6B
:10E63000881F991F6E0F711D811D911D6839B9E9E1
:10E640007B078B07B9E19B0748F0FD2DF66006C0FC
:10E65000EE3F49F4D3FC43C0FD2DF860D801CD90C6
:10E660008D01DF2ECDCFE53311F0E531C1F5F80195
:10E67000A081AD3219F4F0E1DF2A07C0AB3229F0F6
:10E680000F5F1F4F21E030E006C0F801A1810E5F4F
:10E690001F4F22E030E0A053AA3018F0021B130BEA
:10E6A0001EC0F80120E030E020384CE034075CF474
:10E6B000A901440F551F440F551F240F351F220F6A
:10E6C000331F2A0F311DA191A0538F01AA3060F38F
:10E6D000D4FE03C0319521953109C20FD31FD1FE5D
:10E6E00008C0E114F10429F001501109D7010D937C
:10E6F0001C930E94076F2D2D2370233019F04B01BE
:10E700005C0105C0DC01CB01B0584C015D0120E08B
:10E7100030E0A901682D792D8A2D9B2D0E94676E0E
:10E72000882309F444C0D7FF06C0D195C195D1090B
:10E7300001E113E102C009EF12E16801B8E1CB1A6F
:10E74000D10890E2E92EF12C13C0F8018591959142
:10E75000A591B491282F392F4A2F5B2F682D792D41
:10E760008A2D9B2D0E943C714B015C01CE19DF0963
:10E77000CE15DF0554F704501109F594E7940C15F4
:10E780001D05B1F7B401C501282F220F292F221F23
:10E790002F3F39F020E030E0A9010E94676E81111F
:10E7A00006C082E290E09093B20E8093B10E9A2D53
:10E7B0008B2D06C08FEF04C0812C912C90EC8FE73D
:10E7C0009C01682D792D832F922FCDB7DEB7ECE019
:10E7D0000C945578A0E0B0E0E0EFF3E70C943578C6
:10E7E0005B01EA016115710519F0FB0180839183DA
:10E7F000209739F09E01225031092332310508F06B
:10E80000E6C07C01F70191907F018F01892D90E096
:10E810000E940075892BB1F7FDE29F1206C0F70137
:10E8200091908F018824839407C0FBE29F1203C05C
:10E83000F70191908F01812C209709F4D6C0C03147
:10E84000D10581F4CEC0F8018081883719F0883570
:10E8500009F0C1C0F80191800E5F1F4FF2E08F2ACE
:10E86000C0E1D0E0C830D105D9F024F4C230D105E0
:10E87000F9F407C0CA30D10551F0C031D105C1F457
:10E8800025C0C12CD12CE12C40E4F42E24C0CAE0D8
:10E89000D0E03CECC32EDC2CEC2C3CE0F32E1BC077
:10E8A000C8E0D0E0C12CD12CE12C20E1F22E13C025
:10E8B0009E01442737FD4095542F60E070E080E0D2
:10E8C00090E80E94397269017A0105C0C12CD12CEF
:10E8D000E12C98E0F92E40E060E070E0CB012E01E1
:10E8E000662457FC6094762CE92DE053EA3060F002
:10E8F000292D21542A3110F4E75006C0292D215624
:10E900002A3128F5E92DE7552E2F30E02C173D0749
:10E91000F4F447FD18C0C616D706E806F90680F0DD
:10E920009B01AC01C301B2010E9415726E0F711DF3
:10E93000811D911D61307105810520E8920710F05D
:10E940004FEF01C041E0F80191908F01CDCFA114AC
:10E95000B10481F0442331F001501109F501118314
:10E96000008308C081FE1AC002501109F50111830D
:10E97000008314C047FF12C080FE05C060E070E055
:10E9800080E090E804C06FEF7FEF8FEF9FE722E217
:10E9900030E03093B20E2093B10E16C080FE08C056
:10E9A00090958095709561957F4F8F4F9F4F0CC0CC
:10E9B00097FF0AC082E290E09093B20E8093B10E6E
:10E9C0006FEF7FEF8FEF9FE78B019C0112C000E09C
:10E9D00010E098010EC080E3982E209709F460CFD4
:10E9E00041CFF0E39F123ECF2ECF20E392124FCFC4
:10E9F0002ACFB801C901CDB7DEB7E0E10C94517858
:10EA000091118EC2803219F089508550D0F7089547
:10EA10009111089581548A5108F4805E855A0895B1
:10EA2000FB01DC014150504088F08D9181341CF095
:10EA30008B350CF4805E659161341CF06B350CF401
:10EA4000605E861B611171F3990B0895881BFCCFE2
:10EA5000FB01DC0104C08D910190801921F441502B
:10EA60005040C8F7881B990B0895FB01DC0102C0D8
:10EA700001900D9241505040D8F70895FB01DC0100
:10EA80000D900020E9F7119701900D920020E1F719
:10EA90000895FC018191861721F08823D9F79927E1
:10EAA00008953197CF010895FB01DC0101900D928B
:10EAB0000020E1F70895FB01DC014150504030F0A7
:10EAC0008D910190801919F40020B9F7881B990BDA
:10EAD0000895FB01DC014150504048F001900D9237
:10EAE0000020C9F701C01D9241505040E0F7089541
:10EAF000FB0151915523A9F0BF01DC014D91451750
:10EB00004111E1F759F4CD010190002049F04D91F8
:10EB100040154111C9F3FB014111EFCF81E090E0B5
:10EB200001970895AEE0B0E0E8E9F5E70C9441788C
:10EB30000D891E8986E08C831A8309838FEF9FE7F6
:10EB40009E838D83CE014996AC016F89788DCE016D
:10EB500001960E94B475EF81F885E00FF11F1082D5
:10EB60002E96E4E00C945D78ACE0B0E0EAEBF5E7DB
:10EB70000C9433787C016B018A01FC0117821682A8
:10EB8000838181FFC6C188248394912C8C0E9D1EA5
:10EB9000F7019381F60193FD859193FF81916F01B8
:10EBA000882309F4B2C1853239F493FD859193FF2E
:10EBB00081916F01853229F4B70190E00E94A97715
:10EBC000E7CF512C312C20E02032A8F48B3261F0B9
:10EBD00028F4803251F0833271F40BC08D3239F059
:10EBE000803349F4216028C02260246025C0286059
:10EBF00023C0206121C027FD27C0382F30533A3071
:10EC000078F426FF06C0FAE05F9E300D1124532EE3
:10EC100013C08AE0389E300D1124332E20620CC0C0
:10EC20008E3221F426FD71C1206406C08C3611F4A9
:10EC3000206802C0883641F4F60193FD859193FF68
:10EC400081916F018111C0CF982F9554933018F0A6
:10EC50009052933028F40C5F1F4FFFE3F9830DC0EF
:10EC6000833631F0833771F0833509F05EC023C0FD
:10EC7000F801808189830E5F1F4F44244394512CF7
:10EC8000540115C03801F2E06F0E711CF801A0802C
:10EC9000B18026FF03C0652D70E002C06FEF7FEFEB
:10ECA000C5012C870E949E772C0183012C856FE77C
:10ECB000262E222218C03801F2E06F0E711CF801D6
:10ECC000A080B18026FF03C0652D70E002C06FEF09
:10ECD0007FEFC5012C870E9493772C012C8550E88B
:10ECE000252E222A830123FC1CC006C0B70180E226
:10ECF00090E00E94A9773A94832D90E04816590637
:10ED0000A8F30FC0F50127FC859127FE81915F01D3
:10ED1000B70190E00E94A97731103A94F1E04F1AC0
:10ED200051084114510471F7EDC0843611F0893651
:10ED300041F5F80127FF07C06081718182819381CD
:10ED40000C5F1F4F08C060817181882777FD809517
:10ED5000982F0E5F1F4F4FE6B42EB22297FF09C0C7
:10ED600090958095709561957F4F8F4F9F4FF0E8FC
:10ED7000BF2A2AE030E0A4010E94D577A82EA81867
:10ED800043C0853731F43FEEB32EB2222AE030E0A3
:10ED900024C099EFB92EB2228F36B9F020F488350D
:10EDA00009F0B3C00DC0803721F0883709F0ADC03D
:10EDB00002C020E1B22AB4FE0BC084E0B82A08C029
:10EDC00024FF09C0E6E0BE2A06C028E030E005C006
:10EDD00020E130E002C020E132E0F801B7FE07C0D8
:10EDE00060817181828193810C5F1F4F06C06081B9
:10EDF000718180E090E00E5F1F4FA4010E94D577E3
:10EE0000A82EA818FFE7BF22B6FE0BC02B2D2E7F21
:10EE1000A51450F4B4FE0AC0B2FC08C02B2D2E7EFF
:10EE200005C07A2C2B2D03C07A2C01C0752C24FF31
:10EE30000DC0FE01EA0DF11D8081803311F4297EA1
:10EE400009C022FF06C07394739404C0822F867891
:10EE500009F0739423FD14C020FF0FC05A2C7314C3
:10EE600060F4530C5718732C08C0B70180E290E08F
:10EE70002C870E94A97773942C857314B0F304C077
:10EE8000731410F4371801C0312C24FF12C0B701DD
:10EE900080E390E02C870E94A9772C8522FF1EC07A
:10EEA00021FF03C088E590E002C088E790E0B70149
:10EEB0000CC0822F867891F021FD02C080E201C053
:10EEC0008BE227FD8DE2B70190E00E94A97706C092
:10EED000B70180E390E00E94A9775A94A514C0F38B
:10EEE000AA94F401EA0DF11DB701808190E00E941F
:10EEF000A977A110F5CF06C0B70180E290E00E948B
:10EF0000A9773A943110F8CF43CEF70126813781A3
:10EF100002C02FEF3FEFC9012C96E2E10C944F782D
:10EF2000992788270895FC010590615070400110D1
:10EF3000D8F7809590958E0F9F1F0895FC01615022
:10EF4000704001900110D8F7809590958E0F9F1F0B
:10EF500008950F931F93CF93DF938C01EB018B8167
:10EF600081FD03C00FEF1FEF1AC082FF0DC02E817D
:10EF70003F818C819D812817390764F4E881F981EC
:10EF80000193F983E88306C0E885F985802F099508
:10EF9000892B41F78E819F8101969F838E83C801C3
:10EFA000DF91CF911F910F910895FA01AA27283080
:10EFB00051F1203181F1E8946F936E7F6E5F7F4F46
:10EFC0008F4F9F4FAF4FB1E03ED0B4E03CD0670FC2
:10EFD000781F891F9A1FA11D680F791F8A1F911D15
:10EFE000A11D6A0F711D811D911DA11D20D009F465
:10EFF00068943F912AE0269F11243019305D3193A7
:10F00000DEF6CF010895462F4770405D4193B3E08F
:10F010000FD0C9F7F6CF462F4F70405D4A3318F036
:10F02000495D31FD4052419302D0A9F7EACFB4E0E7
:10F03000A6959795879577956795BA95C9F700979F
:10F040006105710508959B01AC010A2E0694579540
:10F05000479537952795BA95C9F7620F731F841F97
:10F06000951FA01D08952F923F924F925F926F922D
:10F070007F928F929F92AF92BF92CF92DF92EF9248
:10F08000FF920F931F93CF93DF93CDB7DEB7CA1BC9
:10F09000DB0B0FB6F894DEBF0FBECDBF09942A88F4
:10F0A000398848885F846E847D848C849B84AA849C
:10F0B000B984C884DF80EE80FD800C811B81AA8129
:10F0C000B981CE0FD11D0FB6F894DEBF0FBECDBFF4
:10F0D000ED01089513E1C8E1D3E104C0FE010E94EF
:0EF0E00099722296CA31D107C9F7F894FFCF72
:10F0EE000000B30E200000004D4300004D43000011
:10F0FE00F0426400640000803B4500803B45000008
:10F10E007043000000000080BB440160EA0000CDA7
:10F11E00CCCC3D0000524300007A430101010101B5
:10F12E000000803F75608944A97E443E713DE841F0
:10F13E00FF3FFF3F0133338E4233338E42000020B8
:10F14E0045000016440000FA430000FA430000A0F8
:10F15E0040000034422823000028230000640000F1
:10F16E0000102700005573696E672044656661754F
:10F17E006C742073657474696E67733A004D313127
:10F18E0030002569206D696E2C202569207365631A
:10F19E00004D31303920496E76616C696420657896
:10F1AE0074727564657220004D31303520496E766B
:10F1BE00616C696420657874727564657220004DA7
:10F1CE0031303420496E76616C69642065787472D2
:10F1DE0075646572200054524947474552454400B4
:10F1EE006F70656E005265706F7274696E67206520
:10F1FE006E6473746F7020737461747573003F0066
:10F20E006F6B0020703A0020693A0020643A0020AB
:10F21E00633A005400496E76616C696420657874B7
:10F22E007275646572004163746976652045787401
:10F23E0072756465723A20004D32390058595A453C
:10F24E00000001001A0019000A000000FFFF1C0058
:10F25E001B000A000100FFFF170016000A00020043
:10F26E00FFFFFFFFFFFF04000E00180015000A004D
:10F27E0003000000010002000200000000008036C2
:10F28E007436056B537465707261746520746F20EB
:10F29E0068696768203A2000504944204175746FB0
:10F2AE0074756E6520737461727400504944204108
:10F2BE0075746F74756E65206661696C65642E2059
:10F2CE00426164206578747275646572206E756D26
:10F2DE006265722E002F0043616E6E6F74206F7028
:10F2EE00656E20737562646972006175746F25694D
:10F2FE002E67004D3233202573004D3234004D38C9
:0AF30E003420582059205A204500F1
:00000001FF
